:020000040000FA
:040000006FD00400B9
:101000006F00507B000000000000000090200020D6
:10101000AA220020A9BDF9F56C23002000000000E1
:10102000000000006C230020902000200000000041
:101030000000000090200020000000009020002010
:101040000000000090200020902000209020002030
:101050009020002090200020242F00205E240020DB
:101060000000000090200020902000200424002098
:1010700090200020D22300209020002090200020EB
:101080009020002090200020902000209020002020
:101090009020002001A04111B7170040985F3AC688
:1010A000945F3247E39CE6FE3245410182800111A4
:1010B00013078008F337078093F787083EC20100C3
:1010C0000100B7170040930570052380B70413068D
:1010D00080FA2380C7040100010083C6B70493F699
:1010E000F60DA385D704238007049246F3A6068055
:1010F0000100010093760502D5CEF336078093F602
:10110000860836C4010001002380B7042380C70489
:1011100001000100B70614007D89558D88C70100C4
:1011200001000100010023800704A246F3A6068007
:101130000100010073370780137787083AC6010062
:1011400001002380B7042380C704010001000100CF
:1011500001003727004093061005A303D7802380A2
:101160000704B247F3A70780010001009307800836
:10117000F3B7078093F787083ECE01000100B71749
:101180000040130770052380E704130780FA2380CB
:10119000E7040100010003C7B70413670708A3852C
:1011A000E70423800704F247F3A70780010001004A
:1011B0000561828093760504BDC6F336078093F6F9
:1011C000860836C8010001002380B7042380C704C5
:1011D00001000100B7061400938606047D89558D31
:1011E00088C7010001000100010023800704C246F6
:1011F000F3A6068001000100733707801377870884
:101200003ACA010001002380B7042380C70401000B
:1012100001003727004093062005A303D7802380D1
:101220000704D24781B773370780137787083ACC12
:10123000010001002380B7042380C70401000100DE
:1012400098471367070C98C723800704E24719BF24
:101250000111814601468145114506CE97000000E7
:10126000E780005593078008F3B7078093F7870856
:101270003EC601000100B717004013077005238028
:10128000E704130780FA2380E7040100010003C785
:101290006704136717002383E70423800704B2471A
:1012A000F3A7078001000100F2400561828041112F
:1012B000814601468145114597000000E780404F77
:1012C00013078008F337078093F787083EC40100AF
:1012D0000100B7170040130670052380C70493066A
:1012E00080FA2380D70401000100FD552396B70240
:1012F00023800704A245F3A5058001000100733790
:101300000780137787083AC6010001002380C704CD
:101310002380D7040100010003C767041367170087
:101320002383E70423800704B247F3A70780010063
:10133000010001A0BD473305F50201007D1575FDD3
:101340008280411122C426C206C6AA8401446317C2
:101350009400B24022449244410182800504130566
:10136000803E420497000000E78000FD4180C5B741
:101370009305000273A04580824573901534924016
:101380002242B2424243D2436244F2440255925551
:101390002256B2564257D2576258F25806499649D9
:1013A000264AB64A464BD64B664CF64C065D965DD1
:1013B000265EB65E465FD65F09617300203041113C
:1013C000B7170040985F3AC6945F3247E39CE6FE49
:1013D000324541018280B71700401307000323887C
:1013E000E702854717170000232EF74273002030CD
:1013F000411122C406C637040020976000E0E78050
:1014000000D81C408297D5BF37370040834747003C
:101410009146BD8B6389D70099466394D700834773
:101420005740730020309736000083C6662C9387A0
:10143000160017360000230DF62A0347870097375A
:1014400000009387E71AB6972380E700B7E7040008
:10145000BC4F0946894517150000034565F482977E
:10146000C9B7B787004003C76700098B6309071036
:1014700003C777009306000313770703630DD708AC
:10148000173800000348586217360000130606613B
:101490000547B30606012380E60083C577001737AA
:1014A000000013072760429793F5F50F2300B7005C
:1014B00003C58700973500009385855EC295137537
:1014C000F50F2380A5000347070089451377F7032D
:1014D000630CB70C63E7E50A6306071A8545630CDE
:1014E000B7129737000083C7375C3307F60003470E
:1014F00007001377F70F19CB850793F7F70F0D4701
:101500006363F71A17370000A300F75AB787004044
:1015100009472383E700B787004083C77700E207C6
:10152000E18763DE07049737000083C7F757173753
:1015300000001307A7563E9785462300D7001737AC
:101540000000130727563E97930600032300D70099
:10155000173700001307C7543E97A146850723009D
:10156000D70093F7F70F0D476364F71417370000A0
:10157000A30CF752B787004009472383E7007300A5
:101580002030930610026300D70E930620026305F5
:10159000D70693060002E316D7F403C72702137792
:1015A000C70F13672700D5A803C767001377070481
:1015B00065CB03C7A702173800001308A82F1735FB
:1015C00000001305E526134707082385E70203C734
:1015D000A7021377370F136787002385E702814738
:1015E00013070004B305F5008C41B306F80091071A
:1015F0008CC2E399E7FEF5B503C7A70213470704BA
:101600002385E70203C7A7021377C70F13672700D5
:101610002385E702F9B503C767001377070449C3B9
:1016200003C76702173800001308881C173500002D
:101630001305C513134707082383E70203C767028F
:101640001377370F136787002383E7028147130758
:101650000004B305F5008C41B306F80091078CC275
:10166000E399E7FEBDBD03C7670213470704238361
:10167000E70203C767021377C70F136727002383A7
:10168000E70285B503C767001377070411CB03C7CB
:1016900027021377370F136787002381E70291B57D
:1016A000238006003DBD97370000A38F073EB9BDDC
:1016B00097370000A38A073E75BD230304801547B2
:1016C0002303E48001002302A480828083076480D6
:1016D000E3CE07FE23030480828083076480E3CE89
:1016E00007FE03454480828083076480E3CE07FEC3
:1016F0002302A4808280411126C44AC24EC006C67D
:101700001377F50BAD47AA892E899544630CF70032
:10171000194597000000E78080FA97000000E780F5
:1017200020FB8D444E8597000000E78040F9FD596D
:10173000FD1463983401B240A24412498249410128
:101740008280135509011375F50F97000000E7809B
:10175000E0F92209F1BF011126CC06CEB70408003A
:1017600097000000E780C0F6154597000000E7806D
:1017700000F597000000E78080F697000000E78002
:1017800000F62AC697000000E78080F43245937780
:10179000150089EB136515001375F50FF240E2444F
:1017A00005618280FD14E9F00145CDBF397126DC69
:1017B0004ADA4ED852D656D45AD25ED006DE62CE1F
:1017C00066CCB7E700E07D5783AA070022C603AACC
:1017D000470023A0E71823A2E718B7170040130714
:1017E00070052380E704130780FA2380E70483C78A
:1017F0004704930B75FFB684E20793FBFB0F854606
:10180000AA892E8B328937240040E187015763FA79
:1018100076016308D5008946130700026313D500DB
:101820000157D98F93F7F70FB71C00402382FC04B0
:1018300011472303E4801305F00F97000000E780B1
:1018400000E8094C97000000E78080E863657C159C
:10185000B7050700DA9537870700795563FEE50479
:10186000B3879500636AF704370B0800A94733EB89
:1018700065016395F90881E8814497000000E780DD
:1018800020E5268515A8DA85094597000000E78040
:10189000C0E605090345F9FFFD14050B970000009C
:1018A000E780C0E481C49377FB0FE5F79700000061
:1018B000E780A0EA69F17D55B7170040130770056E
:1018C0002380E704130780FA2380E70403C7470453
:1018D000418B2382E704F250B7E700E023A05711C1
:1018E00023A24711E25432445259C259325AA25AE1
:1018F000125B825B724CE24C21618280A547639B44
:10190000F90685691309F00FB3069900B3742B012A
:10191000B6941349F9FFB3749900856B3379690163
:10192000416B9387F9FFB3F7270199E363FC340117
:1019300093D94900C147E3E637FF3DBF0569C16957
:101940007D19D9B71305800D63886901130500025D
:101950006384790113051008CA8597000000E780A9
:10196000C0D997000000E78040DF31D54E99B3849D
:1019700034416DBFDA852D4597000000E780E0D740
:10198000CA94E30B99EE050997000000E78020D583
:10199000A30FA9FEFDB79387F9FF93F7F70F636DC8
:1019A000FC0C83C71C04130730086315F7063707C0
:1019B00008006361EB06B3079B00B706100063FBEA
:1019C000D704334BEB0089476399F9068980D549E1
:1019D000E38404EADA85094597000000E780E0D156
:1019E00011090327C9FF91472320E480030764807E
:1019F000E34E07FE23033481FD17EDFBFD14110BAD
:101A000081C49377FB0FE9FF97000000E780E0D4E3
:101A100061F155B5B717004003C75704B707080071
:101A20001377070219E3B78707007955E376FBE8D8
:101A300033079B00E3F9E7F841B58547E380F9F008
:101A4000DA852D4597000000E78020CB9389F4FFCD
:101A5000E38404E297000000E78060C893F7390050
:101A600091EB832604800327090093074900E3963E
:101A7000E6E03E89CE84D9BFB5476399F9001305E6
:101A8000900B97000000E78080C3FDB3B1471305BA
:101A9000B00AE388F9FE99476397F904B70508008F
:101AA000B365BB002D4597000000E78000C5814469
:101AB0008D4BA14997000000E78060C263967401D6
:101AC000832704802320F9008504E39534FF8327CE
:101AD000048013172B01635507002312F90069BB1B
:101AE0002322F90051BB9D47639FF90281451305ED
:101AF000B00497000000E78040C0BD4423200900E7
:101B000023220900FD5997000000E78040BD93F7AC
:101B10007400CA9703C70700FD14398D2380A700FE
:101B2000E39334FF91BBA1476397F9069700000048
:101B3000E780A0C28144630D0B008D479304C0036E
:101B40006308FB009304000563048B0193044004C5
:101B50001375C507E30295D2194597000000E78089
:101B600000B697000000E780A0B60545970000008A
:101B7000E780E0B4268597000000E78020B709459C
:101B800097000000E78080B697000000E780E0BC87
:101B9000E31405CE0DB39147639FF900130560066A
:101BA00097000000E780A0B197000000E78040B2F6
:101BB00013059009F9B5E38109CCF1547DB9BD66EF
:101BC0000147173600001306660B938606A6854567
:101BD0008347060093F7F70F91C382800507E3F967
:101BE000E6FE97370000238BB708DDB77D16620647
:101BF000618693178601E18763D4070001458280DF
:101C0000931726003307F500AE9718439C4363E70C
:101C1000E7007D16E37FF7FC7D55828005458280D5
:101C2000FD15E205E18513978501618793F7F50FAF
:101C300063480700FD15139725002A97584365D779
:101C4000138517006205618582803308B5021C4246
:101C500083A80600B335B502C29733B50701AE9825
:101C6000469585486367B5006394A50063E3070163
:101C700081480C43C6950CC388C21CC28280814730
:101C80001397870161876343B7008280139727000A
:101C90002A97232007008507E5B7814701479396D8
:101CA0008701E18663C5B6001335170082809396DD
:101CB0002700AA9694428507558FD5B793D75540EC
:101CC0008A07AA979C4305453315B5007D8D828010
:101CD00017F3FFDFE702A33D2A8497000000E780A7
:101CE00060F405C5931725003E940327C4FF814780
:101CF00011EB7D1516053E954205418517F3FFDF73
:101D00006700233D05838507E5B70145C5BF8147CA
:101D10001397870161876343C70082801397270069
:101D2000B386E50094422A97850714C3D5B77D167C
:101D300062066186014793178601E18763D5070034
:101D400013351700828093172600B306F500AE976F
:101D500094429C437D16B58F5D8FF1BF8A05AA958D
:101D600001476363B500828083A6C5FFF11593D751
:101D70001600D98F9CC11397F601E5B72A83014855
:101D8000014701456343D7008280B387050183A8DB
:101D90000700B30706019C43C697AA976384F8001F
:101DA00033B517010507B3080301620723A0F80044
:101DB00061871108C1BF2A8301478147014563C379
:101DC000D70082803388E50083280800330EE600C0
:101DD000032E0E003388A8403308C84163840801ED
:101DE00033B508018507B308E300E20723A0080123
:101DF000E1871107E9B717F3FFDFE702432B011172
:101E0000B286B2842E86AA850A8597000000E780F4
:101E1000C0FA2A84A6850A8597000000E78020E89A
:101E200033348000060413351500018D056117F366
:101E3000FFDF6700032A17F3FFDFE702C324411126
:101E4000AA89AE8A328BB68402C202C402C6014499
:101E5000131C8401135C8C4163499C02939B140006
:101E6000FD1B0549138CF4FFF15C33048901620406
:101E700061846340740792478E04CE9423AEF4FECF
:101E8000410117F3FFDF6700832313192400B30B0D
:101E90002B01014A93172A00D69783A50B0088438C
:101EA00078003400500097000000E78040DA050A0F
:101EB00093178A01E187F11BE35EFCFC92474E9980
:101EC00005042320F900A2473EC2B24702C63EC421
:101ED00041B7131A8901135A8A41131D240093171D
:101EE0008A01E18763CF970092470A044E941CC091
:101EF000A24705091379F90F3EC2B24702C63EC494
:101F0000ADB7B3079A0313152A0056950841780018
:101F100034005000050AEA97DA978C4397000000D6
:101F2000E780E0D26DBF0000197106C212C416C668
:101F30001AC81ECA22CC26CE2AD02ED232D436D6E9
:101F40003AD83EDA42DC46DECAC0CEC2D2C4D6C6D9
:101F5000DAC8DECAE2CCE6CEEAD0EED2F2D4F6D6C9
:101F6000FAD8FEDA971500009385458B8841E70083
:101F7000050092402242B2424243D2436244F244BC
:101F8000025592552256B2564257D2576258F258CD
:101F900006499649264AB64A464BD64B664CF64CFD
:101FA000065D965D265EB65E465FD65F096173008C
:101FB00020300000972100209381C1041751002098
:101FC0001301418417F5FFFF130505049705002051
:101FD00093854503171600201306C6FD63FAC50056
:101FE0008322050023A0550011059105E3EAC5FEF3
:101FF00017050200130585C797150020938585FBFB
:10200000171600201306066563FAC5008322050033
:1020100023A0550011059105E3EAC5FE1715002020
:102020001305456397450020938545116377B500F7
:10203000232005001105E36DB5FEFD42739002BC3F
:102040008D4273904280B722000093828288739001
:102050000230970200209382E2FA93E232007390FA
:102060005230975200009382828C739012346FB07A
:10207000347973002030397101436EC619A039716B
:1020800041536AC866CA62CC5ECE19A03971015349
:102090005AD056D252D44ED64AD826DA22DC06DEA0
:1020A00033016140828241114AC026C222C406C661
:1020B0008282B24D4101024D924C224CB24B410101
:1020C000024B924A224AB2494101024992442244B7
:1020D000B240410182803D432A876373C3029377F4
:1020E000F700BDEFADE5937606FF3D8ABA960CC3C7
:1020F0004CC30CC74CC74107E36BD7FE11E282808B
:10210000B306C3408A069702000096966780A60031
:102110002307B700A306B7002306B700A305B7003F
:102120002305B700A304B7002304B700A303B70037
:102130002303B700A302B7002302B700A301B7002F
:102140002301B700A300B7002300B700828093F5F6
:10215000F50F93968500D58D93960501D58D61B7C2
:10216000939627009702000096968682E78086FA6B
:102170009680C1171D8F3E96E374C3F8A5B73367E9
:10218000B500FD530D8B79E7B7877F7F9387F7F70E
:1021900010419441B372F6003363F600BE92B3E28D
:1021A00062006397720C6318D6065041D441B37233
:1021B000F6003363F600BE92B3E262006398720ADF
:1021C000631BD60410459445B372F6003363F600E2
:1021D000BE92B3E262006391720A631ED60250455A
:1021E000D445B372F6003363F600BE92B3E26200E8
:1021F000639A72086311D60210499449B372F600CB
:102200003363F600BE92B3E2620063937208510535
:10221000D105E30FD6F61317060193970601631C49
:10222000F7001357060193D706013305F74093755E
:10223000F50F91E982804183C1833305F74093759F
:10224000F50F91E182801377F70F93F7F70F3305BE
:10225000F74082800346050083C605000505850515
:102260006313D60065FA3305D640828011059105C7
:10227000E312D6FE014582802105A105E31CD6FCB0
:10228000014582803105B105E316D6FC0145828007
:102290004105C105E310D6FC01458280B717004017
:1022A00003C777051377E70FA38BE704130700F83D
:1022B000A38DE7043D47238CE70413075003A38C49
:1022C000E70403C7A7051377D70F238DE7048280A0
:1022D000B717004003C7E7020D8941111377C70FF5
:1022E000498F93068008F3B6068093F6860836C6B3
:1022F00001000100930670052380D704930680FA3D
:102300002380D704010001002387E702238007040C
:10231000B247F3A70780010001004101828041110B
:102320002A83014E930E407E130F0019930F40062F
:1023300063E56E129308001913034006B378150382
:10234000854E0D4FA14F337365020D89133515006E
:1023500063EFBE121308F6FF7946729842081358CD
:1023600008013307C70213D61700BE07329761462C
:10237000B3F6C60213068070B386C6023697A1660E
:10238000F58F42075D8FB716004083C7F60293F7BB
:102390000708A303F1000346710083C7F60293F711
:1023A0000708E394C7FE83477100B716004093F710
:1023B000F70F6388071293078008F3B7078093F736
:1023C00087083EC401000100B7170040930670055E
:1023D0002380D704930680FA2380D70401000100EC
:1023E00023AA070383C6170393E60608A388D70228
:1023F00023800704A247F3A70780010001001166AC
:10240000B71700407D16D45BC85F93854703A98E3C
:10241000F18EF5FA93068008F3B6068093F68608E7
:1024200036C601000100930670052380D704930689
:1024300080FA2380D7040100010098C103C7170365
:1024400013670704A388E70223800704B247F3A7B2
:10245000078001000100410182807D133368E3039E
:102460009308E016630E08003368F3039308D01650
:10247000630808009378330093B818009388D8163F
:1024800033081E01131E0801135E0E0155B5639338
:10249000E5030548638608000148630303002A88B2
:1024A00071087298FD15131E0801C205135E0E0116
:1024B000C18179BD13F8150063F4BF007908D5B761
:1024C00013381800E5BF83C7F60293F70708A30384
:1024D000F1000346710083C7F60293F70708E394FF
:1024E000C7FE8347710093F7F70FF1DFE9B531714C
:1024F0004AD966CB06DF22DD26DB4ED752D556D32E
:102500005AD15ECF62CD6AC96EC7AA8C02D8971025
:102510000000E78020B12A8993078008F3B707807D
:1025200093F787083EDA01000100B7170040130750
:1025300070052380E704130780FA2380E704010075
:10254000010003C7F7021377770FA387E70203C7DA
:10255000F70213678700A387E70223800704D25797
:10256000F3A7078001000100054597000000E78000
:1025700060D6130780C13347E902116A93070AE85E
:1025800093065002BD69930BA004814A014B1304CA
:102590008008930470057D1AB347F9023307D70208
:1025A0003EC0FD873ECC938709A69309803E334702
:1025B000F7023AC27D873AC4334739038549B39954
:1025C000990193D93940B306D702B30B7703B3C649
:1025D000F602B3CBFB0236C6FD8636C893D6FB4166
:1025E00036CEB7460F00938606243349D902856656
:1025F000938606FAB3969601B389E90213076055EC
:102600003309D90293060010B389E9023349D9028C
:10261000B3C9F9029316390036CA37190040FD864E
:1026200036D0930D090493D7F9413ED2F336048096
:1026300093F6860836DC01000100930770052380BD
:10264000FD00930680FA2380DD000100010083462F
:10265000390593F6860FA309D9048346390593E615
:102660001600A309D90423800D00E256F3A60680C4
:1026700001000100130C80FA116DF336048093F60B
:10268000860836DE01000100930770052380FD00F7
:1026900023808D010100010083463905216693E600
:1026A0000602A309D90483560905B3E6A601231837
:1026B000D90483560905D18E2318D90423800D002F
:1026C000F256F3A60680010001008346390593F611
:1026D00006026381061A03463905218A6DDE081851
:1026E00097100000E7800098733604801376860800
:1026F000B2C20100010023809D0023808D010100F2
:102700000100B717004003C637051376F60DA389FD
:10271000C70403C6370513660602A389C704835698
:1027200009052166B3E6A6012318D90483560905D5
:10273000D18E2318D90423800D009646F3A6068077
:10274000010001008346390593F60602638B0614E7
:1027500083463905A18AEDFE97000020E780A0930B
:10276000AA8636D497000020E780E092A256E30ABA
:10277000D5FE835609054255B3E6A6012318D904B0
:1027800097100000E780C08F83463905A18AEDDEEF
:10279000035609058346290582473376CA00B306E6
:1027A000DA0293D5F641B296B388F640E24733B8E1
:1027B000C6002E983308F840A247B3B61601330876
:1027C000D84063C70701631DF800924763FA1701F9
:1027D000C247634FF80E63950701B24763EAF80EEC
:1027E000894663E9660FF2469315180013D3F80182
:1027F0005E8613951800B365B30042D646D497B0F1
:102800000100E780C06F3258050B137BFB0F634755
:102810000001631A0838A2586387083813081500A6
:10282000B336A800B69513D6F5013298B336C80072
:10283000AE9613581800FE06B3E606017336048000
:1028400013768608B2C60100010023809D00238014
:102850008D01010001000356C902B296C206C18271
:102860002316D90223800D00B646F3A60680010088
:10287000010021B5F336048093F68608B6C0010046
:10288000010023809D0023808D010100010083460B
:10289000390593E60602A309D90423800D00864674
:1028A0000DB5F336048093F68608B6C40100010026
:1028B00023809D0023808D0101000100834639059E
:1028C00093E60602A309D90423800D00A646BDB5F0
:1028D000E30B0BF0F336048093F68608B6C80100CC
:1028E0000100930680FA23809D002380DD00010013
:1028F00001008346390593F5FC0F93F6860FA30973
:10290000D90483463905CD8EA309D90423800D004F
:10291000C646F3A6068001000100130580FA0346AF
:102920003905930639051D8A631C96297336048080
:1029300013768608B2CC01000100130680FA2380CA
:102940009D002380CD000100010003C60600137620
:10295000F60D2380C60003C6060013660602238018
:10296000C600835609051166D18E2318D9048356F3
:1029700009052166D18E2318D90423800D00E6466F
:10298000F3A6068001000100130680FA834639058C
:1029900093F606026380062683463905130C390533
:1029A000A18AFDDA081897000000E780A06BF336D3
:1029B000048093F68608B6D001000100930680FAE1
:1029C00023809D002380DD000100010083460C0070
:1029D000116693F6F60D2300DC0083460C0093E6A7
:1029E00006022300DC0083560905D18E2318D90482
:1029F000835609052166D18E2318D90423800D0042
:102A00008656F3A6068001000100130680FA83466D
:102A1000390593F60602638A062083463905A18AA2
:102A2000EDFE97F0FF1FE78000672A8C97F0FF1FED
:102A3000E7806066E30C85FF835609051166425501
:102A4000D18E2318D90497000000E7806063834685
:102A5000390513063905A18AFDDAF336048093F6A9
:102A60008608B6D401000100930680FA23809D00F9
:102A70002380DD00010001008346060093F6F60D79
:102A80002300D60023800D00A656F3A60680010081
:102A900001008356090503462905D247B376DA00BB
:102AA0003306CA021305800C9355F6413696330D52
:102AB000F6408257333CD6002E9C3336A601330CA9
:102AC000FC40330CCC403308850392564E86B33518
:102AD000A5033305A503C29597B00100E780204206
:102AE00063468001631E0C16630C0D161306150059
:102AF0003335A6002E959356F5013696B335D6009C
:102B0000AA959396F50105828585D18E6346B0001E
:102B1000639D051A638B061A0356C9021582330595
:102B2000D6003336C500B2956348B00063910524E2
:102B30001306F00F637DA622894663F356159307AB
:102B40008008F3B7078093F78708BED6010001001D
:102B500037170040930770052300F704930780FAA6
:102B60002300F704010001008356C702896781171B
:102B7000D58FC207C1832316F70223000704B65777
:102B8000F3A7078001000100FA506A54DA544A5949
:102B9000BA592A5A9A5A0A5BFA4B6A4CDA4C4A4D8D
:102BA000BA4D296182801308F5FF3335A800FD1561
:102BB0002E951356F5013298B336C800AA9695B9EA
:102BC000F336048093F68608B6CA0100010023801C
:102BD0009D002380AD000100010083463905CD8EA4
:102BE000A309D90423800D00D646F3A60680010070
:102BF000010035B3F336048093F68608B6CE0100A3
:102C0000010023809D002380CD0001000100834648
:102C1000390593E60602A309D90423800D00F64680
:102C2000F3A606800100010095B3F336048093F605
:102C30008608B6D20100010023809D002380CD00CC
:102C4000010001008346390593E60602A309D90471
:102C500023800D009656F3A606800100010045BBB7
:102C60009306F5FF33B5A600FD152E959355F50196
:102C7000AE96B3B5B600AA951396F501858269B5EF
:102C8000F336048093F68608B6D801000100930657
:102C900080FA23809D002380DD000100010083561F
:102CA000C9020566011693F6F60FD18EC206C182DF
:102CB0002316D90223800D00C656F3A60680010014
:102CC0000100850A93FAFA0F95B233E6B60045C2C1
:102CD0000356C9023305D0403338A000B305B040D5
:102CE000B385054115826345B000D1E16371A60843
:102CF000894663F0560593078008F3B7078093F77A
:102D00008708BEDA01000100B717004013077005FD
:102D10002380E704130780FA2380E7040100010001
:102D200003D7C7027D8B2396E70223800704D6577B
:102D300081BDF336048093F68608B6DC01000100FD
:102D4000930680FA23809D002380DD0001000100AE
:102D50008356C9020566011693F6F60FD18EC20698
:102D6000C1822316D90223800D00E656B9B7930716
:102D70008008F3B7078093F78708BEDE01000100E3
:102D800037170040930770052300F704930780FA74
:102D90002300F704010001000356C7029397560071
:102DA000B297C207C1832316F70223000704F65720
:102DB000C1BB914763EEB70217D701001307C7FFE6
:102DC0008A05BA959C41BA978287B717004003A736
:102DD000470B1345F5FF698F23AAE70A03A7070BE3
:102DE000698F23A8E70A03A7070A798D23A0A70AFA
:102DF0008280B717004083A6470B1347F5FFF98E73
:102E000023AAD70A83A6070B558D23A8A70A83A652
:102E1000070A758F23A0E70A8280B717004003A72F
:102E2000470B498F23AAE70A03A7070B1345F5FFB2
:102E300045BFB717004083A6470B1347F5FF758FB3
:102E400023AAE70A03A7070A598D4DB7B717004011
:102E500003A7470B498FEDB7914763EEB70217D72A
:102E600001001307A7F68A05BA959C41BA97828795
:102E7000B717004003A7470D1345F5FF698F23AA35
:102E8000E70C03A7070D698F23A8E70C03A7070C1E
:102E9000798D23A0A70C8280B717004083A6470D29
:102EA0001347F5FFF98E23AAD70C83A6070D558D7E
:102EB00023A8A70C83A6070C758F23A0E70C82809C
:102EC000B717004003A7470D498F23AAE70C03A7B4
:102ED000070D1345F5FF45BFB717004083A6470D03
:102EE0001347F5FF758F23AAE70C03A7070C598D2D
:102EF0004DB7B717004003A7470D498FEDB779715C
:102F000022D43714004026D24AD0035924028354D5
:102F1000040206D64209C2044ECE52CC56CA1359F8
:102F20000901C1802DE11379F9F793F4F49F420967
:102F3000C20413590901C18093078008F3B70780C1
:102F400093F787083EC40100010093077005230032
:102F5000F404930780FA2300F40401000100231114
:102F600024032310940223000404A247F3A707803C
:102F700001000100B250225492540259F249624AAF
:102F8000D24A45618280B7F5070081463000B1051D
:102F9000194597000020E7806081A2471397270119
:102FA000E34A07FC1369090893E404409309800885
:102FB000F3B7098093F787083EC001000100930A28
:102FC000700523005405130A80FA2300440501000C
:102FD00001002311240323109402230004048247D8
:102FE000F3A7078001000100294597F0FF1FE78044
:102FF0006034F3B9098093F989084EC201000100D9
:1030000023005405230044050100010083570402F6
:1030100093E707202310F402230004049247B9B772
:10302000B71700408847420541819377050491EB2B
:103030009377F5013755E801130505803345F5020F
:1030400082809377050C130700046397E70093775A
:10305000F50137459C1CCDB72165130505D082804D
:1030600037E700E01C435443A183E206D58F1CC11F
:10307000FD572320F7182322F718828013178500A5
:10308000B7E700E023A0E710618123A2A7108280A8
:10309000B7F700E08847CC47828081473737004048
:1030A000A14663C4C700328582800345B740E38EE2
:1030B000A6FE3385F5000345050085072304A740D8
:1030C000CDB7970700209387E7EE9C431737002082
:1030D0001307C7063E95636EE500173700201307F8
:1030E00067526368A700170700202325A7EC3E85D9
:1030F0008280FD57EDBF8280411122C406C62A841A
:1031000097000000E78000F22947B307E502B240CC
:103110008D83B3D7870222449507B3D7E7023737A9
:103120000040C207C1832316F70041018280716508
:1031300041111305052006C697000000E78000FC3A
:10314000B7370040130770F82381E7000D47A381CC
:10315000E70013070004A380E70005472387E70083
:10316000B2404101828037370040834727001A056B
:1031700093F7F703C98F93F7F70F2301F7008280C6
:10318000B737004003C7170019C9D98DA380B7000E
:1031900003C70700136787002380E700828093C579
:1031A000F5FFF98DA380B7008280AE872A87B736F6
:1031B000004021463738004089E7170300006700C8
:1031C000C3F383C8B600E30916FF05078348F7FF7A
:1031D000FD17C20723041801C183F9BF411122C49E
:1031E00006C62A8497000000E780C0E32947B3079A
:1031F000E502B2408D83B3D7870222449507B3D747
:10320000E70237370040C207C1832316F740410168
:103210008280716541111305052006C697000000E4
:10322000E78000FCB7370040130770F82381E740C0
:103230000D47A381E74013070004A380E74005473B
:103240002387E740B24041018280CC41411106C64C
:10325000328503C6150083C5050022064D8E420641
:103260008D654186138875A2630C0611634BC804F3
:10327000138845A26300060D634AC800938535A2F2
:103280006301B6082390060029464DA0138855A275
:103290006305060D938565A2E316B6FE8D451D46B2
:1032A00063E6E5081146198E63F3C7003E86B7E76B
:1032B00004002390C600FC4797D50100938545B3D1
:1032C0009DA0138895A263030611634E060D138813
:1032D000A5A263000613938505A5E315B6FA9945E3
:1032E0001D4663E5E504198E63F3C7003E86B7E724
:1032F00004002390C600FC47970500209385C5D5A0
:103300001DA09D451D4663E3E5022146198E63F32A
:10331000C7003E86B7E70400FC472390C600970528
:1033200000209385A533BA9582970146B240328535
:1033300041018280AD451D46E3EAE5FE3146198E26
:1033400063F3C7003E86B7E704002390C600FC473E
:1033500097D50100938545ACF9B7B1451D46E3E724
:10336000E5FC3546198E63F3C7003E86B7E70400D7
:103370002390C600FC4797D501009385E5AA65B761
:103380008D451D46E3E4E5FA1146198E63F3C70047
:103390003E86B7E704002390C600FC4797D501009E
:1033A0009385C5A549B78D451D46E3E1E5F811466E
:1033B000198E63F3C7003E86B7E704002390C6006A
:1033C000FC4797D501009385E5A7B1BFA5451D46EC
:1033D000E3EEE5F42946198E63F3C7003E86B7E7AE
:1033E00004002390C600FC4797D501009385C5A132
:1033F0001DBFB5451D46E3EBE5F23946198E63F373
:10340000C7003E86B7E704002390C600FC4797D567
:1034100001009385E59C01BFB7E7040003A30713F0
:1034200097060020938646C24146A5451705002011
:10343000130585B802832D455DE703C505000947DF
:10344000631FE50803A84500411106C6034718009D
:1034500032850346080022074168518F930828FEF1
:103460006307170563E9E800051863030703239062
:103470000600294591A8130648FE630AC7041518DB
:10348000E31707FF15463E87637BF600154701A843
:10349000130600023E876374F60013070002B7E7C5
:1034A00004002390E600FC471316070111A83E868E
:1034B00091C30546B7E70400FC472390C6004206C7
:1034C000CC45418282970145B2404101828013067A
:1034D00000083E87E375F6FC13070008C9B7239080
:1034E0000600054582808280416779176304E50400
:1034F000411122C406C685472A84639FF500B7E7B9
:10350000040022852244B24003A3871397050020BC
:103510009385052F4101028389476399F500B7E739
:10352000040083A7070B8545829771D9B2402244D6
:10353000410182808280797122D452CC2E842A8AE1
:1035400097D501009385059217D5010013050594C1
:1035500006D63AC626D24AD0B68432894ECE97B025
:103560000100E78000E5A68517D501001305059346
:1035700097B00100E780E0E3294597B00100E780BC
:1035800020E88347840093F70702E1E783490400BA
:103590008947054532476396F908544083C71600AA
:1035A00083C60600A207D58FC166138616FE638CFC
:1035B000C7028D16638FD7068D66938626902945A0
:1035C0006391D706B7E70400A285225403A34714EA
:1035D000B250F249A6864A86925402595285624AEE
:1035E0008547456102832D450DEF93070002354560
:1035F00063E99702B7E70400FC474844130600025A
:10360000CA858297814997070020938727209C438A
:10361000014581CB9C4391C74E852686CA858297FA
:103620000145B250225492540259F249624A45610E
:1036300082802D457DF79307700F3545E3E397FEB4
:10364000B7E70400FC4748441306700FCA85829709
:103650005DBF2145F9B7411122C437E40400832737
:10366000841326C2AA84416506C697050020938567
:1036700025197D1582978327C40A170500001305B5
:10368000E5E68588829795C0032304132244B2405F
:103690009244970600209386A6AD4146C54517057E
:1036A00000201305E59B41010283B240224492446D
:1036B00001454101828019C59707002023A8A7145E
:1036C00001458280454582801147636AA70A97C6F3
:1036D00001009386E6770A0536951841411106C622
:1036E0003697AE87B2850287130700026145639D56
:1036F000E700B7E70400FC471306000217050020A7
:10370000130545F682970145B24041018280054785
:103710006145E39BE7FEB7E70400FC470546170554
:103720000020130525F6F9BF1307700F6145E39DCF
:10373000E7FCB7E70400FC471306700F17050020ED
:10374000130585F4C1B7130700086145E39EE7FA46
:10375000B7E70400FC47130600081705002013050F
:1037600025024DB715476145E390E7FAB7E7040036
:10377000FC471546170500201305C50861B7094524
:103780008280411126C2B7E4040083A7C41322C477
:103790004AC006C62E8497050020938565062A89AF
:1037A0008297058905C5970700209387678B83D784
:1037B000A70BA28503A3440D2310F4002244B240BA
:1037C00092444A850249014641010283B2402244A3
:1037D000924402494945410182809707002023898C
:1037E00007029707002023A70702B717004003A787
:1037F000070CB706C0FFFD16758F23A0E70C03A7C3
:10380000070DB7064000558F23A8E70C03A7070C48
:103810003D9B23A0E70C03A7070D1367070123A80F
:10382000E70C8280B717004003A5470C83A7470C1D
:10383000598113451500C18B058999E3136525004E
:103840009707002083C7C7FC6380A7029707002063
:103850002380A7FC11C9970700209387A7FB03A328
:1038600007006303030002838280114517F3FFFF03
:10387000670023C8411193962500AA852D4506C6E9
:1038800097F0FF1FE78080F2B2400145410182803E
:10389000011122CC06CE3714004026CA4AC84EC6B3
:1038A00052C483447405034AB4058349840503491B
:1038B000940597F0FFFFE780A09E8347A40593F44B
:1038C000F40F137AFA0F93E71700230DF40493F91A
:1038D000F90F1379F90FB717004003C7A705058B38
:1038E0006DFF03D5C705A38D4705238C3705A38C32
:1038F0002705A38B9704F2406244D2444249B2495F
:10390000224A0561828041119397050122C406C6AF
:1039100026C2C1872E8463DC0700B7E40400FC5490
:10392000829719C1BC5482972165218D15A893F700
:10393000150013C515008DE793F725009DC7970067
:103940000000E78060EEB7E70400BC4F1306000AF2
:10395000894517050020034565EC8297134524002F
:10396000B24022449244410182809397250163D85A
:103970000702B7E4040083A7C41E829797000000E3
:10398000E780E0EEBC4C3756070013060630896529
:1039900017050020034585E88297096579B7939755
:1039A00015010145E3DE07FA17C5010013050557A8
:1039B00097B00100E780C0B7B7E70400BC4F13061B
:1039C0000064916517050020034545E58297116560
:1039D000A9BF2D71232A9110FD74E98C232C81102D
:1039E00023282111232631112A84AE893289930696
:1039F00000100A86A6852D45232E111097F0FF1F73
:103A0000E780C0DA13154401B7E70400FC47518191
:103A10000A0513962900CA850A958297A6858566A8
:103A20000146254597F0FF1FE78040D80A86A68506
:103A300093060010294597F0FF1FE78020D78320C9
:103A4000C111032481118324411103290111832908
:103A5000C11015618280B7F7070003C70701411144
:103A600006C622C426C24AC0A547631DF7009700B8
:103A70000000E78040F6B2402244924402490145EA
:103A80004101828013942500AA843289A286AA85E6
:103A90000146254597F0FF1FE78040D1A2864A8660
:103AA000A685294597F0FF1FE78040D0E9B71D7133
:103AB000A2CC37E404005C5C485886CE494697C5E2
:103AC000010093852541829711E917C5010013056F
:103AD000A54197B00100E780A0A501A0B7F600E0DE
:103AE000795798CAFD57DCCA0567B7E700E023A0FD
:103AF000E7101306F00290C223A0E71801000100AE
:103B00003707002018471306000481459706002058
:103B100023A4E6D04157A38AE7403C440808829793
:103B2000970700209387476C3EC885671387074037
:103B3000231AE1001D673ACC370701051307071068
:103B40003ACE938757D11307B00F2310E102231207
:103B5000F102054797F7FFFF9387C7532301E1025F
:103B60003ED817070000130727D197070000938757
:103B700067D2B7F50700BAC23EDC1707000013078B
:103B8000C7ED97070000938787CE81463000E10597
:103B90001945BAC43EDE97F0FF1FE78020C1180820
:103BA0008147994630003E96034606008507050783
:103BB000A30BC700E398D7FEC24791C70357410143
:103BC00085676373F70001A0B7E7040083A7470A7E
:103BD00008088297AA8511C917C501001305053287
:103BE00097A00100E780E07C01A0F64066442561D3
:103BF0008280411126C2B7E4040083A7040806C6E8
:103C000022C417050000130545D082971704002031
:103C10001304C4C02300A40097000000E7808002C2
:103C200097000000E780A0BB03450400224403A3E3
:103C30008405B24092441306003289654101028333
:103C4000797106D622D413078008F337078093F7DB
:103C500087083EC201000100B717004093057005B8
:103C60002380B704130680FA2380C70401000100F3
:103C700083C6F70293F6A60FA387D7022380070413
:103C80009246F3A606800100010073370780137780
:103C900087083AC4010001002380B7042380C704C9
:103CA0000100010003C7F70213672700A387E7029B
:103CB00023800704A247F3A7078001000100054500
:103CC00097E0FFFFE780006197000000E78020BADF
:103CD000014781468147054685451305407E97E0AB
:103CE000FFFFE780006437E404003C44680051466D
:103CF00081458297B707C0A83EC8B787E803938776
:103D000007D03ECA97E7FF1F9387676B3EC67C5874
:103D100068008297B250225445618280411197D544
:103D200001009385E58517C501001305251606C614
:103D300097A00100E780E06717D501001305059DF6
:103D400097A00100E780E066B2402945410117A332
:103D500001006700E36A411197D5010093858583CF
:103D600017C501001305851206C697A00100E7805C
:103D7000406417D501001305259897A00100E7803E
:103D80004063B2402945410117A301006700436722
:103D9000411122C406C6834705002A849DC797D5D2
:103DA00001009385E58417C501001305250E97A032
:103DB0000100E78000604C4017D50100130545A3C2
:103DC00097A00100E780E05E3DA058410DEF97D538
:103DD00001009385E58117C501001305250B97A008
:103DE0000100E780005D17D501001305E5A197A04C
:103DF0000100E780005C2244B2402945410117A33D
:103E000001006700E35FA1679386D7036313D702BE
:103E100097C501009385C57D17C5010013050507EA
:103E200097A00100E780E05817D501001305C59E53
:103E30007DBFED0797C501009385857B17C5010000
:103E40001305C504631BF70097A00100E7806056C7
:103E500017D501001305859D59BF97A00100E78084
:103E600040554C4017D501001305459E91BF4111A7
:103E700097C501009385457317C50100130505011A
:103E800006C697A00100E780C052B2402945410113
:103E900017A301006700C356797122D426D24AD0F5
:103EA0002E842A898145B2844800714606D697E05F
:103EB000FFFFE780802297F7FF1F9387274CDC479F
:103EC00083D70700231421012313F100974000003A
:103ED000E78060769547A305F1009307401F3EC633
:103EE000FD572305A100230AF10097500000E78049
:103EF000C0882686A285480097400000E78080762B
:103F0000B250225492540259456182809717002082
:103F1000239F077C971700202388076CB7E70400CE
:103F2000BC47411106C641468145170500201305CF
:103F3000251A829797200000E780A056972000005E
:103F4000E780C031014597500000E780601B1707EC
:103F500000200347E7199307F00A6315F702930758
:103F6000F0F889451705002013058518170700206C
:103F70002300F71897070020A38C0716975000001E
:103F8000E780A04297500000E780604F81453705E9
:103F900004009707002023AB071297070020239502
:103FA0000712970700202382071297070020239308
:103FB000070A9707002023910708970700202394FA
:103FC000071097070020239D071097300000E78017
:103FD00060BA014597500000E780204697C5010070
:103FE0009385055F17C50100130545EA97A00100F9
:103FF000E780203C17D501001305858B97A00100B1
:10400000E780203BB2402945410117A3010067002A
:10401000233F411122C406C626C293F715002E8401
:10402000638F0710814617F6FF1F1306663285451A
:10403000170500200355050097C00000E78020A960
:1040400015C997C501009385655917C5010013056A
:10405000E5E397A00100E780C03517C5010013050F
:10406000A5FA97A00100E780C034294597A0010078
:10407000E780003997C501009385455617C50100B3
:104080001305C5E097A00100E780A03217C5010025
:104090001305C5F897A00100E780A031294597A036
:1040A0000100E780E03517F5FF1F1305252D5C455E
:1040B00005472390E70097300100E780A05997C596
:1040C00001009385A55117C50100130525DC97A0B4
:1040D0000100E780002E17C50100130565F597A0C4
:1040E0000100E780002D294597A00100E7804031BD
:1040F000930710F817070020230CF7FE97070020FE
:1041000083D707F317070020A304F7FE1705002045
:10411000130505FEA183914517070020230BF7FC2B
:1041200097070020A38707FC97500000E780E0274F
:1041300013451400B240224492444101828093F717
:104140002500E1C317070020035707F845CB970662
:1041500000209386A6F7944297C70100938747777C
:1041600017060020034666F6814517050020130553
:1041700025F697700000E780E0B4AA8441C197C596
:1041800001009385654C17C50100130525D097A044
:104190000100E7800022A68517C501001305C5EAC6
:1041A00097A00100E780E020294597A00100E78063
:1041B000202597070020239907F0930710F8170789
:1041C00000202307F7F29707002083D767E6170739
:1041D0000020A30FF7F0A18317070020230BF7F0AF
:1041E00091458D4717050020130585F0170700201E
:1041F000A301F7F097500000E780201B134524002F
:1042000015BF93F74500D1C397C501009385C543FA
:1042100017C50100130585C797A00100E780601945
:1042200017C50100130505E497A00100E780601899
:10423000294597A00100E780A01C930720F81707E5
:1042400000202307F7EA9707002083D7A7E0170786
:104250000020A30FF7E8A18317070020230BF7E83E
:10426000854717070020A306F7E897400000E7807E
:10427000C050170500201305A5E791459750000091
:10428000E780A0121345440075B593F78500A9C7D0
:1042900097C501009385453B17C50100130505BF70
:1042A00097A00100E780E01017C501001305C5DCE9
:1042B00097A00100E780E00F294597A00100E78063
:1042C000201497070020239107E097700000E780F3
:1042D00040AF13458400B9BD93F70501D1C38545AF
:1042E00017050020035505D797500100E78060614E
:1042F00097C501009385453517C50100130505B91C
:1043000097A00100E780E00A17C50100130505D852
:1043100097A00100E780E009294597A00100E78008
:10432000200E930730F8170700202303F7DC9707C8
:10433000002083D727D217070020A30BF7DA170531
:1043400000201305E5DAA1838D451707002023021D
:10435000F7DA97500000E780400513450401D9BB08
:1043600093F70502D1C797C501009385E52D17C5C1
:1043700001001305A5B197A00100E780800317C5D0
:1043800001001305E5D297A00100E78080022945CE
:1043900097A00100E780C006930740F817070020A8
:1043A0002308F7D49707002083D707C917070020F1
:1043B000A300F7D4A18317070020230CF7D2854769
:1043C00017070020A307F7D297070020239607C6F8
:1043D00097400000E780603A17050020130545D19B
:1043E000914597500000E78040FC1345040299B3C3
:1043F00093F70504FDC397C501009385E52417C510
:1044000001001305A5A897A00100E78080FA17C551
:104410000100130565CB97A00100E78080F92945CD
:1044200097A00100E780C0FD9707002083C747CC15
:104430001307700A6386E7061307800A638CE70890
:104440001307600A6393E704930760F817070020D7
:104450002300F7CA9707002083D7E7C61707002075
:10446000A308F7C8A183170700202304F7C88547CE
:1044700017070020A303F7C8B1451705002013054F
:1044800025C797500000E78040F297400000E78082
:10449000C02E1345040497070020239607C259B97C
:1044A000930770F8170700202304F7C4970700202C
:1044B00083D767C117070020A30CF7C2A183170792
:1044C00000202308F7C2854717070020A304F7C27E
:1044D000994565B7930780F8F1B793F7050801454B
:1044E000E38A07C497C501009385051617C5010027
:1044F0001305C59997A00100E780A0EB17C501003F
:10450000130505BE97A00100E780A0EA294597A002
:104510000100E780E0EE9307A0F8170700202309C9
:10452000F7BC9707002083D7A7BB17070020A3017C
:10453000F7BCA18317070020230DF7BA854717079B
:104540000020A308F7BA97070020239B07B89740DD
:104550000000E780802217050020130565B991450A
:1045600097500000E78060E413450408E1B641116C
:1045700022C497C501009385E5082A8417C5010068
:104580001305C59006C697A00100E78080E24C4065
:1045900017C501001305452397A00100E78060E1DE
:1045A000294597A00100E780A0E503470400930791
:1045B000F00F631FF70297C501009385A50417C587
:1045C00001001305A58C97A00100E78080DE4C4018
:1045D00017C501001305452097A00100E78060DDA5
:1045E0002244B2402945410117A30100670043E17D
:1045F000B240224441018280B1C1411122C417C599
:1046000001001305A5882E8497C50100938585FABE
:1046100006C697A00100E780C0D9A28517C5010092
:104620001305C52697A00100E780A0D82244B24018
:104630002945410117A30100670083DC82804111F5
:1046400022C426C22E84AA8497C50100938545F70B
:1046500017C501001305858306C697A00100E780F2
:1046600040D517C501001305252397A00100E78059
:1046700040D4294597A00100E78080D897C5010064
:10468000938505F4970700202396979A17B50100A4
:104690001305C57F854497070020239B87989707BC
:1046A000002023989798971700202392870497A0BB
:1046B0000100E78000D09715002083D5450317C57A
:1046C00001001305E51D97A00100E78080CE294574
:1046D00097A00100E780C0D297170020238697F0AB
:1046E00097200000E78080B7228597500000E78080
:1046F00020A1054597500000E78020D497F7FF1FC1
:104700009387C7C7DC4703D70700C167FD1763124C
:10471000F7022244B7E70400B240924403A387059E
:1047200017F5FF1F034505101306000A85454101D3
:104730000283B2402244924441018280011122CC82
:1047400037E404005C5C06CE354697C501009385CE
:1047500025FD17D50100130525B7829711E917B577
:1047600001001305657897A00100E78060DC01A0D7
:1047700097F7FF1F9387C70B3EC4B7F50700856700
:1047800093870780814617F6FF1F1306E609E105A8
:1047900019453EC697E0FF1FE78040017C4419465B
:1047A00097F5FF1F93854508170500201305C58A57
:1047B0008297340017F6FF1F1306060797C50100FE
:1047C0009385054817C5010013050549976000004A
:1047D000E78040242A841DCD97C501009385C5E557
:1047E00017B501001305856A97A00100E78060BC3A
:1047F000A28517C501001305A5F397A00100E78066
:1048000040BB294597A00100E78080BFF240624489
:104810000561828097E00000E780A08617C501004F
:10482000130505E897500000E780801897A0000066
:10483000E780E0DA97500100E780603F17F5FF1F3F
:10484000130545B097500100E780002817C5010007
:10485000130505E697500100E780E03F2A84975052
:104860000000E780C07E97000100E7804017978036
:104870000100E78060B097700000E78000D7976084
:104880000000E780C0F497300100E780A0D897C50A
:104890000100938565DA17B501001305255F19C876
:1048A00097A00100E780E0B0A28517C501001305BD
:1048B00065EAA1B797A00100E780A0AF17C5010086
:1048C000130585EB97A00100E780A0AE294597A0CE
:1048D0000100E780E0B297300100E78080B497F0F4
:1048E0000000E78040D355C985453705040097206F
:1048F0000000E780202897C501009385E5D317B510
:1049000001001305A55897A00100E78080AA17C5EC
:1049100001001305E5E797A00100E78080A929457C
:1049200097A00100E780C0AD97F7FF1F9387C7945A
:1049300083D7070017170020231BF7DA85471717BF
:1049400000202303F7CA97200000E78000B09720DB
:104950000000E780A09017150020035545D9974027
:104960000000E780E079054597500000E780E0AC63
:1049700097C50100938545CC17B501001305055176
:1049800097A00100E780E0A217C50100130585E2AA
:1049900097A00100E780E0A1ADB597C50100938520
:1049A000A5C917B501001305654E97A00100E78062
:1049B00040A017C501001305A5EF97A00100E780EF
:1049C000409F294597A00100E78080A3014569BF6A
:1049D000411122C437E404008327041A06C68297D3
:1049E00097400000E78080758327040817F5FFFFD4
:1049F00013056562829797F7FF1F2385A7E217F5D6
:104A0000FF1F1305A59797400000E780A0092244E7
:104A1000B240410117030000670083D2B7E70400EA
:104A2000FC471171A2DDCAD986DFA6DBCED72E8462
:104A300032892E86AA8517F5FF1F1305656B8297AD
:104A400017F7FF1F1307C76A834707009306800203
:104A50009387E70793F7F70FE3ECF610BA898A0715
:104A600017B701001307C74BBA979C43BA978287C1
:104A70008D4797C50100938565BE17B501001305E5
:104A8000E540630FF40097A00100E780809217B51E
:104A900001001305657B97A00100E7808091BDA40C
:104AA00097A00100E780E09017B501001305457B52
:104AB00097A00100E780E08F294597A00100E780DB
:104AC0002094930720F8114697F5FF1F93854562C0
:104AD0004A8517F7FF1F230DF76097F7FF1FA38A7B
:104AE000076097F0FFFFE780603B2A841DC997C5E8
:104AF00001009385A5B617B501001305253997A0C8
:104B00000100E780008BA28517B501001305057928
:104B100097A00100E780E089294597A00100E78080
:104B2000208E97C50100938565B317B50100130565
:104B3000E53597A00100E780C08717B50100130590
:104B4000257797A00100E780C086294597A001003E
:104B5000E780008B4165930730FA054697F5FF1F04
:104B6000938505597D1517F7FF1F2303F75897F015
:104B7000FFFFE780A0322A841DC997C501009385F5
:104B8000E5AD17B501001305653097A00100E7807A
:104B90004082A28517B501001305457097A001005A
:104BA000E7802081294597A00100E7806085B7E76D
:104BB0000400BC4F0566130606C8A14517F5FF1F84
:104BC000034545C68297FE506E54DE544E59BE5979
:104BD0001161828091476303F40297C501009385B8
:104BE000E5A717B501001305652A97900100E78036
:104BF000407C17B501001305E56E71BDB7E70400F1
:104C0000FC4F914517F5FF1F0345C5C1829797C516
:104C100001009385A5A417B50100130525279790DA
:104C20000100E780007917B501001305656D9790C5
:104C30000100E7800078294597900100E780407CDB
:104C400097400000E78060B3914535A48547630332
:104C5000F40297C50100938565A017B501001305FF
:104C6000E52297900100E780C07417B50100130595
:104C7000A56A15B597F7FF1F239E273DB7E70400E8
:104C80000566BC4F130606C8C1450DBF8D476303BB
:104C9000F40297C501009385659C17B501001305C3
:104CA000E51E97900100E780C07017B5010013055D
:104CB0006568D5B3930740F8114697F5FF1F9385B4
:104CC00025434A8517F7FF1F2304F74297F7FF1F75
:104CD000A381074297F0FFFFE780401C2A84E3048A
:104CE00005EE97C501009385659717B5010013057B
:104CF000E51997900100E780C06BA28517B5010008
:104D00001305C55997900100E780A06A294597903F
:104D10000100E780E06E45BD9147E31CF4F6B7E77C
:104D20000400FC4F9305000217F5FF1F034585AFF4
:104D3000829797C501009385659217B50100130509
:104D4000E51497900100E780C06617B501001305D0
:104D5000E55FF1BD894763E3870297C5010093854D
:104D6000E58F17B501001305651297900100E780E4
:104D7000406417B501001305A55E31BB97F4FF1F12
:104D800083C4243797F7FF1F83C7973697C5010061
:104D90009385C58CA20417B501001305250FDD8C82
:104DA00097900100E780E060A28517B50100130528
:104DB000655C97900100E780C05FC2042945979029
:104DC0000100E780E063C1849305D4FF939604015A
:104DD000C1824A8693F5F50F17F5FF1F130575314C
:104DE00097200000E780C0DCE35F90DC930750F879
:104DF00017F7FF1F230EF72E83C73900228697F57A
:104E0000FF1F9385E52E85074A8517F7FF1FA3022D
:104E1000F72E97F0FFFFE78060082A84E30505DAA4
:104E200097C501009385858317B501001305050615
:104E300097900100E780E057A28517C50100130590
:104E4000E5A3C9B5894763E3870297C50100938548
:104E5000E58017B501001305650397900100E78011
:104E6000405517B501001305A55235B19740000014
:104E7000E780A090A28517F5FF1F130565279740CF
:104E80000000E780805281B38D476303F40297B539
:104E900001009385A57C17B50100130525FF9790A8
:104EA0000100E780005117B5010013052550E5B654
:104EB000B76602000146B7750200054597E0FF1F7F
:104EC000E780C08E930760F817F7FF1F2302F722D1
:104ED00097F7FF1FA38F07209307000617F7FF1F01
:104EE000230AF720894717F7FF1FA305F72097F735
:104EF000FF1F2382072097F7FF1FA38E071EC147BE
:104F000017F7FF1F230AF71E930720F917F7FF1F54
:104F1000A304F71E314697F7FF1FA380A71E97F53E
:104F2000FF1F9385E51C4A8597F7FF1F2387071C02
:104F300097F0FFFFE78080F62A84E30605C897B55F
:104F400001009385A57117B50100130525F497900D
:104F50000100E7800046A28517B5010013058546CC
:104F600055B3B1476303F40297B501009385056F0C
:104F700017B50100130585F197900100E7806043A4
:104F800017B501001305C54539B6B7E70400FC4F56
:104F90009305000417F5FF1F0345C58882979730D6
:104FA0000000E780807DB145F9B5914763E3870252
:104FB00097B501009385856A17B50100130505EDC6
:104FC00097900100E780E03E17B501001305054307
:104FD000D9B497F4FF1F83C4E41197F7FF1F83C769
:104FE0005711A204DD8C8E04B77702006D14BE94B5
:104FF0002286A68517B5010013058541979001000B
:10500000E780203BB7E70400FC47228697F5FF1FA7
:105010009385550E2800829793160401C1823000B3
:10502000A685094597D0FF1FE78040782A8409C9E3
:1050300017B501001305853F97900100E780404FA9
:10504000930770F8194697F5FF1F9385650A4A85FF
:1050500017F7FF1F230EF70897F7FF1FA38C87088A
:1050600097F0FFFFE78080E32A84E30E05B497B54D
:1050700001009385A55E17B50100130525E1979002
:105080000100E7800033A28517B501001305053B39
:1050900095B99947630BF41297B501009385055CA8
:1050A00017B50100130585DE97900100E780603099
:1050B00017B501001305053AF9BA914763E3870272
:1050C00097B501009385855917B50100130505DCD7
:1050D00097900100E780E02D17B501001305053911
:1050E0005DBA97F4FF1F83C4E40097F7FF1F83C7DF
:1050F0005700A204DD8C8E04B77702006D14BE94B5
:105100002286A68517B50100130585379790010003
:10511000E780202AB7E70400FC47228697F5FF1FA7
:10512000938555FD2800829793160401C1823000B3
:10513000A6850D4597D0FF1FE78040672A8409C9DF
:1051400017B501001305853597900100E780403EB3
:10515000930780F8194697F5FF1F938565F94A85EF
:1051600017F7FF1F2306F7F897F7FF1FA38487F8A9
:1051700097F0FFFFE78080D22A84E30605A497B565
:1051800001009385A54D17B50100130525D0979013
:105190000100E7800022A28517B501001305453103
:1051A00095B699476303F40297B501009385054BC3
:1051B00017B50100130585CD97900100E780601FAA
:1051C00017B5010013054530F9B0B7E70400FC4FEF
:1051D0009305000417E5FF1F0345C56482979730C8
:1051E0000000E7808059994579B18D476303F40247
:1051F00097B501009385854617B50100130505C9CC
:1052000097900100E780E01A17B501001305452DBE
:1052100059B017B501001305A52D97900100E7803F
:1052200020311305C01297D0FF1FE7808011014580
:1052300097E0FFFFE78000E30D4597100000E7804F
:10524000009F294597D0FF1FE780A00F97D0FF1F31
:10525000E78000008DBA99476303F40297B5010017
:105260009385C53F17B50100130545C2979001000E
:10527000E780201417B501001305452829B817F752
:10528000FF1F034737E797F7FF1F83C7A7E62207EC
:105290005D8F9166BA96C2061166C1821306F6EF5B
:1052A0008D476365D60297E7FF1F9387270D9C4BB9
:1052B00017F6FF1F0346F6E39386C7002DC203D6F9
:1052C000070069CA8907E39CD7FE89471307A0F83E
:1052D000114697F5FF1F9385A5E14A8597F6FF1FB5
:1052E0002388E6E017F7FF1FA305F7E097F0FFFF1D
:1052F000E780C0BA2A84E308058C97B5010093853E
:10530000E53517B50100130565B897900100E780F2
:10531000400AA28517B501001305851FE5B203D623
:105320000700630EE60A8907E39BF6FE8D4779BF07
:1053300091476304F40297B501009385253217B5B0
:1053400001001305A5B497900100E780800617B50A
:1053500001001305651D6FF00FF4B7E70400FC4F63
:105360009305000817E5FF1F0345C54B8297C9B891
:1053700097B501009385852E17B50100130505B17A
:1053800097900100E780E00217B501001305451B67
:105390006FF06FF02390E70017E5FF1F130505FE80
:1053A00097200100E780602D97B501009385052BBC
:1053B00017B50100130585AD97900100E78060FFE8
:1053C00017B501001305C51897900100E78060FE2E
:1053D000294597900100E780A0028147C5BD239031
:1053E000070017E5FF1F130565F997200100E78007
:1053F000C02897B501009385652617B501001305F0
:10540000E5A897900100E780C0FA17B501001305E1
:10541000A5155DBF411122C406C6834705002A8435
:105420009DC797B501009385251F17B5010013058A
:10543000E5A597900100E780C0F74C4017B5010043
:105440001305054A97900100E780A0F6E1A05841B6
:10545000B707CF009387777D631DF70697B50100E7
:105460009385851B17B50100130545A29790010090
:10547000E78020F41C448356E4008355C40003C62F
:10548000070017B501001305254797900100E78035
:1054900040F2294597900100E78080F60357E40029
:1054A0009707002083D7A7246309F7008355C4001A
:1054B000084497E0FFFFE78080CF0356E400835560
:1054C000C40008442244B240410117F3FFFF6700C3
:1054D0002355B707CC009387777D6315F70497B5FD
:1054E00001009385651317B501001305259A979060
:1054F0000100E78000EC1C448356E4008355C4009F
:1055000003C6070017B501001305053F979001007A
:10551000E78020EA2244B240294541011793010067
:10552000670003EEB707CE009387777D6304F70229
:1055300097B501009385450E17B501001305059534
:1055400097900100E780E0E64C4017B50100130595
:10555000E52FCDBDB240224441018280B7E704006F
:10556000FC4741112E8606C622C426C24AC02E849C
:105570002A89AA8517F5FF1F130585B7829797B566
:1055800001009385650F17B50100130525909790CD
:105590000100E78000E297F5FF1F83C565B517B5E9
:1055A0000100130565B597900100E78080E029456B
:1055B00097900100E780C0E497F4FF1F938444B301
:1055C00083C7040041479387070693F7F70F636A81
:1055D000F75C17B701001307E79E8A07BA979C4349
:1055E000BA9782879D476307F40297B501009385B8
:1055F000A50817B501001305658997900100E7809C
:1056000040DB17B501001305A5AF97900100E780B7
:1056100040DAADAC97F7FF1F83C797ADDDCB17F727
:10562000FF1F034717AD97F7FF1F83C787AC2207FC
:105630005D8F97F7FF1F83C7E7ABC2075D8F97F7B3
:10564000FF1F83C737ABE207D98F17F7FF1F232F41
:10565000F7A683C7640097B501009385E50117B5E8
:1056600001001305A58217F7FF1F2300F7A69790E7
:105670000100E78000D497F7FF1F938727A58C438D
:1056800017F6FF1F034666A417B50100130505A909
:1056900097900100E780E0D1294597900100E780CD
:1056A00020D697F7FF1FA38507A42244B240924457
:1056B0000249930700F817F7FF1F230BF7A29D4538
:1056C00017F5FF1F1305C5A241011743000067002E
:1056D000C3CD97500000E780407E97F7FF1F238AD5
:1056E000A7A09357850017F7FF1FA304F7A09357B0
:1056F00005012A8417F7FF1F230EF79E9357850194
:10570000014517F7FF1FA307F79E97500000E7809A
:10571000807B97F7FF1F2380A79E97B50100938595
:10572000A5F517A501001305657697900100E780A0
:1057300040C817F6FF1F0346069CA28517B5010057
:105740001305459FB1B7CD476303F40297B5010038
:10575000938585F217A50100130545739790010005
:10576000E78020C517B501001305459E79BD37E4D4
:1057700004007C44414697F5FF1F9385759717F504
:10578000FF1F1305E594829717F5FF1F1305459436
:1057900097100000E78080C497100000E78000ACFD
:1057A00097F7FF1F83C7E79517F7FF1F0347579525
:1057B000A20703238405D98F17F7FF1F2316F7903D
:1057C0001306000A89452244B2409244024917E573
:1057D000FF1F03452505410102838D476303F40242
:1057E00097B50100938545E917A501001305056AE2
:1057F00097900100E780E0BB17B501001305C5A431
:1058000029B517F4FF1F0344C48E97F7FF1F83C702
:10581000378E97B50100938525E6220417A5010070
:105820001305C5665D8C97900100E78080B8A2855E
:1058300017B501001305059397900100E78060B745
:10584000294597900100E780A0BB0D4697F5FF1F03
:105850009385058A228597E0FFFFE7802064AA846C
:1058600021C197B50100938525E117A50100130516
:10587000E56197900100E780C0B3A68517B50100E8
:105880001305858F97900100E780A0B22244B240B3
:10589000924402492945410117930100670043B62C
:1058A00097E7FF1F2398877AB7E70400116603A3E1
:1058B0008705130606E8914539B78D476303F4025F
:1058C00097B50100938545DB17A501001305055C1D
:1058D00097900100E780E0AD17B50100130585A59D
:1058E0002DB317F4FF1F0344C48097F7FF1F83C72E
:1058F000378097B50100938525D8220417A50100AC
:105900001305C5585D8C97900100E78080AAA28599
:1059100017B501001305858797900100E78060A9FE
:10592000294597900100E780A0AD0D4697E5FF1F40
:105930009385057C228597E0FFFFE7802056AA84A7
:105940001DC197B50100938525D317A50100130547
:10595000E55397900100E780C0A5A68517B5010023
:105960001305058405B797E7FF1F2397876CB7E7F3
:105970000400116603A38705130606E893050002D9
:1059800099B5894763E3870297B501009385C5CE32
:1059900017A501001305854F97900100E78060A1CE
:1059A00017B501001305C59B8DB197E4FF1F83C494
:1059B000447497E7FF1F83C7B77397B501009385BA
:1059C000A5CBA20417A501001305454CDD8C9790CB
:1059D0000100E780009EA68517A501001305C57D7F
:1059E00097900100E780E09C294597900100E780AF
:1059F00020A1228697E5FF1F9385856F268597E076
:105A0000FFFFE780A0492A84630E051A97B50100BD
:105A1000938585C617A5010013054547979001009A
:105A2000E7802099A28517A501001305257A99BD65
:105A3000854763F98718834519002244B240924490
:105A40000249B335B00097E7FF1F238FB76017A552
:105A500001001305E5784101179301006700639584
:105A6000A2852244B24092444A850249410117036B
:105A700000006700032299476303F40297B5010011
:105A8000938585BF17A50100130545409790010038
:105A9000E780209217B50100130545A6BDB617E4AF
:105AA000FF1F0344046597E7FF1F83C7776497B51B
:105AB0000100938565BC220417A501001305053D6F
:105AC0005D8C97900100E780C08EA28517A501002C
:105AD0001305857297900100E780A08D2945979066
:105AE0000100E780E091194697E5FF1F9385456027
:105AF000228597E0FFFFE780603AAA841DC197B531
:105B00000100938565B717A5010013052538979007
:105B10000100E780008AA68517A501001305C56E60
:105B200095B397E7FF1F239D875AB7E704001166D7
:105B300003A38705130606E89305000869B18547A6
:105B400097B50100938545B317A5010013050534EA
:105B5000630BF40097900100E780A08517A5010072
:105B60001305C56B5DB497900100E780808417A58D
:105B700001001305256C97900100E780808329457B
:105B800097900100E780C0872244B24092440249C6
:105B900097E7FF1F239A0752410117530000670040
:105BA000432297B50100938525AD17A50100130584
:105BB000E52D97800100E780C07F17B50100130530
:105BC0002598A1B4B2402244924402494101828006
:105BD000411106C622C497E0FFFFE780202C93778F
:105BE000F50FA1C32A8497B50100938565AA17A56F
:105BF00001001305A52997800100E780807B93753C
:105C0000F40F17B50100130565C797800100E78001
:105C1000407A2244B24029454101178301006700C0
:105C2000237EB240224441018280411122C4914628
:105C30002A8417E6FF1F1306E6599D652D4506C603
:105C400097D0FF1FE78080B6B7F7070003C70701AB
:105C5000A5476313F70001A09306001001469D6558
:105C6000254597D0FF1FE78060B497E7FF1F238388
:105C700087562244B240914617E6FF1F1306865509
:105C80009D652945410117D3FF1F670023B251715C
:105C9000CAD137E904008327C904A2D52E8686D746
:105CA000A6D32E84AA8517E5FF1F130565448297A6
:105CB00097E7FF1F83C7C7431307700A6387E7107F
:105CC000636CF7001307600A6384E704BE502E5428
:105CD0009E540E596D6182801307800A6388E7160F
:105CE0001307900AE394E7FE8D476309F41C97B508
:105CF00001009385E5CB17A50100130525199780B1
:105D00000100E780006B17B501001305A5C725A0AA
:105D10008D47630CF40297B50100938565C917A5FB
:105D200001001305A51697800100E780806817B56C
:105D30000100130565BE97800100E7808067294553
:105D400097800100E780C06B51B7854717B5010008
:105D5000130545BE17E7FF1F2308F73097800100A2
:105D6000E780007DB7750200B76602000146054571
:105D700097D0FF1FE78080A3930760F817E7FF1F06
:105D80002308F73697E7FF1FA385073693070026FA
:105D900017E7FF1F2320F736E5779387072117E7DB
:105DA000FF1F231BF734B14597E7FF1F23870734F5
:105DB00097E7FF1FA383A73417E5FF1F130545339C
:105DC00097300000E780605E11B7914763E3870278
:105DD00097B501009385C5BD17A501001305050BF7
:105DE00097800100E780E05C17B50100130585B6D8
:105DF00099B797E4FF1F83C4E42F97E7FF1F83C77A
:105E0000572FA204DD8C8327C9046D14228697E5E1
:105E1000FF1F9385352E280082978E049316040168
:105E2000B7750200C1823000A695094597D0FF1FC3
:105E3000E780C097930770F817E7FF1F230AF72A38
:105E4000994597E7FF1FA387A72ABDB7914763E34B
:105E5000870297B501009385A5B517A50100130525
:105E6000E50297800100E780C05417B501001305D3
:105E7000E5AFD1B597E4FF1F83C4C42797E7FF1FA1
:105E800083C73727A204DD8C8327C9046D142286BB
:105E900097E5FF1F93851526280082978E04931699
:105EA0000401B7750200C1823000A6950D4597D058
:105EB000FF1FE780A08F930780F8BDBF17B50100D3
:105EC000130585AD97800100E78080661305C01239
:105ED00097C0FF1FE780E046014597D0FFFFE780AE
:105EE00060180D4597000000E78060D4294597C0F1
:105EF000FF1FE780004597C0FF1FE7806035F9B3BB
:105F000041114AC097F6FF1F83D6667E328917D6A5
:105F1000FF1F0356C64822C426C206C62A84AE8482
:105F200097000000E780C05F35C12DC0994763FF2F
:105F300097048347140003470400A207D98F1397DF
:105F40008700A183D98FC2073167C1831307C75563
:105F5000639EE70297D7FF1F83D76744A301F4002E
:105F6000A1832302F40097F7FF1F83D7477891C7D7
:105F7000A302F400A1832303F400A68517B5010052
:105F8000130505A797800100E780A04297F7FF1F40
:105F900083C78765B9CF97D5FF1F83D5454017B510
:105FA00001001305A5A697800100E78080402686A2
:105FB000A28517D5FF1F0355853E97000000E78097
:105FC00060C16301090497E7FF1F83C7A7219DCB29
:105FD00095C897E7FF1F83C727098DE722852244CD
:105FE000B2400249A6859244410117330000670080
:105FF000C33B17B50100130565A297800100E78038
:106000002053C1B7B24022449244024941018280E8
:10601000834755008345450017B501001305059CCE
:10602000A207DD8D178301006700A33817B50100B3
:106030001305C599178301006700834F8D4763FBE4
:10604000B70A011126CA06CE22CC0344350097E4D4
:10605000FF1F83C4341997B501009385E59CB337BE
:10606000800017E7FF1FA30FF71609C497B50100BB
:106070009385459C17B501001305459C9780010049
:10608000E780203397E7FF1F83C7D7156386970004
:1060900097000000E780802697E7FF1F83C79714CB
:1060A0008DC785472306F100B7E7040083A747178C
:1060B0007000854513055030829717B50100130510
:1060C000E59897800100E780A0469967938757EE8F
:1060D0002316F100680085479145A3078100230737
:1060E000F10097300000E780402CF2406244D24437
:1060F000056182808280894763F7B708011122CC4D
:1061000006CE26CA8344250085472A84639DF4046D
:10611000914763F5B70403454500834734002205E2
:106120005D8D97D7FF1F239CA72697000000E7806F
:1061300000489967938767EE2314F1008347340082
:1061400023059100A305F1008347440095452800ED
:106150002306F10097300000E7802025F2406244DA
:10616000D24405618280FDF89967938767EE231416
:10617000F10097D7FF1F83D78722A305F1002305DE
:106180000100A183E1B782800111996722CCD51764
:1061900017F4FF1F130444452314F1008347040040
:1061A00026CA97F4FF1F938484542305F10083D7F4
:1061B000040028009545A305F100A18306CE23061F
:1061C000F10097300000E780401E03D604008345AD
:1061D000040017B501001305E58897800100E780EA
:1061E000401DF2406244D244056182809D6779710E
:1061F000D9172316F10097F7FF1F83C7E73E06D68E
:106200002307F100A9C3B7E70400FC47414697E51F
:10621000FF1F9385E5EB1305F10082976800CD45DC
:1062200097300000E780601897F5FF1F83C5C53BD6
:1062300017B501001305058697800100E7806017F8
:10624000B25045618280B7E70400BC4741468145B2
:106250001305F1008297D9B7B76702045D71938780
:1062600057AA3EC08567938707E02312F10097F78E
:10627000FF1F9387673783C70700A2C4A3030100EA
:106280002303F10097F7FF1F9387674683D7070023
:1062900037E4040086C62314F10097D7FF1F9387C5
:1062A000071083D70700414668002315F1007C449E
:1062B00097E5FF1F9385C5E18297F1450A85970011
:1062C0000000E780E021231EA1007C448A8508109D
:1062D000794682973C441305E1030946814582973C
:1062E000101093050002014597D0FFFFE780003EA4
:1062F000B640264461618280B7C7A55A01119387D1
:10630000C7333EC497E7FF1F83C7D7ED3EC6B7F735
:10631000070003C7070106CE22CCA5476313F70089
:1063200001A01164930504F0930600100146254571
:1063300097C0FF1FE78080473000930504F0A14617
:10634000294597C0FF1FE780604697E5FF1F83C57B
:1063500075E917B501001305A58497800100E78052
:106360004005F24062440561828001119165A146B9
:106370003000938505F02D4506CE97C0FF1FE780BE
:10638000E0422247B7C7A55A9387C7336314F70281
:10639000B24517A501001305E573B335B00097E7C3
:1063A000FF1FA381B7E497800100E7808000F240DF
:1063B00005618280814517A501001305E57397E704
:1063C000FF1FA38107E297800100E78080FE97000E
:1063D0000000E780A0F2E1BFB7C7A55A79719387A3
:1063E000F7353EC6B7E70400FC47AA8506D622D497
:1063F000414608088297B7F7070003C70701A5477A
:106400006313F70001A01164930504E893060010DC
:106410000146254597C0FF1FE7804039700093056E
:1064200004E8D146294597C0FF1FE780203817A50B
:1064300001001305A57A97800100E780600FB25034
:1064400022544561828079719165D14670009385AF
:1064500005E82D4506D697C0FF1FE7802035324757
:10646000B7C7A55A9387F73517A501001305C5705F
:106470006310F702B7E70400FC4717E5FF1F130599
:1064800025C541460C08829717A501001305C56C68
:1064900097800100E780C009B25045618280B7F75C
:1064A000070003C70701A5476313F70001A0916523
:1064B0004111930600100146938505E8254506C65F
:1064C00097C0FF1FE780802EB24017A5010013057B
:1064D000A55E41011783010067008305C1676976E6
:1064E0008146FD1705061397060141836364B700D3
:1064F0003E8582803307D50003470700B98F2147C7
:1065000013F81700858363050800B18FC207C183A4
:106510007D171377F70F6DF78506F1B741C5A547CE
:10652000054763F2B7088347150003470500316844
:10653000A207D98F13978700A183D98FC207C18380
:106540001308C855054763900707411106C622C4C2
:1065500026C203442500914763F087049307540043
:1065600063ECF502A301C50021822302C500930458
:10657000340091C6A302D500A1822303D5002A844A
:10658000A68597000000E780A0F526942300A400CC
:106590002181A300A4000147B240224492443A85DD
:1065A0004101828005473A858280B7C7A55A01110B
:1065B0009387E7343EC42AC6B7F7070003C707012D
:1065C00006CE22CC26CAA5476313F70001A091642A
:1065D0002A84938504EE930600100146254597C052
:1065E000FF1FE780A01C3000A146938504EE2945DB
:1065F00097C0FF1FE780801BA28517A50100130528
:10660000255C97800100E780C0DA97000000E780F2
:10661000E0C4F2406244D244056182800111916578
:10662000A1463000938505EE2D4506CE97C0FF1F8D
:10663000E780C0172247B7C7A55A9387E734631886
:10664000F702B24517A501001305054D97D7FF1FA7
:106650002397B7D4C205C18197800100E78060D538
:1066600097000000E78080BFF24005618280D1473B
:10667000D14517A501001305254C17D7FF1F23107F
:10668000F7D297800100E780C0D217D5FF1F0355CE
:1066900005D197000000E78080F1F9B7011126CA03
:1066A00006CE22CC93F71500AE848DCBAD6737179D
:1066B00000409387A7AA1CC3B7E70400BC4F13068A
:1066C0000019854517D5FF1F034545CD829713C592
:1066D0001400F2406244D2440561828093F72500A1
:1066E0006386071897A50100938545532D464800FA
:1066F00097800100E78080C097F5FF1F83C505FFE5
:10670000854793C4240063E5B7049DC9854517F503
:10671000FF1F1305A5ED97200000E78060AA97E70B
:10672000FF1F83C727AC89CF97F5FF1F83C505FCE3
:1067300017F5FF1F130585EB97300000E780E0C6D3
:106740001395040197F7FF1F238207FA418151B780
:1067500017F4FF1F034484E997F7FF1F83C717E966
:1067600022045D8CAD67C2059387B755C181630D67
:10677000F40C63E18704A9679387A755630FF40CB2
:1067800017F5FF1F130585E697200000E78040A35B
:1067900097E7FF1F83C707A5D1CF97F5FF1F83C5D5
:1067A000E5F417F5FF1F130565E497300000E78057
:1067B000C0BF49A0B1679387C7556302F404B567AA
:1067C0009387D755E31EF4FA17F5FF1F130505E26B
:1067D00097300000E78060BD97F5FF1F83C505F186
:1067E000894763F9B704F915C205C18117F5FF1F81
:1067F0001305E5DF97200000E780809C25A805466B
:1068000017F5FF1F130585DE97F0FFFFE780806F08
:1068100097F7FF1F83C747DD91EF4800978001007E
:10682000E780C0D993150501C181480097D0FFFFCB
:10683000E780E097A28517A501001305253C978006
:106840000100E78000B7EDBD17F5FF1F130505DA5E
:1068500097F0FFFFE780007CF1BF17F5FF1F1305DE
:10686000E5D897F0FFFFE780A07CE9B793F74500F4
:106870000145E38007E617A50100130565399780F8
:106880000100E780E0CA97300000E78000C113C52F
:10689000440081B5411122C437E404005C5C06C6A3
:1068A000354697A501009385A5E717B501001305A7
:1068B000A5A1829711E917A501001305E536978078
:1068C0000100E780E0C601A08327041C82972A8488
:1068D000054597B00000E780207A97600100E780C7
:1068E00040FF97600100E78040D497B00000E78048
:1068F000A08B2285B2402244410182801567B717E0
:1069000000401307575598C3D8439D66558FD8C389
:10691000D843FD76758FD8C3D8431367F70FD8C314
:1069200035671307C7CC98C382804111054506C659
:1069300022C426C297C0FFFFE780A05C1305800435
:1069400097B0FF1FE780A076757585457D1597C0C8
:10695000FFFFE78040467D7585451305F53697C0F6
:10696000FFFFE780A04F371400408327840A8D453E
:106970001305002093E707202324F40A97C0FFFFA4
:10698000E7806043B7E4040097D0FFFFE780A0886A
:10699000C85897800100E780A0B917B5010013051A
:1069A000A59297800100E780A0B88327840C8545D5
:1069B000414593E707082324F40C97C0FFFFE780C5
:1069C000E0498D451305000897C0FFFFE7800049A7
:1069D00097C0FFFFE780E075014597C0FFFFE780A4
:1069E000C07885450545894717F7FF1F2302F7D073
:1069F00097C0FFFFE780007937070004B7E700E0A2
:106A000023A0E71097D0FFFFE780A00A97D0FFFFF1
:106A1000E780601E97000000E78000E89700000014
:106A2000E780E09497000000E78080BF97E0FFFFD9
:106A3000E78040FA97000000E780601097000000B0
:106A4000E780600B83A7040817050000130545C500
:106A5000829797D7FF1F2383A794BC4C130600642B
:106A60008545829797000000E78080E997C0FF1F67
:106A7000E780009801458280B7F7070003C7070148
:106A8000A547AE866316F7009397450191C301A011
:106A9000AA850146254517C3FF1F670023D1411171
:106AA000B2862E86AA852D4506C697C0FF1FE780B1
:106AB000E0CFB2400145410182809307000463E8C2
:106AC000C7021D71A2CC2A84080886CE32C69780E0
:106AD0000100E780A082B2461008A285294597C030
:106AE000FF1FE780A0CCF6406644256182803955BF
:106AF000828041110D658D4506C697C0FFFFE78076
:106B0000802BB71700408D6623A6D70A17F5FF1F05
:106B1000130545BE1387C70A9387870A1CC15CC546
:106B2000856689675CC958C114C518C9B7E70400F0
:106B3000B24003A3871E4101028397F7FF1F83C75B
:106B4000E7BC99EF411106C697100000E78060612D
:106B5000B240854717F7FF1F230AF7BA4101828029
:106B6000828011C589C517C3FFFF67004364828017
:106B7000411126C2AE848D4522C406C62A8497C020
:106B8000FFFFE780A02DB717004099C803A5C70CE9
:106B9000418D23A6A70CB240224492444101828039
:106BA00003A5870C418D23A4A70CF5B783470500E7
:106BB00003471500A207D98FC2076177C187130762
:106BC0002720639AE7008345250037050400170353
:106BD0000000670023FA828017F6FF1F130646B3F2
:106BE0008147B2861303F00FA9483308F600034823
:106BF000080013F7F70F6307A80C63066800850702
:106C0000E39517FF2947B387E6002380A70097F78E
:106C1000FF1F9387A7B05DA8411113D765001347E5
:106C2000170006C693F63500058B954791CA0546B1
:106C300099476387C60009469D476383C600A147FD
:106C400013F645003336C00093F68503050685C26A
:106C5000A145638BB604E145638AB60493058002BF
:106C60006388B604930580036393B600914697F555
:106C7000FF1F238AF5D097F5FF1F2385C5D097F511
:106C8000FF1FA381D5D0BE8517A5010013054503BD
:106C900097700100E780E071B240854717F7FF1F4A
:106CA000A303F7CE410182808546D1B78946C1B79B
:106CB0008D4675BF17A50100130505031773010065
:106CC0006700236F17F7FF1F130747A5BA972380A5
:106CD000B700E147E302F5F493077002E30CF5FC1B
:106CE00082802A8723800500814717F5FF1F13053F
:106CF00025A21308F00F2946B306F50083C6060047
:106D00006396E60297F6FF1F938646A1B69783C760
:106D1000070005452380F5009947636EF7029D47FC
:106D200063FDE700E147630DF7008280638506019C
:106D30008507E393C7FC0145C5B723800500828022
:106D4000B737004003C7370083C7050093F7070430
:106D5000D98F2380F5008280797126D24AD097F4AA
:106D6000FF1F83C424D417F9FF1F1309E9D206D6E5
:106D700022D44ECE52CC56CA5AC8B307990083C704
:106D8000070093F7F70FA5C79387140093F7F70F42
:106D90000D476361F70C17F7FF1F2305F7D097F72F
:106DA000FF1F9387E7CFA69783C70700130710023B
:106DB00093F7F703638FE7286363F70A054463805B
:106DC0008720E389076E09476389E71413070002E8
:106DD000E38EE758B7E700E03707400023A0E71845
:106DE00001000100CA942380040023A0E710B787A4
:106DF000004003C76700058BE30F077897F6FF1F76
:106E000083C666CA0547E39AE67629472381E702E7
:106E100009472383E7022385E70297F7FF1FA3852E
:106E200007B697F7FF1FA38007C8B7870040A38165
:106E3000070017F7FF1FA30B07B405472383E700DD
:106E4000B250225492540259F249624AD24A424BF9
:106E50004561828097F7FF1F238607C489B7130710
:106E600030026386E70A63E6E71413074002638A89
:106E7000E70813070003E39FE7F497F7FF1F9387E3
:106E8000E7C1A69703C70700A1471377F70FE31AD7
:106E9000F71C17FAFF1F130A2A8983476A0097F61F
:106EA000FF1F2389F6AC97F7FF1F83C7578891C749
:106EB000FD5797F6FF1F238FF6AA97F5FF1F83C58F
:106EC000B58697F7FF1FA387B7AA97F7FF1F83C75A
:106ED000A78593F907089306000493F707066393C1
:106EE000D7529307A009638DF51A63EAB716930783
:106EF000F005638AF54E930750096388F52E014427
:106F000079ABFD5717F7FF1F2305F7A6E1B5FD572E
:106F100017F7FF1F230EF7A475BD17A50100130572
:106F200025EE97700100E780A06097F7FF1F938719
:106F3000E7B6A69703C40700814917FAFF1F130A93
:106F40002A971374F40F97AA0100938AEAEB63C798
:106F50008904294597700100E780804A854717F723
:106F6000FF1FA305F79417F7FF1F2302879417F756
:106F7000FF1F230BF7A037E700E0B70640002320F0
:106F8000D71801000100378600408347A60293F717
:106F9000370F2305F6022320D7102DBDB3073A0182
:106FA00083C507005685850997700100E78060401A
:106FB00079BF854717F7FF1F230AF78E21BD17A555
:106FC00001001305E5E397700100E780605697F72D
:106FD000FF1F9387A7ACA69703C40700814917FA40
:106FE000FF1F130AAA801374F40F97AA0100938A53
:106FF000AAE163C58904294597700100E7804040F4
:10700000854717E7FF1FA301F77E17E7FF1F230E32
:10701000877C17F7FF1F2309F79637E700E0B706CD
:1070200040002320D7180100010037860040834725
:10703000660293F7370F2303F602B1BFB3073A0195
:1070400083C507005685850997700100E780603683
:107050004DB7854717E7FF1F2308F778A5BB9307B0
:10706000400A638DF5349307200B6388F536930748
:10707000100AE396F5E883072A00014463D107422A
:1070800097E7FF1F83C7776A93F63700638E061A68
:107090000546638EC62209466399C61A1D4775A226
:1070A00017E5FF1F03456568C94717EAFF1F034A35
:1070B000DA6797E5FF1F83C5656717E4FF1F034481
:1070C000F4666319F510CD476316FA10930770083C
:1070D000639CF5021307300FB7170E006308E40036
:1070E0001307900DB7B704006314E40817F7FF1FE8
:1070F0002328F788BE8517A50100130565D1977071
:107100000100E780002BE5BB93078008639DF50035
:1071100033048040B77746001374F40F938787CD0C
:10712000B3D78702E1B793079008639AF500330459
:10713000804091671374F40F9387C766D5B79307A0
:10714000A008639BF50033048040B7173D0013741B
:10715000F40F93870790E9B79307B008639AF50097
:107160003304804091671374F40F938797D04DBF19
:1071700093F5F5078D47639BF50033048040B7977F
:107180005B001374F40F938707D859BF8947639B3B
:10719000F50033048040B7770B001374F40F938726
:1071A000071BBDBF8547639AF50033048040DD6748
:1071B0001374F40F938767E3A5B789E9330480401C
:1071C0008D671374F40F938777DC99BFF16793870A
:1071D000072029BF97000000E78040A0A2855285C4
:1071E00097000000E780809F19BB9305610017E5B9
:1071F000FF1F0345855317E4FF1F034414539700F3
:107200000000E78040AE93057100228597000000E2
:10721000E78060AD3C0017F7FF1F232DF7868347FB
:1072200061002304F10083477100A304F100894742
:1072300017E7FF1F2300F7748357810017E7FF1F2D
:107240002314F74E0944A1AC154793F64700B33613
:10725000D00093F78703850685C32146638BC70655
:107260006146638AC706130680026388C706130651
:1072700080036393C700914717E6FF1F2304D6706E
:1072800097E6FF1FA380F67097E7FF1F238DE76E39
:1072900017E7FF1F034787499376070497E7FF1F08
:1072A00083C7D7488DEE1377770C93067008630C6D
:1072B000D7021377F7078D46631ED70AB307F0404E
:1072C000B7955B0093F7F70F938505D881A8194709
:1072D000ADBF854755B7894745B78D4771BF930601
:1072E00070086311D7021307300FB7150E006389BA
:1072F000E7021307900DB7B504006383E702130795
:10730000700845BF9306800C6311D702B307F040A5
:10731000B775460093F7F70F938585CDB3D5F50282
:1073200097E7FF1F23AEB764F9B39306900C631A77
:10733000D700B307F040916593F7F70F9385C566C3
:10734000F1BF9306A00C631BD700B307F040B7153D
:107350003D0093F7F70F93850590C9B79306B00CDE
:10736000E319D7F4B307F040916593F7F70F9385CE
:1073700095D06DB78946631BD700B307F040B7754A
:107380000B0093F7F70F9385051B49BF8546631ADA
:10739000D700B307F040DD6593F7F70F938565E3FA
:1073A000B5BF09EBB307F0408D6593F7F70F9385F1
:1073B00075DCADB7F165938505209DB783472A003D
:1073C000C18B99C7854717E7FF1F2308F75A05BEEA
:1073D00097E7FF1F2383075A1DB6854717E7FF1F4F
:1073E000A303F75A29BE3C0017E7FF1F2324F76ABF
:1073F0000947930700032314F10097E6FF1F238B2F
:10740000E6562DBD639A0758A94763ECB74417A702
:107410000100130727888A05BA959C41BA9782878D
:1074200017E4FF1F03447430094A630C440F636C74
:107430008A0885476309F40A9307F00F17E7FF1FCF
:107440000347475363F6E70017E7FF1F2304F7528C
:1074500017EAFF1F034A0A52930700041374FA0F36
:1074600063F447011304000497E7FF1F93878762C3
:1074700083AA0700228617E5FF1F1305E52AD68594
:10748000330A8A40A29A97700100E78020E797E7C5
:10749000FF1F2381474F97E7FF1F23AD575F97E7F4
:1074A000FF1F83C7374D1547639AE762B7E700E0D0
:1074B0003707400023A0E71801000100B78600400D
:1074C000238086028DA58D47630CF40A9947E31546
:1074D000F4F697A701009387678217E7FF1F232B16
:1074E000F75AA947A1BF17E7FF1F0347C75B97E7F5
:1074F000FF1F9387274A494697A501009385058971
:107500006306870097A50100938545843E859770A3
:107510000100E780A0DE17E7FF1F232DA756C9470C
:1075200031BF97E6FF1F83C60658054797E7FF1F41
:10753000938747466394E6023E851306700297A53B
:1075400001009385258297700100E78020DB17E713
:10755000FF1F2321A75493077002CDB53E85130664
:107560003004979501009385257A97700100E78094
:10757000E0D817E7FF1F232FA750930730047DBDE6
:1075800097E5FF1F83C5651A17A5010013058589B7
:1075900097700100E780E0E1854A17EBFF1F034B7E
:1075A0008B5097E5FF1F83C5451817A501001305EC
:1075B000658763185B0B97700100E78080DF97E7B2
:1075C000FF1F83C78716B5CBE368F4E617A4010055
:1075D00013040480638C6701179401001304C47FB3
:1075E0006386470117A401001304848022859770E5
:1075F0000100E780A0FC1375F50F930715008607BF
:1076000017E7FF1F2308F7388D4717E7FF1FA3036E
:10761000F73897E7FF1F9387E7370147BE86137652
:10762000F70F89076365A60297E7FF1F23A4D746D4
:1076300097E7FF1F83C7073611B597970100938718
:10764000277217E7FF1F2327F7449147C5BB33066F
:10765000E40003460600A380070005072380C70057
:107660007DBF97700100E780C0D497E7FF1F83C7F5
:10767000C70BE1D7E362F4DC1794010013044472F2
:10768000638C570117940100130404726386470149
:10769000179401001304C472228597700100E780DB
:1076A000E0F11375F50F93071500860717E7FF1F25
:1076B0002302F72E8D4717E7FF1FA30DF72C97E73F
:1076C000FF1F9387272D0147BE861376F70F890783
:1076D000E37CA6F43306E40003460600A38007001B
:1076E00005072380C700D5B797E5FF1F83C5E503CE
:1076F000179501001305C57397700100E78060CBF3
:1077000097E7FF1F83C7D72893E7470017E7FF1FB7
:10771000A300F72883472A0017E7FF1FA308F726CF
:107720006FF0EFFD179501001305C571977001000B
:10773000E78000E097E7FF1F9387472583C707008F
:1077400017E7FF1F2302F7FE17E4FF1F03448422FD
:1077500033348000A9B3179501001305E56F9770C6
:107760000100E780E0DC97E7FF1F83C7772293E7FC
:10777000070117E7FF1FA30DF72083472A0017E72C
:10778000FF1F2305F7206FF08FF7179501001305F2
:10779000E56D97700100E780A0D903470A007D8B53
:1077A00051EFB787004003C767021377C70B136712
:1077B00027002383E70203C7A7021377C70B1367CA
:1077C00027002385E70203C7E7021377C70B136778
:1077D00027002387E70203C727031377C70B136725
:1077E00027002389E702854717E7FF1F230EF7FECF
:1077F00017E7FF1F230CF70A17E7FF1F230AF716E7
:1078000017E7FF1F2307F71697E7FF1FA38E07FC55
:1078100097E7FF1FA38C070897E7FF1FA38A0714AA
:1078200097E7FF1FA387071497E7FF1FA38E07148F
:1078300097E7FF1FA38907266FF06FEC8947631254
:10784000F70297E7FF1F83C767EE9146638CD7085F
:1078500063E0F604638EE70C6369F70A054763800B
:10786000E70EFD5717E7FF1FA306F7103707400085
:10787000B7E700E023A0E71801000100B786004049
:107880001306F0FC2381C60223A0E7106FF08FD40B
:10789000130720086382E7086362F70213071008E2
:1078A000E391E7FC378700408347670293F7C70BF4
:1078B00093E727002303F7026FF06FE41307300804
:1078C0006389E70213074008E39DE7F83787004024
:1078D0008347270393F7C70B93E727002309F70292
:1078E0006FF0EFE1378700408347270393F73707AF
:1078F000F5B7378700408347E70293F7C70B93E755
:1079000027002307F7026FF08FDF37870040834798
:10791000E70293F73707F5B7378700408347A70299
:1079200093F7C70B93E727002305F7026FF02FDDCE
:10793000378700408347A70293F73707F5B73787A4
:1079400000408347670293F73707ADB717950100EB
:107950001305C55297700100E78080BD97E7FF1FB0
:10796000238407DCD5B317950100130525529770C2
:107970000100E780E0BB97E7FF1F239707DA97E74F
:10798000FF1F938727FF03C40700894763F387001E
:1079900009441374F40F21B613070002E393E7ECD4
:1079A0006399090A638FF500930720026381F50844
:1079B000179501001305055197700100E780609F3E
:1079C0004DB5179501001305254D97700100E7800F
:1079D00020B60144179B0100130B4B4DA14AB3077E
:1079E0008A0083C507005A85050497700100E78067
:1079F000409CE31654FF179501001305E5AF9770FF
:107A00000100E780E0B217E4FF1F034424D211E431
:107A100097E7FF1F238D07CE59B48947E313F4E49A
:107A2000854717E7FF1F2304F7CE6FF04FCD17E60A
:107A3000FF1F034696CF97E5FF1F83C505CF179518
:107A400001001305254797700100E78080966FF0CD
:107A50000FCB638FF50493071002E39BF5F497E5D2
:107A6000FF1F83C5A5CC179501001305A546977088
:107A70000100E780009497E7FF1F23AD470197E7D8
:107A8000FF1F9387E7EF944383D7470017E7FF1F54
:107A9000034767EF17E6FF1F2328D6C81D4497E664
:107AA000FF1F2395F6C897E7FF1F2382E7C8C5BAD3
:107AB00097E5FF1F83C585C717950100130505438B
:107AC00097700100E780E08E97E7FF1F238107C4CE
:107AD00097E7FF1F239A07C46FF0CFF62547E38788
:107AE000E79C19476391E702B7860040238086022E
:107AF000B7E700E03707400023A0E71801000100C6
:107B0000130600FC41B31307100A6391E702B7861E
:107B1000004023808602B7E700E03707400023A03B
:107B2000E71801000100130680FCA9BB1307A00998
:107B3000E38FE7FC1307400AE38BE7FC13072002FF
:107B4000E386E7960547E383E796B7E700E0370764
:107B5000400023A0E718E391099601000100B786D1
:107B6000004023808602130620FC29BB17E7FF1F75
:107B7000034757E06308F71E63E7E7029547630E84
:107B8000F70E99476308F704B78600402380060282
:107B9000B7E700E03707400023A0E7180100010025
:107BA0001306A0FCC5B19307F005630AF70093071D
:107BB00050096306F70093071002E317F7FCB7E7D5
:107BC00000E03707400023A0E71801000100B78656
:107BD000004051BF97E9FF1F83C9C9D9930700042B
:107BE000CE8A63F43701930A000497E7FF1F938757
:107BF00067EA03AA070013F4FA0F2286D28517E575
:107C0000FF1F130565B297600100E780206FB387FF
:107C10008940529417E7FF1F230EF7D497E7FF1F01
:107C200023AA87E6638E0902B787004023805703A3
:107C3000B7E600E03706400023A0C61801000100A7
:107C400003C72702134707042381E70203C727025C
:107C50001377C70F2381E70223A0C6106FF08F9719
:107C6000B786004023800602B7E700E037074000F0
:107C700023A0E71801000100FDB5378700408347C6
:107C8000370097E6FF1F83C676D093F70708D58F96
:107C9000A301F700B7064000B7E700E023A0D7181C
:107CA000010001001306A0FC2301C70223A0D71086
:107CB0006FF04F9297E7FF1F938747DEA69783C722
:107CC000070093F7F70FD9CF97E7FF1F83C7A7DD0B
:107CD000D1EB17E7FF1F0347F7C9930700026313B0
:107CE000F70897E7FF1F938727A403AB070097EADE
:107CF000FF1F83CAAAA317EAFF1F034A3AA397E903
:107D0000FF1F83C9C9A2D2875687CE865A8697E5B8
:107D1000FF1F83C5C59F179501001305A51E97601A
:107D20000100E780006997E7FF1F23AB67C597E76E
:107D3000FF1F238957C597E7FF1FA38547C597E70F
:107D4000FF1F238237C597E7FF1FA381879CB7E7F3
:107D500000E03707400023A0E71801000100B786C4
:107D60000040D1B3B7E700E03707400023A0E71891
:107D700001000100B786004025B529472381E702AD
:107D800009472383E7022385E7022387E702238944
:107D9000E7026FF08F8803C76700118B6302078AC1
:107DA00083C75700918BB5CF17E7FF1F0347A7CFB6
:107DB00085476313F70697E7FF1FA386E7BC97E79E
:107DC000FF1F238307A297E7FF1F238107AE97E7D3
:107DD000FF1F238F07B897E7FF1F238C07B897E78C
:107DE000FF1FA38307A097E7FF1FA38107AC97E7B7
:107DF000FF1FA38F07B697E7FF1FA38C07B697E770
:107E0000FF1FA38307B897E7FF1FA38E07C8B78795
:107E1000004011476FF08F8217E7FF1FA308F78E0E
:107E200079BF854717E7FF1F2300F79C17E7FF1F60
:107E3000230EF7A617E7FF1F230CF7B217E7FF1F64
:107E40002309F7B269BF854717E7FF1F230EF7988D
:107E500017E7FF1F230CF7A417E7FF1F230AF7B04C
:107E600017E7FF1F2307F7B017E7FF1FA30E0796BB
:107E700017E7FF1FA30C07A217E7FF1FA30A07AE10
:107E800097E7FF1FA38707AE8280411106C69700C0
:107E90000000E78080FBB7870040238007001307BE
:107EA00040FC2386E7001307C004A386E70017E71A
:107EB000FF1F130767872398E70017E7FF1F1307C4
:107EC000A78A239AE70017E7FF1F13072796239C2B
:107ED000E70017E7FF1F1307A7A1239EE700294725
:107EE0002381E70209472383E7022385E7022387EB
:107EF000E7022389E702A3810700930600F8A38025
:107F0000D700930690022380D700FD562383D70025
:107F10002381E700B706400037E700E02320D710B1
:107F200003C7170013671700A380E700B24097E765
:107F3000FF1F239D07A441018280411106C69700BF
:107F40000000E78080F0B787004023800700130718
:107F500000FC2386E7003147A386E70017D7FF1F01
:107F60001307877C2398E70017D7FF1F1307C77FE6
:107F7000239AE70017E7FF1F1307478B239CE700AF
:107F800029472381E70209472383E7022385E70284
:107F9000A3810700930600F8A380D7009306900200
:107FA0002380D700FD562383D7002381E700B7063F
:107FB000400037E700E02320D71003C717001367FE
:107FC0001700A380E700B24097E7FF1F2390079CAC
:107FD00041018280F1679387072017E7FF1F232164
:107FE000F79A854717E7FF1F231EF798A14717E762
:107FF000FF1F230AF79897E7FF1FA386079897E7C5
:10800000FF1F2383079897D7FF1F2382077097D7F7
:10801000FF1FA38D076E814717D5FF1F1305456FFF
:10802000FD5517D6FF1F1306666F2947B306F500E7
:108030002380B600B306F600238006008507E39789
:10804000E7FE97E7FF1F238907A497E7FF1FA38594
:1080500007A497E7FF1F238207A497E7FF1FA38CBE
:10806000079097E7FF1FA38A079097E7FF1F2385D5
:10807000079097E7FF1F2380079097E7FF1F238F45
:10808000078E97E7FF1FA389078E97E7FF1F2386B9
:10809000078E97E7FF1FA38207A0828017E7FF1FC5
:1080A000034767A085476316F700170300006700C2
:1080B00003E917030000670083DD411122C406C6EF
:1080C00017E7FF1F0347279E85472E8613F4F50FFA
:1080D000AA856317F70417D5FF1F13052579976045
:1080E0000100E780A02197D7FF1F2381077CB78776
:1080F000004023848702B7E600E03706400023A053
:10810000C6180100010003C7A7021377C70F238514
:10811000E702B240224423A0C610014541018280FB
:1081200017D5FF1F1305456897600100E780001D04
:1081300097D7FF1F238A076AB787004023828702E9
:10814000B7E600E03706400023A0C6180100010092
:1081500003C767021377C70F2383E7025DBF41118F
:1081600006C697000000E78020E7B24041011703F0
:1081700000006700E3F2411106C697F0FFFFE780B9
:10818000E0BD97D7FF1F83C7376695C797D5FF1FF9
:1081900083C5A56589C917D5FF1F1305256597F008
:1081A000FFFFE780409C97D7FF1FA38F076297D7F9
:1081B000FF1F238B077CB2404101828041C9D9C592
:1081C00097D7FF1F83C7877CD1C3011122CC4AC830
:1081D0004EC656C25AC006CE26CA52C42E89AA8995
:1081E0000144930A0004371B030063772403B30799
:1081F0008940C207C183BE8463F4FA00930400047B
:10820000C204C180130A1BD497D7FF1F83C7C75D61
:108210009DE37D1A631C0A00F2406244D244424945
:10822000B249224A924A024B0561828097F0FFFFD1
:10823000E780C0B2D1BF338589002694A685420469
:1082400097000000E780A0E7418045B7828097E76C
:10825000FF1F9387E78818429C4383D64500034558
:10826000070083C5C700035646006396A50083D563
:10827000E700638DD502011106CE2386A700239760
:10828000D700B705CF00DC4B9385757D05077D16BC
:108290002EC2230001003AC42316C1002317D100C7
:1082A00099C30A858297F240056182808280DC4D05
:1082B000DC4B81CFB7E70400904503A387059145C8
:1082C00017E5FF1F03450582028382806D713C081C
:1082D0003EC6B707E500232291103EC8AA843C0899
:1082E0003285232611103ECA232481102320211118
:1082F0002E8997300000E78020562A849795010048
:108300009385C5C317850100130545B89760010023
:10831000E780200AA285179501001305A5D2976072
:108320000100E7800009294597600100E780400DC2
:10833000B705CB009385757D680097100000E78036
:10834000405FA285680097300000E7804043014706
:1083500081467000CA85268597200000E780C0828C
:1083600005CD2A8497950100938545BD17850100A9
:108370001305C5B197600100E780A003A28517959A
:1083800001001305E5CC97600100E78080022945D4
:1083900097600100E780C0068320C110032481108C
:1083A00083244110032901105161828097D7FF1F58
:1083B0009387077318429C43797122D406D60348E9
:1083C000070083C807012A8483D645000355460069
:1083D0006396080183D82701638DD802238807019B
:1083E00005072399D7003708CC00DC4B1308787DAC
:1083F0003ACC1307F5FF42CA23080100231EE1000F
:10840000231FD10099C7080832C62EC4829732466E
:10841000A245228597000000E78080EBB2502254ED
:10842000456182806D713C083EC0B707E5003EC2E1
:108430003C083EC4232611102324811023229110CE
:10844000231701002318010023190100231A01003A
:10845000231B010097B7FF1F83D7C7F699E3C167B6
:10846000FD172316F10097B7FF1F83D7C7F591EBD0
:1084700097D7FF1F9387C7669C439C43DC4783D7EE
:10848000070017B4FF1F1304E4F3584C2317F1003F
:1084900083574400484B2318F10031E197950100C0
:1084A0009385C5B0178501001305459E97600100AF
:1084B000E78020F017950100130585B09760010053
:1084C000E78020EF294597600100E78060F3832073
:1084D000C11003248110832441105161828097B719
:1084E000FF1F83C797EE89EBB7E70400BC5782975D
:1084F0005C4C23AA0700E1BFFD1797B6FF1FA386B8
:10850000F6EC03560701834704014C470A85230B09
:10851000F10097300000E780A02397D7FF1F9387D3
:10852000275C9C430147814688430A866C0097106C
:108530000000E7806065AA8429C1979501009385B2
:10854000E5A6178501001305659497600100E78093
:1085500040E6A68517950100130545A79760010021
:10856000E78020E5294597600100E78060E9584CE5
:10857000B7E70400BC57484B9DBF97B7FF1F83C7A1
:10858000D7E4F5D7B7E70400BC4F1044854517D5AD
:10859000FF1F0345255582971DBF5C4EDC4BB9CFAD
:1085A000B1CD411122C4178501001305258E2E84FB
:1085B000979501009385C59D06C697600100E780E9
:1085C00040DFA28517950100130505A39760010000
:1085D000E78020DE294597600100E78060E2B7E789
:1085E00004002244B24003A3870517D5FF1F0345AB
:1085F000654F130640069145410102838280411177
:1086000022C417B4FF1F1304A4D91C4C06C689C783
:10861000DC4399C34C488297584CB7E70400BC57D9
:10862000484B82975C4CB240224423AA0700410188
:10863000828017B7FF1F1307A7D883470700930649
:10864000F00B850793F7F70F63E9F60097B6FF1F66
:108650002388F6D6034507008280930700F8FDB70C
:10866000835745006386071001114AC817B9FF1FD9
:10867000130949D552C4032AC90106CE22CC0327C7
:108680004A0126CA4EC656C2F15735E31307D00D2C
:10869000FD57636EC704B7E9040083A709072A845E
:1086A0001305860042054181B284AE8A8297232A4F
:1086B000AA000325C9015C49A9E7979501009385A4
:1086C000258B177501001305657C97600100E78015
:1086D00040CE179501001305659A97600100E78069
:1086E00040CD294597600100E78080D1DD57F240F9
:1086F0006244D2444249B249224A924A3E850561C7
:10870000828093874400B705CF002319F500938535
:10871000757D310597100000E780A0210325C90170
:1087200083456400310597300000E780400503254C
:10873000C9012686D685310597300000E7804001C3
:108740007146A2854A8597600100E78020BB5044AE
:1087500019CA83A78905854517D5FF1F03458538A5
:108760008297814769B797000000E780E0CBD5BFCB
:10877000FD573E858280411126C297B4FF1F938426
:1087800064C4D84C22C437E404003C54484B06C6A9
:108790008297DC4C0323C4052244B240924423AAAE
:1087A000070017D5FF1F0345E533854541010283C7
:1087B000411126C297D4FF1F938484329C4006C681
:1087C00022C44AC0D5C3DC43C5C35CC12300B50085
:1087D0002A84978501009385E574177501001305B8
:1087E000E56A97600100E780C0BC294597600100F9
:1087F000E78000C19C4023A4070023A2070097B78D
:10880000FF1F9387E7B9DC4FDC4B91C729559700D1
:108810000000E78000DF97B7FF1F9387A7BADC4F00
:10882000DC4B89C797000000E78020F537E904009A
:108830008327C905894517D5FF1F0345A52A8297B8
:108840008327C905914517D5FF1F0345A5298297A1
:108850009C4003A347016309030022852244B240E0
:108860009244024941010283B240224492440249A7
:10887000410182800111328506CE22CC26CA2E8487
:1088800097300000E78040FDAA849785010093851A
:10889000A56C177501001305655F97600100E780FF
:1088A00040B1030784000356640083554400A68644
:1088B000178501001305457697600100E78060AFDA
:1088C000294597600100E780A0B397B7FF1F83C7D2
:1088D00087AD639D9700014597000000E78060D257
:1088E00081450A8597000000E780C0ECF2406244B1
:1088F000D244056182806D712324811023261110DA
:108900002322911093F745002E84638707143C08B7
:108910003EC0B707E5003EC23C083EC42317010035
:108920002318010023190100231A0100231B010051
:1089300097B7FF1F83D7C7A699E3C167FD17231613
:10894000F10097B7FF1F83D7C7A591EB97D7FF1FFC
:10895000938707199C439C43DC4783D7070017B7CD
:10896000FF1F1307E7A32317F100544F8357470056
:108970002318F100DC4AA1E7978501009385056281
:10898000177501001305855097600100E78060A20C
:10899000178501001305C56297600100E78060A19B
:1089A000294597600100E780A0A513454400832076
:1089B000C11003248110832441105161828097B734
:1089C000FF1F83C7579E2555D9C3FD1717B6FF1F35
:1089D000A30BF69C03D6060183470701CC460A8504
:1089E000230BF10097300000E78080D697D7FF1F58
:1089F0009387070F9C4317B7FF1F1307679A978644
:108A000001009386E65E88430A866C00971000009A
:108A1000E7808017AA8451D997850100938505586E
:108A2000177501001305854697600100E78060987F
:108A3000A685178501001305655997600100E78039
:108A40004097294597600100E780809B2685970025
:108A50000000E78000BB91BF93F725009DC7B7E7F3
:108A60000400BC4741468145280882972555970058
:108A70000000E78000B928089305F00F9700000078
:108A8000E78040D3134524001DB793F71500014537
:108A900099DF97000000E78020991345140001BF7B
:108AA0005C4D411106C688C317D7FF1F232AF70262
:108AB000B7E7040083A70708170500001305E5E3DF
:108AC0008297B24097D7FF1F238EA700014541012F
:108AD000828001113335A000A307A100B7E704008D
:108AE00083A7471706CE1306F100854513055030BE
:108AF0008297F240056182808280411122C406C6BD
:108B000097D7FF1F83C787FF014489EF97B7FF1FE0
:108B100083C7576D054499E717D4FF1F0344C4ACBE
:108B200013441400228597000000E780C0FA1785DF
:108B300001001305656009E4178501001305C56090
:108B40002244B240410117630100670083867971B6
:108B500022D4A30F010037E404008327841726D210
:108B60004AD006D6AA842E89130550309305F10108
:108B700032C6829732468347F10193150601C181BF
:108B800085CB01452EC697000000E780C0F48327FF
:108B90004417B2454A86268582970545970000000E
:108BA000E78060F3B25022549254025945618280AA
:108BB000832744174A8626858297EDB741119397FC
:108BC000050122C406C626C2C1872E8463D40702CB
:108BD000B7E40400FC5417B5FF1F0345A581829735
:108BE00019C1BC5482972165218DB2402244924420
:108BF0004101828093F715008DC7B7E7040083A772
:108C0000471A17A6FF1F1306E67D97D5FF1F93850A
:108C100025EE17A5FF1F0345E57D82971345140038
:108C2000E9B793F7250099CFB7E70400BC4F1306C7
:108C30000064894517A5FF1F0345C57B829713452F
:108C4000240065B793F785009DC7B7E7040003A824
:108C5000871A1307401F97A7FF1F83C7A77981466D
:108C600013064006994517D5FF1F035565E902987D
:108C7000134584009DBF93F745000145BDD7B7E478
:108C8000040083A7041817D5FF1F035565E78297D3
:108C9000BC4C13060064914517A5FF1F034585755D
:108CA00082971345440091B797D7FF1F83D747E5B5
:108CB0006398A70217D7FF1F2315B7E417D7FF1F25
:108CC0002312C7E417D7FF1F231FD7E22E8617856D
:108CD00001001305A54CBE85175301006700636DA5
:108CE000178501001305054D1763010067004384D4
:108CF0000357450097D7FF1F83D787E0631AF70410
:108D0000C1674111F91722C417D7FF1F232AF7DEC5
:108D100037E4040097D7FF1F23A607DE97D7FF1F6E
:108D2000A38E07DC7C4C06C6894517A5FF1F0345AB
:108D3000656C82977C4C914517A5FF1F0345856B99
:108D400082972244B240410117030000670023DBF1
:108D50001785010013050546175301006700437D81
:108D60007D15954763E2A71C178701001307873A13
:108D70000A053A951C41011122CC06CEBA972E84E1
:108D80008287178501001305654397500100E7802E
:108D9000207AA1A203C7250099476311F7022E8507
:108DA00097000000E78000F5834564001785010007
:108DB0001305C54197500100E780A05F97B7FF1FDB
:108DC0002382074217850100130505427DBF03C7B3
:108DD000250095476319F702C16717D7FF1F03578F
:108DE00027D2F91703D5A5006309F702B7E70400F6
:108DF00083A7C7178297178501001305E53F975092
:108E00000100E780E072854717B7FF1F230CF73C8E
:108E1000178501001305C5408DBF97D7FF1F23910C
:108E2000A7CE83D7E50097D6FF1F239CF6CC83D728
:108E3000050197D6FF1F2397F6CC83D7250197D638
:108E4000FF1F2392F6CC97D7FF1FA38907CA631B86
:108E5000E502B7E70400BC4F096613060690A1457A
:108E600017A5FF1F0345055982970356E400835554
:108E7000A400178501001305653997500100E780AC
:108E8000405351B79307700F2316F100B7E7040062
:108E900083A7870D17A6FF1F0346C6556C00829750
:108EA0004DF9854717D7FF1FA30AF7C45DB717858C
:108EB00001001305A537D1BD83C5250091476392F5
:108EC000F502178501001305E53797500100E7808B
:108ED000206697000000E78080C2F240624405618E
:108EE000828099476392F502228597000000E7800F
:108EF00060E083456400178501001305252D975018
:108F00000100E780004BD1BF9547639AF500834786
:108F10001400E1F31785010013050535BDB517856C
:108F200001001305E534E1BF82806D7123248110B7
:108F30002326111023229110328401CD8947630A20
:108F4000F5028320C1100324811083244110516154
:108F500082801785010013056532AE8497500100A9
:108F6000E780005DA285268597C0FFFFE780405F10
:108F7000C9BFB7E70400FC472800829717850100A6
:108F80001305853097500100E780805A83478100A0
:108F900039C41307000B6380E7021387A705137713
:108FA000F70F8D4663EDE602A285280097D0FFFFFC
:108FB000E78020CE79B78547E3F587F883459100B0
:108FC000177501001305C521B335B00097B7FF1F12
:108FD000238CB70897500100E780A03D9DB7034759
:108FE0009100A207D98F35671307D7556385E70826
:108FF0006368F7022D671307B7556387E706316784
:109000001307C755638AE70429671307A7556394B5
:10901000E702A285280097D0FFFFE780600115B71F
:1090200039679306E765638DD70663E9F600130792
:10903000E7556380E706A28528003DB73D679306A4
:10904000F7556386D7061307F766E396E7FE97D0D2
:10905000FFFFE780E019F5B50146A285280097D00B
:10906000FFFFE78020EAF1BDA285280097D0FFFF2F
:10907000E78040FAF9B58947E3F587EC9305E4FF0B
:10908000C205C1811305A10097A0FFFFE780201250
:109090004DBDA285280097D0FFFFE78060FA55B547
:1090A000A285280097D0FFFFE780200559BD97D003
:1090B000FFFFE780A00D71B5411122C417A4FF1F67
:1090C00013048434AA861786010013062606228517
:1090D000C14506C697500100E780C04603574400CB
:1090E00097A7FF1F938747332393E7000357640035
:1090F0002394E700B240224441018280411106C618
:1091000097000000E78080FBB7E7040083A787147F
:1091100017A6FF1F1306462FD54501458297B2407B
:109120004D4697A5FF1F9385252F130570304101EC
:10913000170300006700E3A161712324811A37E45B
:109140000400832704082326111A2322911A2320BE
:10915000211B232E311917050000130565A68297E0
:1091600017A9FF1F13090929994785442300A9005E
:10917000231CF10097850100938545FF9307400666
:1091800017750100130585D0231CF10823089100F1
:1091900097C9FF1F9389A95597500100E780602167
:1091A00083D5090017850100130545FB9750010081
:1091B000E7802020294597500100E780602403D5EF
:1091C0000900856997000000E78040EF8327441776
:1091D000100885451305503082978327441717A63A
:1091E000FF1F13066623CD45130570308297832732
:1091F000441717A6FF1F13062620B5451305603038
:1092000082978327441730088945130510318297C8
:109210008327441730098945130520318297832716
:109220004415938509C80D45829783274415938576
:1092300009C811458297A3059100230691002308D0
:10924000910002CD230C010083278416300991453B
:10925000130570408297832784161306B100854555
:1092600013050040829783278416700085451305F7
:1092700010408297832784163008854513052040C7
:1092800082978327841610088545130550408297DE
:10929000832704157D558297832744137D55829734
:1092A0007D5597A0FFFFE780403B8327440C8297C2
:1092B00097A0FFFFE78080168327841417A6FF1F5F
:1092C00013068614D5450145829789471306700F0A
:1092D000814528092306F1009790FFFFE780E0DF32
:1092E0008D471306000881452808230CF108979044
:1092F000FFFFE78080DE9147230CF10097770100A4
:10930000938747AA984383C747003AC8230AF100C6
:1093100097D0FFFFE78080F470008545054597A052
:10932000FFFFE780A03A30099305700F094597A029
:10933000FFFFE780A0393008930500080D4597A08E
:10934000FFFFE780A03810089545114597A0FFFF63
:10935000E780C037C16717C7FF1F1307677AF91780
:109360001CC32322070017A5FF1F1305650897A03C
:10937000FFFFE78080348327C41D17C5FF1F130537
:10938000A57682973C48034509008545829783204E
:10939000C11A0324811A8324411A0329011A83293B
:1093A000C1195D618280C16717C8FF1F03584875E6
:1093B000F9176301F8083DCDB5CD011126CAB7E410
:1093C000040083A7841222CC2E862315B10006CE7A
:1093D0002A8401478146ED45428582972AC611EDD0
:1093E00017850100130585D997500100E7804014C7
:1093F000F2406244D24405618280FC440356A100DD
:10940000A28582972C0017C5FF1F0355656F97A093
:10941000FFFFE780403769DD17850100130545D759
:1094200097500100E780C01083A7C412ED452800C3
:1094300082977DBF8280411106C61DC9854717A747
:10944000FF1FA300F7FC354697A5FF1F9385C5FABC
:109450001305603097A7FF1F238607FA97F0FFFFD9
:10946000E780206FB240410117F3FFFF67002369D7
:1094700097A7FF1FA38707F8F9B7C16717C5FF1F95
:1094800003550568F9176307F500B7E7040003A360
:10949000C71702838280854717C7FF1F2300F7661F
:1094A000014517F3FFFF670003631793FFFFE70210
:1094B00023BE2A8408452E89B28919C900C197158F
:1094C00000009385A586610597300100E780800143
:1094D00081447D5A97100000E780E03963C7A404F7
:1094E000814497100000E780003A63C8A40497C73E
:1094F000FF1F938767619C43DC47B307F94091875F
:109500002302F400638309048327C900B307F440EE
:109510009587A302F4001C4C89C79C4799C32285F8
:1095200082971793FFFF6700E3B95C441397140019
:109530008504BA972390470171BF1C481397140004
:109540008504BA972390070069BF832789000547E0
:10955000B307F4409587A302F40083570400638E99
:10956000E7028DC309476384E7040D47E395E7FAF3
:1095700097870100938707241CCC97870100938766
:10958000672411A897870100938747EA1CCC978727
:1095900001009387A7EA5CC8BDBF97870100938746
:1095A000E7D51CCC97870100938747D6EDB79787FF
:1095B00001009387E7241CCC9787010093874725F8
:1095C000D9BF95E51793FFFFE70223AE0046184485
:1095D0008347940075839D8B6317F70097100000F5
:1095E000E78060B448C41793FFFF670043AE8280F2
:1095F0001793FFFFE702C3A913893500C16442092D
:109600004111AA890144F11413590901054A2EC6D2
:1096100097100000E7802026B2456348A40001456A
:1096200041011793FFFF6700E3A983A70900131700
:109630001400BA9783D707006388B7006394970034
:1096400063742A010504E1B70545D9BF1793FFFFED
:10965000E70223A3AA892E89328BB6843A8ABE8A6E
:1096600097A00000E78020FB71C9268597200000A5
:10967000E78020098D4763E7A7007D551793FFFF1B
:109680006700A3A383DB440097100000E780A024B9
:109690002A8497100000E780402593077400314426
:1096A0003305850263CDA70297100000E780A02252
:1096B00097100000E78020222A8497100000E7809E
:1096C000C0229307740031443305850263C3A704A5
:1096D00097100000E78020209307450029A89710E5
:1096E0000000E7808020330585021307F0179307F9
:1096F000C017E35FA7FA2D55E3C277F963040B02A5
:10970000D6865286A6854A8597200100E78020BA32
:10971000B5B797100000E780401D33058502930719
:10972000C5FFD1BF832749001385C90083D5270012
:1097300097000000E78000EC61F581B769553DBFF7
:1097400097C7FF1F2394A73C97C7FF1F9387C73B6B
:10975000904381470C463307F500420741836393EA
:10976000B70082805446139847008507C29623901D
:10977000E600D5B797C7FF1F938707399C4303C5FA
:109780008700828017C5FF1F0355453882801793D5
:10979000FFFFE7028391C1671387D7FF630BE502E1
:1097A000636AA700F1176300F50201451793FFFFF5
:1097B0006700E3911387E7FF6302E502FD171D8D44
:1097C00013351500E5B797500000E780C0267D15DA
:1097D000C5BF97500000E78040FBD5BF9750000001
:1097E000E78060F9EDB71793FFFFE702038C4111A3
:1097F000AA8401442EC697100000E780C008B24535
:109800006348A400014541011793FFFF6700238CC3
:109810009C48131514003E9583570500E385B7FE59
:109820000504C9BF03485500814693F7F60F63E569
:10983000070181473E858280584593975600BA9725
:1098400003D727006316B70003D70700E304C7FE5A
:109850008506E1BF8346450001479377F70F63E430
:10986000D700814711A81C45131657000507B2976A
:1098700003D60700E313B6FE3E8582801793FFFFF1
:10988000E702038193170501C18797CAFF1F938AD7
:10989000AA27635BF00883A70A00C0479C470357C9
:1098A0000400198D420541816368F5000144228559
:1098B0001793FFFF6700038112052A94CDBFDC4791
:1098C00013944900014A3E94834744006341FA02DD
:1098D000014A834754006349FA028509C20993D9B2
:1098E000090183A70A009847E3EBE9FCC1B71C44D0
:1098F00013195A00A6853E994A8597000000E78013
:10990000C0EE05E1050AC9B75C4413195A00A685E3
:109910003E994A8597000000E78020ED19E1050A8D
:109920004DBFE30C09FA61B7AA8481495DBF178373
:10993000FFFFE70283771C452A8481E79307C50070
:109940001CC51C44231204001CC09307F00F63EDD8
:10995000B70093F5F50F228597200000E78020E2FD
:109960001783FFFF6700A37693940501C167C18049
:1099700063F9F500A685228597200000E78040E581
:10998000C5B7C18193F5F50F228597200000E780C8
:1099900000DFA685228597200000E78040E0C9B758
:1099A00097C7FF1F93874716884382801C4599C736
:1099B00097C7FF1F23AAA714014582807D55828087
:1099C00097C7FF1F9387471498438347450048472D
:1099D00092073E9582801783FFFFE702036D617156
:1099E00000451C183EC6B70780013EC81C183ECA79
:1099F0008357440002CE02D002CC231EF1008347DD
:109A000084002A8902D22301F1023C083ED402D606
:109A100097000000E78000FB835705002316F10242
:109A200097500000E78060C42307A1025C40035503
:109A30006400F18313F717008347F1025205518147
:109A4000F99BD98FA307F10297100100E780807579
:109A500039CDAA840355050097A00000E78080BC9B
:109A600083D704002AD26800231CF10083D7240086
:109A7000231DF1001C4803D647008C4397200000AB
:109A8000E78000CD8347B400CA861786010013061D
:109A900066808117A305F4006C0048109720010030
:109AA000E780E0805D611783FFFF67004362215517
:109AB000D5BF1C45B1CF03C5A70089461357650024
:109AC000630BD7028D46630ED70285466300D7022B
:109AD000130740063305E50203C7B700418B15CBDA
:109AE00083C7B700BD8B3355F54082801375F503EE
:109AF0001307803EC5B709671375F5031307077190
:109B0000D1BF372709001375F5031307077CD9B7B1
:109B1000014582801783FFFFE702235903A98500CF
:109B2000630C09048347B900AE8493F7070E85C31D
:109B300003459900930520030D810505B305B50282
:109B40008844610597300100E780E0A935A02E85A3
:109B500097000000E78020F62A8419CD97000000C6
:109B6000E780605C8325C900B307B54063FA8700CE
:109B70002E94B305A440E9F51783FFFF6700235532
:109B800085457DBF1783FFFFE70223522A8403D553
:109B90000500011132C636C43AC22EC002CA02CC38
:109BA00002CE97A00000E780E0A782452ACA22855E
:109BB0002ECC97000000E780E0E003570500231E4D
:109BC000E10097500000E78040AAA2463246924743
:109BD000230FA10036874C08B286228501469700E4
:109BE0000000E780E0A605611783FFFF6700234EB2
:109BF0001783FFFFE702634B61711C183EC6B7076E
:109C000080013EC81C183ECA3C0800453ED4AA84C8
:109C100002CC02CE02D002D202D697000000E7802A
:109C200060DA8357050035592316F102975000007A
:109C3000E780A0A32307A10209C48357440081EB56
:109C400021594A855D611783FFFF6700434803552B
:109C500064005205518197100100E780A0542A89C1
:109C600065D18347B40093F7070E99C713058401A4
:109C700097300100E780609983574400231EF1006C
:109C8000834784002301F1025C4003550900D98316
:109C900013F7070883471102231CA10093F7F70766
:109CA000D98FA300F10283572900231DF1005C40E6
:109CB000F18313F717008347F102F99BD98FA307AC
:109CC000F10297A00000E780E0952AD235D98347BA
:109CD00094006800139757008347B400FD8BD98F19
:109CE000A305F4001C4803D647008C4397200000CE
:109CF000E78000A6A687177701001307A75974000D
:109D000005464C10268597000000E78060942A895C
:109D10000DD98347B400A685FD8BA305F4009700F9
:109D20000000E78060DF31BF1783FFFFE702E33702
:109D3000832485FE2A844111268597000000E78050
:109D400080D7834734FF93F7070E8DCB2AC626852D
:109D500097000000E78060C809CD834734FFB24513
:109D6000FD8BA309F4FE91C5228597300100E780A1
:109D7000808741011783FFFF670063357DD9832703
:109D8000C4FF2685829775F5834734FF93F7070E46
:109D900091C7228597300100E7802087032584FE44
:109DA00097000000E78000E5E9B71783FFFFE702AF
:109DB000C32C9C4141112A8903C7070089472E847F
:109DC000935667006380F6040D466388C6049307C4
:109DD000F0076304F7022E8597200000E780C0A7F4
:109DE000AA848149C16B130C490097C7FF1F938751
:109DF000A7D19C43984763E4E90441011783FFFF1F
:109E00006700632B03D745008547E3F8E7FE2E85FF
:109E100097200000E780A0A9E1B703D74500E3FE43
:109E2000E7FC2E8597200000E78000A3AA84228506
:109E300097200000E78060A4C204C98C5DB7DC47AE
:109E40000355A900139A49003E9A93170501C1874B
:109E5000635DF00083570A006397A70263E774030A
:109E60008327CA00034D5A002DA0A1672167A98F3F
:109E70001307F7EFE374F7FE6397090097000000FC
:109E8000E780209161FD85098DB783278A00034D06
:109E90004A00835DA90003576900216A138BC7003C
:109EA0003AC6814A33CA4D01631E5D0197C7FF1F41
:109EB000938707C69C43E1DBA2866286814526859F
:109EC0008297D1B7A1679387F7EF930C4BFF63F2AB
:109ED0004703B2455A8597F0FFFFE780A0710DC197
:109EE00003278B00104709CE10436382C402310759
:109EF000D5BFEE85668597000000E780008F71F979
:109F000093861A0093FAF60F130B0B0271BF835658
:109F100044005C43E3E9F6F622853AC69710000058
:109F2000E780807DA1679387D7042A8A035D440078
:109F3000324763E897008347D90093E707F8A30601
:109F4000F9001C4766852286E2858297C16708442E
:109F5000FD17337AFA00529508C02312A40125B7E1
:109F600097C7FF1F938747BA9843814715C3144784
:109F7000814763FFD500939745004C47BE9519C9AB
:109F800003C7550081476375E600DC451606B297A6
:109F90003E85828003C745008147E37BE6FE1606C7
:109FA0009C45F5B71783FFFFE702830EAA892E8A27
:109FB000814497CAFF1F938A2AB583A70A0098474E
:109FC00063E6E4001783FFFF6700C30FDC471394C9
:109FD000440001493E9413BB140083474400634B83
:109FE000F900014913BB140083475400634FF90083
:109FF0008504E1B70844931759005287DA86014671
:10A00000A2853E9582990509C9BF48449317590016
:10A010005287DA860546A2853E9582990509E9B7F9
:10A020001783FFFFE7026308814517F5FFFF13055C
:10A03000054897C7FF1F239B07AC97000000E780E8
:10A04000A0F61783FFFF6700830897C7FF1F93875A
:10A05000A7AB9C4395C31783FFFFE7020305814528
:10A0600017F5FFFF1305A54497000000E780C0F334
:10A070001783FFFF6700A30582801783FFFFE702B6
:10A08000230137E404008327841241112315E100E2
:10A09000AE893289368A3A8681460147ED45AA84DF
:10A0A00082972AC621C90356A100D2859740010094
:10A0B000E780C0248327C413CE852685829705892F
:10A0C00005C98327440D2314210101462C00268550
:10A0D00082972A8401C9B7E7040083A7C712ED4518
:10A0E00028008297228541011783FFFF670083FDC7
:10A0F0004944D5B76554FDB75C41FD175CC182800A
:10A100001783FFFFE70263FAB7E70400FC5F82975B
:10A1100095473305F50281450D811783FFFF6700E1
:10A1200003FB1783FFFFE70243F8B7E70400FC5F78
:10A13000829795473305F5020D811783FFFF67006E
:10A1400003F91783FFFFE70243F6B7E7040083A78D
:10A15000870B0355050082971783FFFF670023F7DE
:10A160001783FFFFE70263F4035505003287AE86CD
:10A170001796FF1F0356663097C5FF1F9385859975
:10A1800097000000E780A0EF1783FFFF670023F42C
:10A190001783FFFFE70263F1B7E7040083A7C71740
:10A1A00082971783FFFF670083F21783FFFFE702A1
:10A1B000C3EFB7E7040083A7871397C5FF1F9385F5
:10A1C0006595829701451783FFFF670043F017836A
:10A1D000FFFFE70283EDB7E7040083A7C71F8145B0
:10A1E0001795FF1F0355652582971783FFFF6700AB
:10A1F00003EE1783FFFFE70243EBB7E7040083A7F3
:10A20000871397C5FF1F9385E591829701451783B3
:10A21000FFFF6700C3EB1783FFFFE70203E9B7E720
:10A22000040083A7C71F81451795FF1F0355E52627
:10A2300082971783FFFF670083E91783FFFFE70219
:10A24000C3E62E8597800000E780E0AF978000008E
:10A25000E780E0EC1783FFFF670063E71783FFFFEA
:10A26000E702A3E497800000E780E0F61783FFFF92
:10A270006700E3E55C49E1175CC95CC583572501CC
:10A28000A1072319F50083570501A1072318F5003D
:10A290008280F1473305F50297C7FF1F9387878AAE
:10A2A0009C433E9582808D476315F60803D7460090
:10A2B000854763F0E7081783FFFFE70203DF368572
:10A2C00036842E8997100000E780005929C98357EA
:10A2D000440093140501C18063E39704228597101D
:10A2E0000000E7806057FD14231294009307A0023A
:10A2F0006300F5029307B0026307F502930790022B
:10A30000631FF500228597000100E780C08501A842
:10A310000146CA85228597A00000E78060B01783B8
:10A32000FFFF6700C3DA228597100000E780C003B3
:10A33000FDB7828097C6FF1F938606819C42014528
:10A3400099CF9843D44217B6FF1F232FE67E63961A
:10A35000D70097B6FF1F23ABE67E1385C7FE82802A
:10A360001783FFFFE70263D497000000E780A04B4C
:10A37000714433058502914597900000E78020E9FC
:10A3800011E565551783FFFF670063D497B7FF1F7B
:10A3900023A8A77A97000000E780E04833058502EC
:10A3A000914597900000E78080E661DD97B7FF1F39
:10A3B00023AAA77897000000E780E04697B7FF1F21
:10A3C000239AA77697000000E780E04597B7FF1F24
:10A3D0002393A77697770100938707F117B7FF1F9D
:10A3E000232EF77497070000938707E917B7FF1F1D
:10A3F0002324F774014579B71783FFFFE702E3CA07
:10A40000AA8517B5FF1F1305E57297100000E780B6
:10A41000C05B1783FFFF670083CB1783FFFFE70253
:10A42000C3C897000000E78060FD97100000E78038
:10A43000405B97B7FF1F938727719C4391CF13878A
:10A44000C7FE19CB83D5C7FF17B5FF1F130545708E
:10A4500097200100E78020191783FFFF670023C7BB
:10A460001783FFFFE70263C497000000E780C0EC9A
:10A4700009CD834785002A8493F7070499EB035598
:10A48000E50097000000E78080F91783FFFF670071
:10A4900003C48347C5009304450117B9FF1F13097F
:10A4A000A96A85E3832709005CC997B7FF1F23AD1D
:10A4B000976883274900F1FB97B7FF1F23A8976888
:10A4C000E9B7FD172306F500610597800000E780D6
:10A4D000C0D68307840063CB07048347840093E7D7
:10A4E00007F82304F400B7E704009C5F8297420555
:10A4F000A94741813375F5028347840093F707FC30
:10A50000C98F2304F4008347D4003E951C402318D0
:10A51000A40089CF984319CB8347C400504081459C
:10A5200085073305F502420541810297832709001B
:10A530005CC897B7FF1F23A997608327490089E765
:10A5400097B7FF1F23A497608347C4009DDF8355FF
:10A55000040117B5FF1F1305A55F97200100E780D1
:10A56000800825B71783FFFFE70223B497C7FF1FB3
:10A57000938747839C4701448583858B85E3AE841D
:10A58000B2853A8697100000E780804B2A8419C56F
:10A5900097100000E780C041829408CC2285178381
:10A5A000FFFF6700C3B21783FFFFE70263AE4111ED
:10A5B0002E8932C6AA8997000000E780C031324751
:10A5C00013060502CA86970500009385C5CC17B50A
:10A5D000FF1F1305255697000000E780E0F82A8446
:10A5E00025C99304C50097000000E780E0411946A3
:10A5F000AA85268597100000E78080158545268569
:10A6000097100000E780601117750100130585CBD6
:10A610004E9583450500268597100000E78020169B
:10A620005C4831468145A1075CC85CC4835724015E
:10A63000E1172319F40083570401E1172318F400EC
:10A640001C4C3E859780FFFFE78020A9A3042501CD
:10A65000228541011783FFFF6700C3A61783FFFF11
:10A66000E702A3A44111AA842EC632C497100000A9
:10A67000E7806036004DB2452246834784000CC017
:10A6800050C093F7F70393E707042304F40023185B
:10A690000400268597100000E780803183479400EE
:10A6A000A9462317A40013D7370005073307D7029D
:10A6B0009D8B85072306F400A306E40083C70401ED
:10A6C000D8488507230FF7FE17B7FF1F1307C747A3
:10A6D0005843232A04009307440129E317B7FF1FB7
:10A6E0002326F74617B7FF1F2320F74617B4FF1F8F
:10A6F00013040446228597200100E78000E11C44F2
:10A70000858B5D8D19E58145228597200100E780C5
:10A7100080ED41011783FFFF6700639B1CC317B7E0
:10A72000FF1F2325F742D9B71783FFFFE702E397FF
:10A7300097050000938565B7014597000000E78005
:10A7400000B001451783FFFF670063981783FFFF81
:10A75000E702A39597000000E78080B01783FFFF12
:10A760006700E3968347C500A5E31783FFFFE70271
:10A77000C3932A840355E50097000000E78000C8D2
:10A7800021C18347840093F7F7FB2304F4001C40A6
:10A7900091C7DC4381C74C40014582979700000078
:10A7A000E78080B917B5FF1F1305853A9720010090
:10A7B000E780A0E50355E40097000000E78020C68D
:10A7C0001783FFFF6700A39082801783FFFFE702D4
:10A7D000C38D97B7FF1F9387273797050000938591
:10A7E00065C817B5FF1F1305A53623A0070023A2D0
:10A7F000070097200100E780E0CE1783FFFF670086
:10A80000038D1C4D91CFDC4381CF1783FFFFE702FF
:10A81000C3898345070082971783FFFF6700238B57
:10A82000828097B7FF1F9387E7349C4303C50700D7
:10A83000828097B7FF1F9387E7339C4303C51700B8
:10A84000828097B7FF1F9387E7329C4303C5270099
:10A85000828097B7FF1F9387E7319C4303C547006A
:10A86000828097B7FF1F9387E7309C4303C537006B
:10A87000828097B7FF1F9387E72F9C4303C557003C
:10A88000828097B7FF1F9387E72E9C4303C567001D
:10A89000828097B7FF1F9387E72D9C4303C57700FE
:10A8A000828097B7FF1F9387E72C9C4303C58700DF
:10A8B000828097B7FF1F9387E72B9C4303C59700C0
:10A8C000828097B7FF1F9387E72A9C4303C5A700A1
:10A8D000828097B7FF1F9387E7299C4303C5B70082
:10A8E00011E11D45828097B7FF1F9387A7289C43DE
:10A8F00003C5C700828097B7FF1F9387A7279C4394
:10A9000003C5D700828097B7FF1F9387A7269C4374
:10A9100003C5E700828097B7FF1F9387A7259C4355
:10A9200003D50701828097B7FF1F9387A7249C4315
:10A9300003C52701828097B7FF1F9387A7239C43F6
:10A9400003D54701828097B7FF1F9387A7229C43B7
:10A9500003D56701828097B7FF1F9387A7219C4388
:10A9600003D58701828097B7FF1F9387A7209C4359
:10A9700003C5A701828097B7FF1F9387A71F9C433A
:10A9800003C5B701828097B7FF1F9387A71E9C431B
:10A9900003C5C701828097B7FF1F9387A71D9C43FC
:10A9A00003C5D701828097B7FF1F9387A71C9C43DD
:10A9B0008857828097B7FF1F9387C71B9C4303D597
:10A9C000C702828097B7FF1F9387C71A9C4303D59E
:10A9D000E70219E11305800C828097B7FF1F938768
:10A9E00067199C4303C50703828097B7FF1F9387AE
:10A9F00067189C43C85B828097B7FF1F9387071730
:10AA00008843828097B7FF1F938787168843828089
:10AA100019E17D558280F5DE984265DFFDD917B7D3
:10AA2000FF1F130727381847AA877155058B631D29
:10AA3000072403C507001547E37DA7FC03C73700BC
:10AA40001305F0057D171377F70FE364E5FC03C3E7
:10AA50005700E30003FC83C86700E38C08FA03C7D0
:10AA60007700494579171377F70FE364E5FA03C7D1
:10AA7000A70011481305F7FF1375F50FE36BA8F84E
:10AA800003CE97000D481305FEFF1375F50FE36223
:10AA9000A8F803C8B7006309080065181378F80F11
:10AAA0001305600DE36705F703C5C70079487915FD
:10AAB0001375F50FE36FA8F403C8D7000D457D1893
:10AAC0001378F80FE36705F503D80701930E4017D5
:10AAD0005118420813580801E3ED0EF303C8E700CC
:10AAE0007D181378F80FE36605F303C827017D1876
:10AAF0001378F80FE36F05F103C88700C54E75188A
:10AB00001378F80FE3E70EF103D86701856E938E93
:10AB1000BEE06D18420813580801E3EC0EEF03D8AD
:10AB200047016D18420813580801E3E40EEF03D8FB
:10AB300087017918420813580801E36C05ED03C832
:10AB4000A7017D181378F80FE36505ED03C5B7017C
:10AB50001D487D151375F50FE36DA8EA03C5D701F0
:10AB6000714879151375F50FE365A8EA03D5E70178
:10AB70001308E00F7D1542054181E36CA8E803C589
:10AB80000702494879151375F50FE364A8E8C8531F
:10AB900001C937C834005915130858BFE36BA8E63C
:10ABA00003A8870237C53400130555BF5918E3625F
:10ABB00005E717B5FF1F232DC5FA03C6050117B515
:10ABC000FF1F2329F5FA0545E375C5E403D82501E0
:10ABD000D04933760603E31E06E203C61501E30AF5
:10ABE00006E217B6FF1F2323B6F883C527000146E8
:10ABF0006387A50003C61700F1453306B60283C775
:10AC000007039305C00272971A071307C7051603B7
:10AC10001A9796084697B387B70241553E973297E1
:10AC2000420741836362E8061773FFFFE702E347C9
:10AC3000368597800000E780A06897000100E780D4
:10AC400020482A8497A00000E780805A2A9497F031
:10AC50000000E78060262A9497900000E780A0819A
:10AC60002A9497F0FFFFE780E06F2A949740000056
:10AC7000E78060932A9497700000E780A09C22955B
:10AC80001773FFFF6700A34482801773FFFFE7027B
:10AC9000C3414111A307A10097A00000E780A0C510
:10ACA0009305F100170500001305E5B597F0FFFFC8
:10ACB000E780802F014541011773FFFF67002341A3
:10ACC0001773FFFFE702E33B17B4FF1F1304840D64
:10ACD0000328840079599368180097B4FF1F23A7AD
:10ACE000140D1378180063100802BA84BE89368BDD
:10ACF000328A2E89AA8A97F0FFFFE780E0A77D15A8
:10AD0000269519E531594A851773FFFF6700E33A25
:10AD100097F0FFFFE78040A67D152695A167E353D6
:10AD2000F5FE97B7FF1F9387E73E98433E8C814B14
:10AD300001CB014597F00000E7802044933B1500CC
:10AD40004A85DA865686D28597900000E780C04D06
:10AD50002A8911CD1C44F99B17B7FF1F2328F7043C
:10AD600083270C00CDD3E3800BFA829769BF268539
:10AD700097B7FF1F23AA070297F0FFFFE780809C89
:10AD80004146CE8517B5FF1F1305450B97300100CF
:10AD9000E780C05697D00000E78040990325040B58
:10ADA00097D00000E780009D054597D00000E78020
:10ADB00000A4054597000000E78060EDA9B797B7AC
:10ADC000FF1F938727FE9C47858BEDC71773FFFFF7
:10ADD000E702A32D17B5FF1F1305850497B7FF1FC3
:10ADE00023A207FC97B7FF1F23A007FC97B7FF1FFD
:10ADF00023AE07FA97200100E780208197500000DA
:10AE0000E780E0F597100100E780A04C9710010063
:10AE1000E780A05297B7FF1F938747F79C4391C7DE
:10AE2000054597800000E780402097B7FF1F938774
:10AE3000A7DF9C4399C741657D1597700000E780A7
:10AE400040A297F00000E780E03D97D00000E78047
:10AE5000808F97B7FF1F9387E7099C4313971701CC
:10AE60006356070097F00000E78000AD97B7FF1F1B
:10AE700023A607FC97B7FF1F23A407FC97B7FF1F64
:10AE800023A207FC97B7FF1F23A007FC9700000031
:10AE9000E780008C97000000E780007297F0FFFFCA
:10AEA000E780401897F00000E78040D61773FFFF57
:10AEB0006700E321828097B7FF1F9387A7EE88433F
:10AEC00082801773FFFFE702431E97800000E78030
:10AED000607597800000E780C0771773FFFF6700F9
:10AEE000031F1773FFFFE702A31A2A8493041402B7
:10AEF00001112E85B289A685214636C63A8997303A
:10AF00000100E780403D0DE9B24638082686CE852F
:10AF10001305940497500000E780604121462C08F7
:10AF20004A8597300100E780003B13351500056125
:10AF30001773FFFF670003190145D5BF1773FFFFA4
:10AF4000E702A3169305450617B5FF1F1305C5C2F3
:10AF500097100100E78020691773FFFF6700231730
:10AF60001773FFFFE702631441112EC697F0FFFF2E
:10AF7000E780601BB24588C141011773FFFF67007E
:10AF800003151773FFFFE702A310AA842E8497808E
:10AF90000000E780006CAA898545228597000000A3
:10AFA000E780E07D83C7E4011389940899E313895E
:10AFB0000403CE85228597000000E780407C21466F
:10AFC00093051902228597000000E780607897B703
:10AFD000FF1F938727DD8C43228597100000E780B1
:10AFE000C082214693858402228597000000E78075
:10AFF00020761773FFFF6700E30C1773FFFFE7026C
:10B000004308397197F00000E780E0B493054006EB
:10B0100061E997800000E78000606302051497B73C
:10B02000FF1F83C727B713B7170097B6FF1F2383E8
:10B03000E6B6014499CFC16417B9FF1F130989D639
:10B040009309400EFD1497000000E780C08663421C
:10B05000A40A97F0FFFFE780000D4169B7290900B6
:10B06000096AFD7A2A8B81447D199389F97B130A39
:10B070000A71938A8AC797000000E780C08363D76C
:10B08000A4041304400EB387840217B7FF1F1307ED
:10B0900067D10324070B3E948357C4016382270BB7
:10B0A00018403307EB4063EAE90083474400850713
:10B0B000B3874703D6976365F7080146814509457D
:10B0C00097F0FFFFE780604EAA8B29E597400000CC
:10B0D000E780808385476317F50689659385057149
:10B0E00017B5FF1F130545A997100100E780A04F72
:10B0F00095A0B30734030327090BBA9703D7C701F9
:10B100006308970003C75700A38207002382E70064
:10B11000050415BF9305C500228597000000E78050
:10B1200080E65E852286976501009385E51A97F093
:10B13000FFFFE780E0525E8597100000E780608A9D
:10B14000850415BF97B7FF1F9387C7C59C478D839D
:10B15000858BC1F721611773FFFF670003F6014676
:10B160008545094502D002D202D402D697F0FFFFEE
:10B17000E780A043AA8479DD97F00000E780E09C97
:10B180001389C4002A8481454A8597000000E7801E
:10B19000005F0C4041464A8597000000E780405B15
:10B1A000832944006385090C4E8502D802DA02DC4B
:10B1B00002DE97300100E78060402ACE1410054679
:10B1C0002C0808184ECC97500000E780E00A137551
:10B1D000F50F51ED8355840093E525004A859700CE
:10B1E0000000E780E05E11460C104A8597000000E1
:10B1F000E78000560146976501009385650E268518
:10B2000097F0FFFFE780C045268597000000E780A4
:10B21000407D5C40A1D3014685450D4597F0FFFF79
:10B22000E780A038AA841DD548401389C400973010
:10B230000100E780A0382AC64A8597000000E78011
:10B24000404C3246636FC5004C404A859700000071
:10B25000E780005001468145268597F0FFFFE78093
:10B260002040268597000000E780A077E5B583554C
:10B270008400ADB71773FFFFE70223E397B7FF1F03
:10B28000938747B29C471DC193E7870017B5FF1FFF
:10B290001305858E17B7FF1F232AF7B097100100FB
:10B2A000E78040321773FFFF670063E2DD9B17B74B
:10B2B000FF1F232DF7AE97300000E780E0647DF19B
:10B2C00017B5FF1F1305458B97100100E780E0338A
:10B2D000D1BF1773FFFFE702C3DA4169AA892E8A3B
:10B2E000B28A368BBA8B814417BCFF1F130C8CAB10
:10B2F000930C400E7D1997F0FFFFE780C05B63C49D
:10B30000A40001443DA03384940383270C0B3E9496
:10B310008357C401638627055A87D6865286CE8511
:10B320001305040397000000E780E0BB01C92380F8
:10B330000B0022851773FFFF670023D88347F401B2
:10B3400085C35A87D6865286CE8513059408970002
:10B350000000E78040B909C585472380FB00D1BFC5
:10B36000850451BF835745006380071E1773FFFF95
:10B37000E70203D201112A8497000000E780C04D44
:10B3800009C985476309F50605611773FFFF670063
:10B3900063D397E00000E780007C7DF5835744008D
:10B3A0004947ED9BE392E7FEC145228597000000E7
:10B3B000E7804033AA84228597000000E780204F71
:10B3C0000357440002CE91472A89631AF700228569
:10B3D00097000000E780A0513C082ACC3ECE97E0C1
:10B3E0000000E78080765C55C5D374084A86A68540
:10B3F0000545829751BF03574400D147E3F6E7F86C
:10B40000032A0400C169014997BAFF1F938A8A99E8
:10B41000130B400EFD1997F0FFFFE780C049634F03
:10B42000A90E2285032A040097000000E780C0428D
:10B43000A1452A89228597000000E780A02AAA84D6
:10B44000228597000000E780804A14402A86AA8956
:10B4500078082685CA8597000000E780C0E7AA849F
:10B4600005D503C7F40189476315F7008347C10178
:10B4700081DF5546D2851385640097300100E7804F
:10B48000E0E7014597800000E780C01901C583D738
:10B49000C401A5E797B7FF1F9387C7909C479355B3
:10B4A0001900858913D73700058B01CF8983858BD8
:10B4B0006399B70001452EC697000000E780C0DB06
:10B4C000B2454E8597800000E780601F0346C101AA
:10B4D0002A8493751900268597900000E780E0394B
:10B4E00035C1268597800000E780E018268511C0C9
:10B4F000014597800000E780004C97300000E7800E
:10B50000A0408547E312F5E883C754001307F00F06
:10B51000E38CE7E68507A382F400BDB5B3046903B5
:10B5200083A70A0BBE9483D7C401638B37015546AA
:10B53000D2851385640097300100E780C0D955DDBE
:10B540000509D1BD5DD86DB782801773FFFFE70293
:10B5500023B497800000E780000C05C1C16401445A
:10B5600017B9FF1F130909849309400EFD1497F0C2
:10B57000FFFFE7804034634EA40017A5FF1F1305AB
:10B58000A55F97100100E780E0031773FFFF6700D6
:10B5900063B3330534038327090B3E958357C501F5
:10B5A000638897002312050097800000E780A00CB5
:10B5B000050475BF97A7FF1F9387C77E9C478D83A0
:10B5C000858B8DE31773FFFFE70223AE17A5FF1FDF
:10B5D0001305855A97100100E78020031773FFFFBA
:10B5E0006700E3AE82801773FFFFE70203AC9705A5
:10B5F00000009385C5A017A5FF1F1305E5579710F9
:10B600000100E78020EE1773FFFF670043AC17735C
:10B61000FFFFE70283A98841B7E70400BC5B05058B
:10B6200042054181829709C585472300F50005053C
:10B630001773FFFF6700A3A983C7F5FF2E85850752
:10B64000A38FF5FE828083C7F5FFFD1793F7F70FF1
:10B65000A38FF5FE99EF1773FFFFE70203A5B7E786
:10B660000400BC571385F5FF82971773FFFF67002F
:10B6700003A682801C41035745008D8FBA951CC1DB
:10B680002312B5003E85828093D78500A205144120
:10B69000DD8D835745001387E6FF18C18907231204
:10B6A000F50013D685004111238FB6FEA38FC6FE89
:10B6B0004101828018419307F7FF1CC18357450061
:10B6C00085072312F500A30FB7FE8280835745003C
:10B6D0008D8F2312F5001C41BE950CC12E858280F2
:10B6E000AA8703D7470008410D8FAA952392E70048
:10B6F0008CC38280184108453305A7408280835758
:10B700004500035765001D8F1C4108453385A74040
:10B710003305A74082801773FFFFE70203994111A9
:10B720002EC62A8497000000E780A0FDB24563730F
:10B73000B50001A0835744000840BE952312B40011
:10B740003E9541011773FFFF670063981773FFFF72
:10B75000E702A39541112E84B28532C697000000FE
:10B76000E780A0FB3246A28597300100E78000B950
:10B7700041011773FFFF670083951773FFFFE7020F
:10B78000C3922E84854597000000E78000F92300CE
:10B7900085001773FFFF670083931773FFFFE702AE
:10B7A000C39041112317B100894597000000E7803D
:10B7B000C0F68347E1002300F5008347F100A300B2
:10B7C000F50041011773FFFF670063901773FFFFD8
:10B7D000E702A38D93D78500A2054111DD8D2317C4
:10B7E000B100894597000000E78020F38347E1001E
:10B7F0002300F5008347F100A300F5004101177312
:10B80000FFFF6700C38C1773FFFFE702038A1397DC
:10B81000850193D78501C166938606F0D98F13D72A
:10B820008500758FD98FA2053707FF00F98D41116B
:10B83000DD8D2EC6914597000000E78000EE6C007C
:10B84000114697300100E78060AB41011773FFFF9D
:10B850006700E3871773FFFFE70223851C418545D7
:10B8600003C4070097000000E78080E62285177375
:10B87000FFFF6700C3851773FFFFE70203831C41C7
:10B880004111894503C7070083C717002307E1005B
:10B89000A307F10097000000E78080E30355E10073
:10B8A00041011773FFFF670083821763FFFFE70201
:10B8B000C37F1C414111894503C7070083C7170097
:10B8C0002307E100A307F10097000000E78040E0B4
:10B8D0008357E100410113D58700A2075D8D420522
:10B8E00041811763FFFF6700837E1763FFFFE70255
:10B8F000C37B0C4141112A84114668009730010036
:10B90000E780C09F9145228597000000E78040DCDA
:10B91000B247C166938606F01397870113D5870156
:10B92000598D13D78700758F598DA2073707FF00F0
:10B93000F98F5D8D41011763FFFF670043791C4557
:10B94000BE950CC18280AE87944391E6584101EFC9
:10B950000CC15CC1828003C7570013671700A38224
:10B96000E700B687D5B70CC3EDB7AA87084119CD54
:10B970001841D44398C36313D500D8C32A8703461C
:10B9800057009376160081E62320070082809443B7
:10B9900081CA8C4203A847008CC363930601CCC3C1
:10B9A000799A14C3A302C7003687D1BF1C45DC4770
:10B9B0001D8DB777DBB6938777DB09853305F502F5
:10B9C000420541818280F147B385F50248452E95B5
:10B9D00082808347450085072302F5008280176334
:10B9E000FFFFE702836C2A8409E41763FFFF670007
:10B9F000036E83474400F5DBFD1793F7F70F23022F
:10BA0000F400E5F71C4403D7270005072391E7005E
:10BA1000DC4399C3228582974C4889CD83475400E3
:10BA2000898B99E71C4422859C479C439C478297BD
:10BA3000232A04000040232004007DB71763FFFF82
:10BA4000E702A3668357250041112EC681EB01440E
:10BA5000228541011763FFFF6700636703570500F5
:10BA60008147F146E305F7FEB385D70240458507D8
:10BA70002E948345440008C4F5F5B247AA8481E7B3
:10BA8000232A040009A81C456C0022859C439C4382
:10BA9000829748C84DDD85472312F400B247232022
:10BAA0000400231804002319F4005C485CC483D705
:10BAB0002400FD172391F40061BF1763FFFFE70225
:10BAC000C35E97A7FF1F9387270D88432326050092
:10BAD00023240500410597100100E78000B3176398
:10BAE000FFFF6700C35E1763FFFFE702035C17A455
:10BAF000FF1F1304640A1C40411199CF9C47230087
:10BB0000B5002AC65CC197000000E78040FB1C40DE
:10BB1000DC4399C33245829741011763FFFF6700F9
:10BB2000035B0347450029E3584DAA877D551DCF88
:10BB30001763FFFFE70263571CC3DC4797A6FF1F8D
:10BB400023ACE604F156130507012390D7009705AF
:10BB500000009385050297100100E780A098014539
:10BB60001763FFFF6700A3567D55828082801763AD
:10BB7000FFFFE7028353011161468145280097606A
:10BB8000FFFFE780805597A7FF1F9387E7009C433F
:10BB900028009305F00FDC473EC697000000E780C1
:10BBA000C0F405611763FFFF6700635297A7FF1F8B
:10BBB000938787FE9C43D847A1679387C702631E7C
:10BBC000F70A397106DE22DC26DA80004AD84ED622
:10BBD00052D456D23285B28497000000E780C0C7A5
:10BBE000AA89268597000000E78020C92318A4FCB5
:10BBF000268597000000E78040C82319A4FC26850D
:10BC000097000000E78060C783D744000A8A231AA0
:10BC1000A4FC858393F7F70F230EF4FC8607BD077A
:10BC200093F7073F3301F1408A8A01498347C4FDF6
:10BC30006367F902CE85130584FC232C54FD97001D
:10BC40000000E78080EA5281130104FCF250625444
:10BC5000D2544259B259225A925A21618280268581
:10BC600097000000E78060C193171900D697050977
:10BC70002390A7001379F90F55BF828097A7FF1F64
:10BC8000938787F19C43D847A1679387A702631ADC
:10BC9000F70A397106DE22DC26DA80004AD84ED651
:10BCA00052D456D23285B28497000000E780C0BAE1
:10BCB000AA89268597000000E78020BCFD5723183D
:10BCC000A4FC26852319F4FC97000000E780E0BA65
:10BCD00083D744000A8A231AA4FC858393F7F70FBD
:10BCE000230EF4FC8607BD0793F7073F3301F140AD
:10BCF0008A8A01498347C4FD6367F902CE8513052B
:10BD000084FC232C54FD97000000E78000DE528164
:10BD1000130104FCF2506254D2544259B259225ACF
:10BD2000925A21618280268597000000E780E0B466
:10BD300093171900D69705092390A7001379F90FD7
:10BD400055BF828097A7FF1F938707E59C43D8477D
:10BD5000A16789076310F70A397106DE22DC26DA4B
:10BD600080004AD84ED652D456D2328532899700B6
:10BD70000000E78060AEAA894A8597000000E7804E
:10BD8000C0AF835749000A8A2318A4FC858393F720
:10BD9000F70F230CF4FC8607BD0793F7073F330129
:10BDA000F1408A8A8144834784FD63E7F402CE85AB
:10BDB000130584FC232A54FD97000000E780E0D29D
:10BDC0005281130104FCF2506254D2544259B259C8
:10BDD000225A925A216182804A8597000000E780AA
:10BDE000C0A993971400D69785042390A70093F4D5
:10BDF000F40F55BF828097A7FF1F9387E7D99C4315
:10BE0000D847A1679387E704631EF70A397106DEF6
:10BE100022DC26DA80004AD84ED652D456D2328559
:10BE2000B28497000000E78020A3AA8926859700A6
:10BE30000000E78080A42318A4FC2685970000005A
:10BE4000E780A0A3231AA4FC268597000000E780C2
:10BE5000C0A283D744000A8A2319A4FC858393F7E0
:10BE6000F70F230EF4FC8607BD0793F7073F330156
:10BE7000F1408A8A01498347C4FD6367F902CE8590
:10BE8000130584FC232C54FD97000000E780E0C5D7
:10BE90005281130104FCF2506254D2544259B259F7
:10BEA000225A925A21618280268597000000E780FD
:10BEB000C09C93171900D69705092390A700137902
:10BEC000F90F55BF828097A7FF1F9387E7CC9C434C
:10BED000D847A1679387C704631AF70A397106DE4A
:10BEE00022DC26DA80004AD84ED652D456D2328589
:10BEF000B28497000000E7802096AA8926859700E3
:10BF00000000E7808097FD572318A4FC2685231A9C
:10BF1000F4FC97000000E780409683D744000A8A2B
:10BF20002319A4FC858393F7F70F230EF4FC8607EF
:10BF3000BD0793F7073F3301F1408A8A01498347E0
:10BF4000C4FD6367F902CE85130584FC232C54FDE0
:10BF500097000000E78060B95281130104FCF250A1
:10BF60006254D2544259B259225A925A2161828063
:10BF7000268597000000E780409093171900D69718
:10BF800005092390A7001379F90F55BF828097A761
:10BF9000FF1F938767C09C43D847A167DD076317DE
:10BFA000F7041763FFFFE70243107971328532848B
:10BFB00097000000E780408A2AC62285970000008B
:10BFC000E780A08B2311A102228597000000E78063
:10BFD000A088B2452300A102280897000000E7804E
:10BFE000C0B045611763FFFF6700630E828097A7AB
:10BFF000FF1F938767BA9C43D847A167938787043D
:10C000006317F7041763FFFFE702230A797132858C
:10C01000328497000000E78020842AC6228597009A
:10C020000000E78080852311A1022285970000008F
:10C03000E7808082B2452300A10228089700000013
:10C04000E780A0AA45611763FFFF6700430882806D
:10C0500097A7FF1F938747B49C43D847A16793874F
:10C06000A7046312F7021763FFFFE702030401113D
:10C070002800814597000000E78020A7056117632D
:10C08000FFFF6700C304828097A7FF1F9387C7B095
:10C090009C43D847A167938757026319F702176338
:10C0A000FFFFE70283000111328597F0FFFFE78071
:10C0B000A07A2308A1008145280097000000E780AE
:10C0C000C0A205611763FFFF67006300828097A726
:10C0D000FF1F938767AC9C43D847A1679387E7020C
:10C0E000631BF7041763FFFFE70223FC011132858E
:10C0F000328497F0FFFFE7804078AA84228597F08A
:10C10000FFFFE7808077854709E9228597F0FFFFE9
:10C11000E78080744205B337A000280081452318CA
:10C1200091003ECA97000000E780209C05611763DC
:10C13000FFFF6700C3F9828097A7FF1F9387C7A5FA
:10C140009C43D84799476313F7081763FFFFE7023B
:10C15000C3F579713285328497F0FFFFE780C06FB5
:10C160002AC6228597F0FFFFE78020712310A102E5
:10C17000228597F0FFFFE780206E2301A102228530
:10C1800097F0FFFFE780406DA301A102228597F0A1
:10C19000FFFFE780606C2302A102228597F0FFFF7A
:10C1A000E780806B2313A102228597F0FFFFE780D1
:10C1B000A06AB2452314A102280897000000E78076
:10C1C000C09245611763FFFF670063F0828097A705
:10C1D000FF1F9387679C9C43D847A1679387C7033A
:10C1E0006313F7081763FFFFE70223EC79713285C9
:10C1F000328497F0FFFFE78020662AC6228597F0F9
:10C20000FFFFE78080672310A102228597F0FFFFE0
:10C21000E780A0662311A102228597F0FFFFE78047
:10C22000A0632302A102228597F0FFFFE780C0628E
:10C23000A302A102228597F0FFFFE780E0612303BC
:10C24000A102228597F0FFFFE7800061B245A303BA
:10C25000A102280897000000E78020894561176344
:10C26000FFFF6700C3E682801763FFFFE702E3E397
:10C2700001112A8497F0FFFFE780005EAA842285DF
:10C2800097F0FFFFE780605F228597F0FFFFE78070
:10C29000C05E035744008D4763F7E700228597F09F
:10C2A000FFFFE780805D228597F0FFFFE780E05C7D
:10C2B0002800A68597000000E780208305611763AA
:10C2C000FFFF6700C3E097A7FF1F9387E78C9C439E
:10C2D000D847A167FD07631FF7001763FFFFE70259
:10C2E000C3DC328597000000E78040F81763FFFF4A
:10C2F0006700E3DD828097A7FF1F9387E7899C4350
:10C30000D847A167E5076315F7081763FFFFE70242
:10C31000C3D979713285328497F0FFFFE780C0532B
:10C320002AC6228597F0FFFFE7802055228597F0E7
:10C33000FFFFE78080542310A102228597F0FFFFC2
:10C34000E780A053520551812311A10222852302C7
:10C35000010297F0FFFFE7802050A302A10222858F
:10C3600097F0FFFFE780404F2303A102228597F05B
:10C37000FFFFE780604EB245A303A102280897F0B3
:10C38000FFFFE780807645611763FFFF670023D4D6
:10C39000828097A7FF1F938727809C43D847A16778
:10C3A0009387E703631FF7001763FFFFE702E3CFFD
:10C3B000328597000000E78060EB1763FFFF67009E
:10C3C00003D182809797FF1F9387077D9C43D847AF
:10C3D000A16793874704631EF7021763FFFFE70215
:10C3E000C3CC79713285328497F0FFFFE780C04675
:10C3F0002AC6228597F0FFFFE7802048B24528082B
:10C4000097F0FFFFE780606E45611763FFFF6700ED
:10C4100003CC82809797FF1F938707789C43D84768
:10C42000A167938787026310F7041763FFFFE70292
:10C43000C3C779713285328497F0FFFFE780C0412E
:10C440002AC6228597F0FFFFE7800041B24523000E
:10C45000A102280897F0FFFFE78020694561176374
:10C46000FFFF6700C3C682801763FFFFE702E3C3D5
:10C47000011197F0FFFFE780203EAA85280097F082
:10C48000FFFFE780806605611763FFFF670023C435
:10C490009797FF1F938747709C43D847A167D107A1
:10C4A000631FF7001763FFFFE70223C03285970081
:10C4B0000000E780A0FB1763FFFF670043C1828095
:10C4C0009797FF1F9387476D9C43D847A167C50780
:10C4D000631FF7001763FFFFE70223BD3285970054
:10C4E0000000E780A0F81763FFFF670043BE82806B
:10C4F0009797FF1F9387476A9C43D847A167B9075F
:10C50000631FF7001763FFFFE70223BA3285970026
:10C510000000E780A0F51763FFFF670043BB828040
:10C520009797FF1F938747679C43D847A167AD073D
:10C53000631FF7001763FFFFE70223B732859700F9
:10C540000000E780A0F21763FFFF670043B8828016
:10C550009797FF1F938747649C43D8478947631881
:10C56000F7021763FFFFE70243B40111328532C8B7
:10C5700097F0FFFFE780402EAA85280097F0FFFF85
:10C58000E780A05605611763FFFF670043B4828010
:10C590009797FF1F938747609C43D847A1678D07F4
:10C5A0006311F7041763FFFFE70223B0011132851F
:10C5B000328497F0FFFFE780202A13066100AA84E7
:10C5C0004C00228597300000E780C0232800A68514
:10C5D00097F0FFFFE780605105611763FFFF670079
:10C5E00003AF82809797FF1F9387475B9C4381CF60
:10C5F000DC4391CB1763FFFFE70223AB82971763FE
:10C60000FFFF6700C3AC82801763FFFFE702E3A967
:10C6100079713C08AE843ED2A165B7070A002A842E
:10C620003ED448103C08DD053ED636C432C63AC278
:10C6300097D0FFFFE780E02F12474810BA8597F0A8
:10C64000FFFFE780C01332464810B28597F0FFFF26
:10C65000E780E014A2464810B68597F0FFFFE78018
:10C660000012501001478146A685228597D0FFFF12
:10C67000E780805145611763FFFF670043A517639B
:10C68000FFFFE70283A201117C000329C501AE84EC
:10C690003ECAA165B70707002A843ECC48087C0043
:10C6A000C5053ECE97D0FFFFE780A0288345D9007F
:10C6B000480897F0FFFFE780800C5008014781464B
:10C6C000A685228597D0FFFFE780004C05611763A0
:10C6D000FFFF6700C39F1763FFFFE702039D83C748
:10C6E000950093F7F707A384F50097000000E78013
:10C6F00040F91763FFFF6700839D1763FFFFE702A1
:10C70000C39A79713C08AE843ED2A165B70709008F
:10C710002A843ED448103C08938545043ED632C650
:10C7200036C497D0FFFFE780C020A2464810B685E8
:10C7300097F0FFFFE780A00432464810B28597F0DB
:10C74000FFFFE780C005501001478146A68522857E
:10C7500097D0FFFFE780404345611763FFFF670005
:10C7600003971763FFFFE702439483C795004111C6
:10C770002A8493F7F707A384F50032852EC697F035
:10C78000FFFFE780800F85672AC46370F50297700A
:10C790000000E78020E92246B24509ED11478146B5
:10C7A000228597000000E78060E641011763FFFFE4
:10C7B0006700E39101478346F501DDB71763FFFF8B
:10C7C000E702038D01113C003ECAB7070A003ECCC8
:10C7D0003C003ECE83C79500AA89328593F7F707C0
:10C7E000A384F5002E8497F0FFFFE780000985679A
:10C7F000637DF504A165AA8493858504480897D0D4
:10C80000FFFFE7800013268597700000E78080E136
:10C810002A8929E19145480897F0FFFFE78020F633
:10C82000A685480897F0FFFFE78060F7CA854808AB
:10C8300097F0FFFFE780A0F4014781465008A285EA
:10C840004E8597D0FFFFE780203405611763FFFF17
:10C85000670043878145480897F0FFFFE78020F293
:10C860000349090275BF1763FFFFE702638279710D
:10C870001C103ECAB7070F003ECC404D1C10AA84C6
:10C88000AE894808994532C636893ECE97D0FFFF1B
:10C89000E780200A32464808B28597F0FFFFE7801C
:10C8A00000EE630C0902A545480897F0FFFFE780FA
:10C8B000C0E62546CA8597200100E78020A45008DD
:10C8C00001478146CE85268597D0FFFFE780C02BA4
:10C8D00045611753FFFF6700E37E8355C402480894
:10C8E00097F0FFFFE780A0EB0355E402814505C503
:10C8F000854785456301F502C167FD179305F00F74
:10C90000630BF5007D1597700000E780208E93057E
:10C91000150093F5F50F480897F0FFFFE78020E634
:10C9200083450403480897F0FFFFE78040E583450F
:10C930001403480897F0FFFFE78060E48355240361
:10C94000480897F0FFFFE78080E5835544034808D7
:10C9500097F0FFFFE780A0E49DB71753FFFFE702C2
:10C96000C37483C795008146014693F7F707A384F4
:10C97000F50097000000E78040EF1753FFFF6700C6
:10C9800003751753FFFFE702437279713E841C1051
:10C990003ECA2E89B7070F00A1653ECCFD051C10CD
:10C9A000AA84480842C03AC23ECE36C432C697D0A6
:10C9B000FFFFE78000F832464808B28597F0FFFF96
:10C9C000E780E0DBA2464808B68597F0FFFFE780E6
:10C9D00000DD12474808BA8597F0FFFFE78020DCAA
:10C9E0000248630C08029145480897F0FFFFE78072
:10C9F000C0D21146A28597200100E7802090500800
:10CA000001478146CA85268597D0FFFFE780C0177A
:10CA100045611753FFFF6700836B8945480897F00E
:10CA2000FFFFE78080CF834704002300F5008347A2
:10CA30001400A300F500E1B71753FFFFE7024365B9
:10CA400083C7950001112A8A93F7F707A384F5009D
:10CA50003285AE8432C697F0FFFFE78000E23246AF
:10CA60002A89328597F0FFFFE78000DF85676373CF
:10CA7000F902AA894A8597700000E780A0BA2A8443
:10CA800019ED114781464A86A68552859700000018
:10CA9000E780C0B705611753FFFF6700A362938764
:10CAA000E9FF93F7F70F0547E366F7FE8347F501C4
:10CAB00095EB8947E380F9FE8346F40152850147EF
:10CAC0004A86A68597000000E78040B4A167D90791
:10CAD00048083ECC230A010002CE97000000E78000
:10CAE000A0B04DBF639EE7008947639EF90093079E
:10CAF0001020231FF50097700000E780C0B76DBFBE
:10CB00000947E39BE7FA8D47E398F9FA2285977086
:10CB10000000E78080DF9797FF1F938727279C43BC
:10CB200099E79797FF1F938727109C4399C703D5D1
:10CB3000040097800000E780A0CE231F0400228518
:10CB40005DBF1753FFFFE702435601113C003ECA89
:10CB5000B7070B003ECC3C003ECE83C795002A8928
:10CB6000328593F7F707A384F500AE8497F0FFFFB3
:10CB7000E780A0D093170501C187635AF006A1652D
:10CB80002A849385E502480897D0FFFFE78060DAA2
:10CB9000A285480897F0FFFFE78060C09797FF1FC6
:10CBA000938787089C43A9EB01449375F40F4808C9
:10CBB00097F0FFFFE780A0BC9355844093F5F50FF5
:10CBC000480897F0FFFFE78080BB9355044193F539
:10CBD000F50F480897F0FFFFE78060BA01478146EC
:10CBE0005008A6854A8597D0FFFFE780E0F90561E8
:10CBF0001753FFFF6700A34D416585460546A28593
:10CC00007D1597500000E78060BD59DD5105970004
:10CC10000100E780808F130440063344850271B71A
:10CC20001753FFFFE70263480111B70706003EC62E
:10CC300083C7950021642A8993F7F707A384F50039
:10CC4000AE8428009305A4040AC40AC897D0FFFF45
:10CC5000E78020CE300001478146A6854A8597D0DF
:10CC6000FFFFE78060F297E0FFFFE7808015130485
:10CC70009404480822CC230A010002CE9700000049
:10CC8000E780809605611753FFFF67004344175301
:10CC9000FFFFE702E33FC1642A8901449799FF1F20
:10CCA00093894910130A8002FD1497E0FFFFE78083
:10CCB00080C16347A40001451753FFFF670083400D
:10CCC000B307440303A7C90ABA9703D7070063064B
:10CCD000970083D72700638427010504F9B705452A
:10CCE000E1BF1753FFFFE702A33A2A8A2E8999C1B1
:10CCF00023A0050081498144979AFF1F938A4AEA3D
:10CD0000614B97E0FFFFE78040C263C7A4004E85F8
:10CD10001753FFFF6700033B3384640383A70A00B4
:10CD20003E948357040099E7630409002320890097
:10CD30008504C1BF4146D285130544009710010008
:10CD4000E780605975F5A289E5B71753FFFFE70241
:10CD5000233439717C083ED4B7070A003ED67C08DC
:10CD60003ED883C795002A8A328593F7F707A384B4
:10CD7000F5002E8932C697F0FFFFE78000B0856787
:10CD80006373F5083246AA84328597F0FFFFE78087
:10CD9000A0AC8547AA8963E8A706A16593858504A9
:10CDA000281097D0FFFFE780C0B826859770000055
:10CDB000E78040872A8429ED9145281097F0FFFFEE
:10CDC000E780E09BA685281097F0FFFFE780209D75
:10CDD000CE85281097F0FFFFE780609A01478146D3
:10CDE0003010CA85528597D0FFFFE780E0D9A16750
:10CDF0009387770448183EDC230A010202DE97F08D
:10CE0000FFFFE780607E21611753FFFF6700832BE0
:10CE10008145281097F0FFFFE7806096A6852810CF
:10CE200097F0FFFFE780A0979797FF1F9387472E04
:10CE30009C4381CB22856389090097D00000E7805D
:10CE400040248345040271B797D00000E780C022D8
:10CE5000CDBF1753FFFFE702A32383C795004111FE
:10CE6000AA8993F7F707A384F5003285AE84328A46
:10CE700097F0FFFFE78060A08567637FF5022A894E
:10CE800097600000E780007A2A84914631C5834785
:10CE9000F50105476387E70291C70D476366F7040D
:10CEA000AD461DA89305050303250A0041469710CA
:10CEB0000100E78040420DE941011753FFFF670081
:10CEC00063209305950803250A0041469710010049
:10CED000E7806040814669F54A86A6854E859700C1
:10CEE0000000E780C081C9BF83250A0013059408AC
:10CEF00097700000E780A02919C1C146F1BF97973C
:10CF0000FF1F9387A7E89C4399E79797FF1F938795
:10CF1000A7D19C4399C7228597800000E780208A8B
:10CF200069FD8547A30FF400228597B00000E780D4
:10CF30006084228597600000E780E0734E8581461B
:10CF40004A86A68597F0FFFFE780607BA1679387FD
:10CF5000570448003EC42302010002C697F0FFFFB9
:10CF6000E780806891BF1753FFFFE702831183C7F3
:10CF700095004111AA8993F7F707A384F50032853C
:10CF80002E89B28A97F0FFFFE780208F8567637450
:10CF9000F50EAA8497600000E780C0682A840DED32
:10CFA000416B014A979BFF1F938BCBDF130C400E05
:10CFB0007D1B19A833048A0383A70B0B3E94835768
:10CFC000C40163836705050A97E0FFFFE780A08E31
:10CFD000E342AAFE95460DA08357C50163969702CA
:10CFE0009305050303A50A00414697100100E78059
:10CFF000802E994611E181462686CA854E8597F096
:10D00000FFFFE780C06F85A883A50A00130504030E
:10D0100097700000E780A017C14679FD2285231E86
:10D02000940097A00000E780E074228597600000DC
:10D03000E78060649797FF1F9387870D9C43A9C380
:10D0400023000402228597D00000E78040F04E853F
:10D0500081462686CA8597F0FFFFE780406AA16770
:10D060009387070448003EC42302010002C697F0DC
:10D07000FFFFE780605741011753FFFF6700E3039D
:10D0800089472300F402E1B7397106DE22DC4AD871
:10D09000800052D456D25AD026DA4ED65ECE2E8A90
:10D0A00032892A8B97D0FFFFE780E07D0605710566
:10D0B00041998A8A3301A140232224FC231404FCD1
:10D0C00097D0FFFFE780207C83479A00060535054F
:10D0D00093F7F7072315A4FCA304FA004A85232637
:10D0E00024FC97E0FFFFE780407993170501C18793
:10D0F0006340F0025681130104FCF2506254D25492
:10D100004259B259225A925A025BF24B21618280F3
:10D11000AA844A8597E0FFFFE7802076AA894A859E
:10D1200097E0FFFFE7806075A1659385C5022A89B6
:10D13000130544FC97C0FFFFE780A07F268597C0BA
:10D14000FFFFE780E073854511C94A86CE8597C009
:10D15000FFFFE780606DAA8B21E98945130544FC38
:10D1600097E0FFFFE780A061A685130544FC97E0E8
:10D17000FFFFE780C062CE85130544FC97E0FFFF08
:10D18000E780E061CA85130544FC97E0FFFFE78074
:10D19000006101478146130644FCD2855A8597D029
:10D1A000FFFFE780609EB9B78145130544FC97E017
:10D1B000FFFFE780C05CA685130544FC97E0FFFFF6
:10D1C000E780E05DCE85130544FC97E0FFFFE78034
:10D1D000005DCA85130544FC97E0FFFFE780205CF3
:10D1E000814497D0FFFFE780006AE3D4A4FA83A7C5
:10D1F0000B0113971400BA9783D5070099C513053F
:10D2000044FC97E0FFFFE78080598504D9BF79711E
:10D2100006D622D44AD000184ECE52CC56CA26D2B8
:10D220005AC8AE893289AA8A97D0FFFFE780A065E5
:10D230000605690541990A8A3301A140232A24FC85
:10D24000231C04FC97D0FFFFE780E06383C79900AD
:10D2500006052D0593F7F707231DA4FCA384F90009
:10D260004A85232E24FC97E0FFFFE7800061931797
:10D270000501C187634FF0005281130104FDB250D4
:10D28000225492540259F249624AD24A424B4561B1
:10D290008280AA844A8597E0FFFFE780005EA1654F
:10D2A0009385A5022A89130544FD97C0FFFFE780F7
:10D2B0004068268597C0FFFFE780805C854509C9E7
:10D2C000CA8597C0FFFFE78020592A8B29E189454D
:10D2D000130544FD97E0FFFFE780604AA68513052C
:10D2E00044FD97E0FFFFE780804BCA85130544FDAE
:10D2F00097E0FFFFE780A04A01478146130644FDFF
:10D30000CE85568597D0FFFFE7800088B5B7814569
:10D31000130544FD97E0FFFFE7806046A6851305EF
:10D3200044FD97E0FFFFE7808047CA85130544FD71
:10D3300097E0FFFFE780A046814497D0FFFFE7809A
:10D340008054E3DBA4FA83270B0113971400BA97E8
:10D3500083D5070099C5130544FD97E0FFFFE780DB
:10D3600000448504D9BF1753FFFFE70203D4834766
:10D370004500404DD5EFFD575DC4834694000947F5
:10D380006363D70A0346B400854663EEC608830686
:10D39000E40063CA06085C45F9562390D7009797C6
:10D3A000FF1F83C7278099E3A304E4009797FF1F1B
:10D3B000938787879C4381E78947A306F400979763
:10D3C000FF1F9387E7D49C4381E789472306F40036
:10D3D0009705000093854506AA841305040197F07C
:10D3E0000000E7802010FD57231AF40281471CDC5F
:10D3F00001489787FF1F23A3877A9787FF1F93878B
:10D40000277A232E040304C0804397D0FFFFE780D0
:10D41000C05161463306C502814522859750FFFF02
:10D42000E780A0CB81473E851753FFFF670023CAE3
:10D43000FD57D5BF1753FFFFE70223C72A840355C3
:10D44000450297600000E780E01D19E5231E0400F7
:10D450001753FFFF6700A3C78357E401F5DB93056C
:10D4600004FF174501001305652197E00000E780E0
:10D47000E014F9BF1753FFFFE70223C32E89A1650C
:10D4800041119385E5032A8436C432C6BE843AC26C
:10D4900097C0FFFFE780E04912472285BA8597E0F1
:10D4A000FFFFE780C02D32462285B28597E0FFFF5F
:10D4B000E780E02EA2462285B68597E0FFFFE78051
:10D4C000002E630309029145228597E0FFFFE78064
:10D4D000C0241146A68597100100E78020E2410193
:10D4E0001753FFFF6700A3BE8945228597E0FFFF22
:10D4F000E780A02283C704002300F50083C714003F
:10D50000A300F500E9BF1753FFFFE70203BA83C783
:10D510009500444D054793F7F707A384F5001C4297
:10D52000411183C707006367F7062E842A89B1C0BB
:10D5300003C7D400630FF7021787FF1F1307C76ED7
:10D54000184305C3A386F40097A00000E780404A73
:10D5500083C7D40099E741657D1597400000E780B7
:10D56000403083D72403918B89C797E00000E78080
:10D57000C0134A85A28597F0FFFFE7808010A1675E
:10D58000C10748003EC42302010002C697F0FFFF16
:10D59000E780800541011753FFFF670043B317532E
:10D5A000FFFFE70283B003D745008D47AA844111EE
:10D5B0002E8432892E8563E3E70297E0FFFFE78040
:10D5C000C02BAA8523000900268597C0FFFFE780AE
:10D5D000A02841011753FFFF670063AF97E0FFFFEB
:10D5E000E780A0292AC6228597E0FFFFE780E02890
:10D5F000B24585472A862300F900268597C0FFFF9C
:10D60000E7808022F9B7397106DE22DC26DA800055
:10D610004ED652D456D24AD85AD05ECEAE89B284B3
:10D62000AA8A97D0FFFFE78000250605130525028B
:10D6300041990A8A3301A140232224FC231404FCCB
:10D6400097D0FFFFE780202383C7990006054D058B
:10D6500093F7F7072315A4FCA384F9002685232656
:10D6600024FC97E0FFFFE780402193170501C18765
:10D670006340F0025281130104FCF2506254D25410
:10D680004259B259225A925A025BF24B216182806E
:10D69000AA8B03AB040097C0FFFFE780601E51E533
:10D6A00083D7440001498544F11793B71700A301BC
:10D6B000F4FC834734FCA165C9C79385E5041305D1
:10D6C00044FC97C0FFFFE780C026A685130544FCF5
:10D6D00097E0FFFFE780A00ADE85130544FC97E092
:10D6E000FFFFE780C00B834734FC114691E30946F6
:10D6F000DA85130544FC97E0FFFFE780600581446D
:10D70000630A0900416B7D1B97D0FFFFE780A016DD
:10D7100063CCA40201478146130644FCCE8556859E
:10D7200097C0FFFFE7804046B1B7A685130634FCDB
:10D7300097000000E780E0E6933415002A8986040C
:10D740008DBF9385C504A5BF8327C9001397140017
:10D75000BA9783D5070063886501130544FC97E0F9
:10D76000FFFFE780C003850445B71753FFFFE702BB
:10D77000439179711C103EC4B7070F003EC61C10C0
:10D780003EC883C79500AA8A328593F7F707A3841A
:10D79000F500AE89328497E0FFFFE780000E931713
:10D7A0000501C187635AF0062A8A228597E0FFFFA8
:10D7B000E780A00C2A895285032B040097C0FFFF45
:10D7C000E780000C39ED8357440081440544F1178C
:10D7D00093B71700A303F10083457100DA8722870E
:10D7E000CA865286280097000000E780E0C80147FB
:10D7F00081463000CE85568597C0FFFFE780C03850
:10D80000A1679387D70348083ECC230A810026CE20
:10D8100097F0FFFFE78040DD45611753FFFF67008A
:10D82000C389A2851306710097000000E78060D7C6
:10D83000AA84094455D13544E30055FB4A8597F045
:10D84000FFFFE78000450D4441D9014497D0FFFF19
:10D85000E7806002634DA400C16B0144FD1B97D0BB
:10D86000FFFFE7804001634EA4001544B5B7DC44D8
:10D8700013171400BA9783D707006383270305049F
:10D88000F1B7D84493171400BA9703D70700631B66
:10D89000770123902701268597A00000E78080DB91
:10D8A00001441DBF050465BF1743FFFFE702437E28
:10D8B00083C7950041112A8A93F7F707A384F500DF
:10D8C00032852E89328497E0FFFFE78000FB9317B3
:10D8D0000501C1876353F006AA89228597E0FFFFFF
:10D8E000E780A0F92311A1004E85832A040097C088
:10D8F000FFFFE780E0F839E58357440085440144A1
:10D90000F11793B71700A300F10003481100035764
:10D910002100D6875285CE862686CA8597F0FFFFDE
:10D92000E7806006A167F10748003EC4230291002A
:10D9300022C697F0FFFFE78020CB41011743FFFF8E
:10D9400067004378A2851306110097000000E78066
:10D9500040C52A84894455D98357210011678544DD
:10D96000BA97C2071167C1831307F7EFE36FF7F8A0
:10D970009787FF1F938787419C4381CB854513057C
:10D98000210097500000E7802075835521002285F3
:10D99000814497C0FFFFE78040E525D923100500AB
:10D9A000228597A00000E78040CD85B71743FFFF91
:10D9B000E702236D83C7950041112A8B93F7F70780
:10D9C000A384F50032852E8A328497E0FFFFE7803A
:10D9D000C0EA93170501C1876351F006AA8A228520
:10D9E00097E0FFFFE78060E92A895685832B0400D2
:10D9F00097C0FFFFE780C0E831E5835744008144CA
:10DA00000544F11793B71700A301F1000348310053
:10DA1000DE875A854A87D6862286D28597F0FFFF11
:10DA2000E78060F6A167ED0748003EC4230281004D
:10DA300026C697F0FFFFE78020BB41011743FFFF99
:10DA40006700A367A2851306310097000000E780F6
:10DA500040B5AA8409445DD99167CA97C207116786
:10DA6000C1831307F7EF0544E362F7FACA8597C04D
:10DA7000FFFFE78080D7014451F9814997D0FFFF2C
:10DA8000E78060E063DBA900984893971900BA9794
:10DA900003D7070005EF2390270197D0FFFFE7800A
:10DAA00080DE1544E384A9F6268597A00000E78070
:10DAB000C0BC9787FF1F9387672D9C430144B9D74C
:10DAC0004A8597500000E780C05889B785097DB71F
:10DAD0001743FFFFE702C35B79713E847C083EC8B1
:10DAE0002E8AB7071400A1653ECAE5057C08AA89FD
:10DAF000080836C4428932C6BA8AC6843ECC97C06A
:10DB0000FFFFE78000E3CA85080897E0FFFFE78092
:10DB100000C732460808B28597E0FFFFE78020C8BB
:10DB2000A246630A09049D45080897E0FFFFE780C5
:10DB3000C0BE1D4681459740FFFFE780005A6389BC
:10DB40000A089145080897E0FFFFE78000BD1146ED
:10DB5000A68597000100E780607A1008014781469A
:10DB6000D2854E8597C0FFFFE780000245611743CD
:10DB7000FFFF67002355B685080897E0FFFFE780A1
:10DB800000C21C400808D8439355C7018589120775
:10DB90005183B205D98D97E0FFFFE78040C01C405C
:10DBA000080883C5870097E0FFFFE78040BD1C4061
:10DBB000080883C5A70097E0FFFFE78040BC1C4032
:10DBC000080883C5970097E0FFFFE78040BB85BF4B
:10DBD0008945080897E0FFFFE78020B483C7040069
:10DBE0002300F50083C71400A300F500BDB7174359
:10DBF000FFFFE702E34983C795004111AA8993F724
:10DC0000F707A384F5003285AE84328497E0FFFFE6
:10DC1000E780A0C693170501C187635DF0042A89D8
:10DC2000032A040097C0FFFFE78080C519E98357E6
:10DC300044000548F11793B71700A307F100814688
:10DC400031A81306F100A28597000000E7806095D7
:10DC50001DC51C459DC783D6470001480347F100F9
:10DC600093078500D2884A86A6854E8597000000D6
:10DC7000E78040E641011743FFFF6700A3440948DE
:10DC80007DBF1D486DBF1743FFFFE702634065710D
:10DC90005C083EC4B7077B013EC65C083EC883C72C
:10DCA00095002A8A328593F7F707A384F500AE8999
:10DCB00097E0FFFFE78040BA8357E100E1C789455D
:10DCC000280097C0FFFFE780C0C68145280097E085
:10DCD000FFFFE780C0AA97C0FFFFE780A0CC97872F
:10DCE000FF1F9387E7429C431784FF1F034484EB85
:10DCF000AA843334800099C3136424009787FF1FDC
:10DD0000938787F29C4399C3136444009787FF1F4E
:10DD10009387C7079C4399C31364840083D5040089
:10DD20002800014997E0FFFFE78060A783D5240022
:10DD3000280097E0FFFFE78080A683D544002800F5
:10DD400097E0FFFFE780A0A597D0FFFFE780A0AE98
:10DD500093150501C181280097E0FFFFE78020A40B
:10DD6000A285280097E0FFFFE78060A39C446360E2
:10DD7000F902014781463000CE85528597C0FFFFEA
:10DD8000E78080E059611743FFFF6700A333DC445D
:10DD90001314490028003E9497E0FFFFE780609647
:10DDA000834744000347540089070607BA9786074C
:10DDB000E36AF5FC835524002800814A97E0FFFFC1
:10DDC000E780E09D83454400280097E0FFFFE7805F
:10DDD000009B83455400280097E0FFFFE780209ACE
:10DDE0008347440063C9FA00814A8347540063C1F2
:10DDF000FA020509A5BF1C4413975A002800BA97D8
:10DE000083D50700850A97E0FFFFE7804099C9BFE7
:10DE1000032BC40093975A0028003E9B83552B0088
:10DE2000850A97E0FFFFE780809783550B00280065
:10DE300097E0FFFFE780A0964DBF1743FFFFE70283
:10DE4000C3265C4993E717005CC997A00000E780F0
:10DE500020B61743FFFF670083271743FFFFE70242
:10DE6000C3242E84814597F0FFFFE780C0E705C5F6
:10DE700083570500FD172310F50009C483572500BB
:10DE80002310F40097000000E78060FB0145174372
:10DE9000FFFF6700C32331457DD823100400C5BFB1
:10DEA0001743FFFFE702C31E83C7950041112A8A6B
:10DEB00093F7F707A384F50032852E89328497E023
:10DEC000FFFFE780809B93170501C1876356F0062B
:10DED000AA89C145228597E0FFFFE780A0802A8BB1
:10DEE0004E85832A040097C0FFFFE780609931E9DF
:10DEF00083574400231101000544F11793B717001D
:10DF0000A300F10081440348110003572100D68784
:10DF10005285CE862286CA8597F0FFFFE780A0A6AD
:10DF2000A1679387170248003EC42302810026C6DA
:10DF300097E0FFFFE780406B41011743FFFF670059
:10DF4000631813061100A28597F0FFFFE780606554
:10DF5000AA8409E523110100094475B7930521003E
:10DF60005A8597000000E78080EF835721002A84BC
:10DF7000D9DB9787FF1F938767E19C4381CB85455A
:10DF80001305210097500000E780001583552100FC
:10DF90002685314497C0FFFFE78020852DD52310CB
:10DFA0000500268597900000E780206D0144A1BF01
:10DFB0001743FFFFE702630F41112E896C00AA840B
:10DFC00002C697F0FFFFE78000D20DC1035705009E
:10DFD00005072310E50097000000E78040E6814731
:10DFE0003E8541011743FFFF6700630E32479547A7
:10DFF00065DBCA85268597300000E780400DC14764
:10E00000E34005FE3244854741462310F400835720
:10E010000900A685130544002311F40097000100B0
:10E02000E780C02D228545BF1743FFFFE702430667
:10E0300083C795004111AA8A93F7F707A384F500D7
:10E040003285AE89328497E0FFFFE7800083931723
:10E050000501C1876356F0062A8AC145228597D0FB
:10E06000FFFFE7802068AA845285032B040097C035
:10E07000FFFFE780E08031E983574400231101006E
:10E080008544F11793B71700A300F100014403483A
:10E09000110003572100DA875685D2862686CE8561
:10E0A00097F0FFFFE780208EA16793870702480063
:10E0B0003EC42302910022C697E0FFFFE780C052D2
:10E0C00041011743FFFF6700E3FFA285130611001C
:10E0D00097F0FFFFE780E04C2A8409E52311010057
:10E0E000894475B726859305210097000000E780D5
:10E0F00060ECAA8449FD83552100228597B0FFFF7B
:10E10000E780A06E49F5014997C0FFFFE780A0773F
:10E11000635DA900184893171900BA9703D7070041
:10E120000DEF035721002390E70097C0FFFFE78022
:10E130008075630625039787FF1F938727C59C4338
:10E1400099C70355210097500000E78080F0228591
:10E1500097900000E78060521DBF050975B7954490
:10E160003DB705C19307F00F630FF500C547630C7A
:10E17000F5009307F5FF05453315F500420541818C
:10E1800082800145828041657D158280B9E917430F
:10E19000FFFFE70283F10345060332849700000086
:10E1A000E78060FC9305803EB305B502C205C181DE
:10E1B00081CD0357E402854763F8E70013050401A6
:10E1C00097E00000E78020428357E40241677D1713
:10E1D0006385E700FD172317F4021743FFFF67006D
:10E1E00003EF82801743FFFFE702A3E9004283C7E2
:10E1F0009500444D0349140093F7F707A384F500F5
:10E2000083470400220911673369F900A167B34706
:10E21000F90041112A8BAE8A63ECE70E8347240094
:10E220001307C00EB91793F7F70F6373F71003477F
:10E230003400C14763EEE70E834744001307E0074D
:10E2400093C707086371F70C834984008347740000
:10E25000A209B3E9F900856763F7F90A034A640084
:10E26000834754004E85220A336AFA009750000013
:10E27000E780403B61C123962403834B3400137A2B
:10E28000FA00239A3403238874032399440393895F
:10E290000401631C090023A60402239804024E858E
:10E2A00097E00000E78060363DA0034924004A85DE
:10E2B00097000000E78020EB2397A40283474400E7
:10E2C0004E85A388F402E38D0BFCE30B09FC97E079
:10E2D0000000E780202F97900000E78000738146C0
:10E2E0000146D6855A8597E0FFFFE7800058A16771
:10E2F000938797033EC423020100480002C697E0BB
:10E30000FFFFE780602E41011743FFFF6700E3DA5C
:10E310008544A2862686D6855A8597E0FFFFE7804A
:10E32000C054A167938797033EC423029100F1B7BD
:10E33000BD44C5B79144F1BF1743FFFFE70243D582
:10E3400001111C08404D3EC2B7070F003EC41C0817
:10E350003EC62A89AE8997C0FFFFE780A0DA585CE5
:10E360001C5C6346B70E6394E50063E2A70E338539
:10E37000A740B3B7A700B305B7401306803E814658
:10E380009D8D97000100E78080B793140501C1803F
:10E39000A1659385C503480097B0FFFFE7806059EA
:10E3A0008145480097D0FFFFE780603D8355040416
:10E3B000480097D0FFFFE780803E83552404480043
:10E3C00097D0FFFFE780A03D814589CCC167FD174D
:10E3D0009305F00F6388F400268597500000E780CE
:10E3E000E0E0AA85480097D0FFFFE7804039035559
:10E3F0004404814501CDC167FD179305F00F630704
:10E40000F50097500000E78060DEAA85480097D0AD
:10E41000FFFFE780C03683456404480097D0FFFFC4
:10E42000E780E03583457404480097D0FFFFE7801C
:10E430000035500001478146CE854A8597B0FFFFE1
:10E44000E780807405611743FFFF6700A3C781441D
:10E4500081B71743FFFFE70243C583C7950093F7D2
:10E46000F707A384F50097000000E78020ED17432D
:10E47000FFFF6700C3C51743FFFFE70263C183C700
:10E4800095004111404D93F7F707A384F5002A8AC0
:10E490003285B284AE8997D0FFFFE780003E2A8B99
:10E4A000268597D0FFFFE780403D2A89268597D0B3
:10E4B000FFFFE780603A93170B0163CA0702E17719
:10E4C000CA97C207C183116763E3E7029307091084
:10E4D000C207C1831307B00F637BF70093170901CD
:10E4E000C187AA8A634AF000C54763FE570141010C
:10E4F0001743FFFF670003BD97B0FFFFE780C02809
:10E50000E31725FFD5B763080B02630609028144B0
:10E5100063890A02B7077F002310640523112405CD
:10E520007CC0568597000000E780E0C39304803EDE
:10E53000B304950239A0B7077F00232004047CC0F0
:10E5400081440355240497E00000E780A0A3A1C400
:10E5500097C0FFFFE78000BB269593D7F441333780
:10E560009500AE97BA9708DC5CDCCE8552859700A3
:10E570000000E780A0DC99E023220404A1679387D0
:10E58000B70348003EC42302010002C697E0FFFF24
:10E59000E7808005A9BF814701481CDC232E0403C6
:10E5A000E9B71743FFFFE70243B097C0FFFFE780DB
:10E5B000C037E1473305F502914597500000E780E9
:10E5C00000C5E55711C59777FF1F23ABA75C8147AF
:10E5D0003E851743FFFF670083AF85471777FF1F0F
:10E5E0002302F75C82801743FFFFE70203AC9777B3
:10E5F000FF1F9387A75A80433DC08357040463904D
:10E60000A70683572404639CB7043689B28497C055
:10E61000FFFFE78020AF5C5C63C3B7046395B7007E
:10E620001C5C63EEA7028347640463F3F400A687CF
:10E630002303F4048347740463F39700A687A303BA
:10E64000F4048357440441677D176385E700850719
:10E650002312F4043C4481C7CA8526858297174358
:10E66000FFFF6700C3A69777FF1F938727539C433D
:10E67000014599C303C5870082801743FFFFE70266
:10E68000C3A20111B70707003EC683C79500584DC6
:10E690000AC493F7F7070AC8A384F5002A89AE8451
:10E6A00011CB1C4283C707002304F700979000009A
:10E6B000E7800034216493055402280097B0FFFFDF
:10E6C000E780202797000000E78020FAAA8528002D
:10E6D00097D0FFFFE780A00A300001478146A6855A
:10E6E0004A8597B0FFFFE780204A13044402480898
:10E6F00022CC230A010002CE97E0FFFFE780C0EEA4
:10E7000005611743FFFF6700839C1743FFFFE70284
:10E71000C39901117C003ECAB70707003ECC7C00BC
:10E720003ECE83C795002E84AA8493F7F707A3846F
:10E73000F500A16593855502480897B0FFFFE78073
:10E74000401F97000000E78040F2AA85480897D054
:10E75000FFFFE780C002500801478146A285268559
:10E7600097B0FFFFE780404205611743FFFF670056
:10E7700003969777FF1F938767429C43094599C388
:10E7800003C5970082809777FF1F938727419C439B
:10E79000094599C303C5D70082809777FF1F9387E8
:10E7A000E73F9C43014599C303C5A70082801743F7
:10E7B000FFFFE702E38D0111B70708003EC683C7DC
:10E7C0009500404D0AC493F7F7070AC8A384F500E3
:10E7D0002A89AE8429C41442854703C7060063E032
:10E7E000E70A83479400094681496380C702B3075B
:10E7F000F740A304E400B339F00083C716002305F3
:10E80000F40097900000E780A01E03572403058BB7
:10E8100019C76386090097D00000E78000E92164EA
:10E8200093058402280097B0FFFFE78080109700CF
:10E830000000E78040F4AA85280097D0FFFFE7801A
:10E8400000F497000000E78080F5AA85280097D0A3
:10E85000FFFFE780C0F2014781463000A6854A8568
:10E8600097B0FFFFE780403213047402480822CCBF
:10E87000230A010002CE97E0FFFFE780E0D60561A2
:10E880001743FFFF670003841743FFFFE702E3819D
:10E8900001117C003ECAB70708003ECC7C003ECE8A
:10E8A00083C795002E84AA8493F7F707A384F50005
:10E8B000A16593858502480897B0FFFFE780600750
:10E8C00097000000E78020EBAA85480897D0FFFF5B
:10E8D000E780E0EA97000000E78060ECAA8548083E
:10E8E00097D0FFFFE780A0E9500801478146A28545
:10E8F000268597B0FFFFE780202905611733FFFFCA
:10E900006700E37C9777FF1F938747299C43014566
:10E9100099C303C5B70082801733FFFFE702E3788E
:10E920000111B70707003EC683C79500404D0AC4D2
:10E9300093F7F7070AC8A384F5002A89AE8405C8AF
:10E940001C42054783C707006368F7060347B40006
:10E95000630FF700A305F40097900000E7804009DB
:10E960008347B400B9CF97D0FFFFE78040BE216452
:10E970009305B400280097B0FFFFE78080FB970065
:10E980000000E78060F8AA85280097D0FFFFE780A5
:10E9900000DF014781463000A6854A8597B0FFFF1A
:10E9A000E780801E2904480822CC230A010002CEF9
:10E9B00097E0FFFFE78040C305611733FFFF670063
:10E9C000037197D0FFFFE78020BF55B71733FFFFD4
:10E9D000E702A36D01117C003ECAB70707003ECCD9
:10E9E0007C003ECE83C795002E84AA8493F7F70758
:10E9F000A384F500A165AD05480897B0FFFFE78047
:10EA000040F397000000E78020F0AA85480897D0DF
:10EA1000FFFFE780C0D6500801478146A2852685C2
:10EA200097B0FFFFE780401605611733FFFF6700CF
:10EA3000036A9777FF1F938767169C43094599C31D
:10EA400003C5C70082801733FFFFE7020366011189
:10EA50007C00AE843ECAA165B70707002A843ECC7D
:10EA6000D1057C0048083ECE97B0FFFFE78060EC00
:10EA700097000000E78020FCAA85480897D0FFFF98
:10EA8000E780E0CF500801478146A685228597B0F0
:10EA9000FFFFE780600F05611733FFFF6700236307
:10EAA0001733FFFFE702636083C7950093F7F7070B
:10EAB000A384F50097000000E78020F91733FFFFDB
:10EAC0006700E3601733FFFFE702835C83C79500AD
:10EAD0000329C501411193F7F707A384F5001C42F0
:10EAE00083C90700854763E637079777FF1F93873A
:10EAF00027629C432E84AA8485CF97000000E7807C
:10EB000080F389476306F502630409028347C9005D
:10EB1000638037032306390197900000E78040EDBA
:10EB200083572903898B89C797D00000E780E0B716
:10EB30002685A28597000000E78020F1A167CD0718
:10EB400048003EC42302010002C697E0FFFFE780B1
:10EB5000A0A941011733FFFF6700C3569777FF1F36
:10EB60009387C7039C431D4599C303C5E700828073
:10EB70001733FFFFE70263530111B70707003EC6D3
:10EB800083C79500584D0AC493F7F7070AC8A384B2
:10EB9000F5002A89AE8415C71C4283C707009396E7
:10EBA0008701E18663C4060685466381D7068346EE
:10EBB000E7006388F6002307F70097900000E780DE
:10EBC00020E321649305E400280097B0FFFFE7806D
:10EBD00040D697000000E780A0F8AA85280097D0CB
:10EBE000FFFFE780C0B9014781463000A6854A850E
:10EBF00097B0FFFFE78040F93504480822CC230A8C
:10EC0000010002CE97E0FFFFE780009E0561173309
:10EC1000FFFF6700C34B1733FFFFE70203490111F2
:10EC20007C003ECAB70707003ECC7C003ECE83C7BF
:10EC300095002E84AA8493F7F707A384F500A165B5
:10EC4000B905480897B0FFFFE780A0CE9700000005
:10EC5000E78000F1AA85480897D0FFFFE78020B23F
:10EC6000500801478146A285268597B0FFFFE780BF
:10EC7000A0F105611733FFFF670063451733FFFFFE
:10EC8000E7020341AA8401441779FF1F130949F1E0
:10EC9000E14997C0FFFFE78040C96344A4000145F4
:10ECA00019A833053403832709003E9583572500AF
:10ECB0006397970011051733FFFF6700A340050412
:10ECC000C9BF032E8500630A0E121773FF1F1303BB
:10ECD000E30B03230300631503002943639006122B
:10ECE00003234E01631503001D4363990710173377
:10ECF000FFFFE7020339C689428A3E89BA8AB68491
:10ED0000328BAE8B2A84B5E103554E0019E50143E1
:10ED10001A851733FFFF6700433AA167A98F116770
:10ED200063FBE70097000000E78080F5814597F0DE
:10ED3000FFFFE780C0120844B70700E05841F98F91
:10ED400018455CC1B707001FF98F1CC55C4991C706
:10ED5000610597E00000E780408BE38A09FA22858D
:10ED600097900000E78060C65DB7328597C00000CD
:10ED7000E78040430D4349DD1C44116703D547003C
:10ED8000A167A98F63FBE70097000000E78040EFD1
:10ED9000814597F0FFFFE780800C032384009316E2
:10EDA0004B01D1828347B300035663008588FD8BF6
:10EDB000A305F300FD777D8E558EFD76FD16B2041A
:10EDC000F18E83274301C58E231273012313D300D1
:10EDD0002304530123052301A3044301BDDF22853E
:10EDE00097B0FFFFE78020CDAA850844B5D1610523
:10EDF00097D00000E780207F8DB71D431A85828061
:10EE00001733FFFFE702C3280569AA84AE89328A57
:10EE10000144FD5A7D1997C0FFFFE780C0A56347F5
:10EE2000A40001451733FFFF6700C329D844931797
:10EE30001400BA9703D70700631F370323905701C5
:10EE400063070A00268597900000E780A0809C4415
:10EE50009DC383D76700B3F72701639E3701D2882C
:10EE60000148814701478146014681452685970033
:10EE70000000E78040E5050479BF1733FFFFE70294
:10EE8000232179711C103EC4B7070F003EC61C1029
:10EE90003EC883C79500AA8A328593F7F707A384F3
:10EEA000F5002E89328497D0FFFFE780009D9317ED
:10EEB0000501C187635AF006AA89228597D0FFFF12
:10EEC000E780A09B2A8A4E85032B040097B0FFFFA2
:10EED000E780009B39ED8357440081440544F117D6
:10EEE00093B71700A303F10083457100DA872287E7
:10EEF000D2864E86280097E0FFFFE780E057014763
:10EF000081463000CA85568597B0FFFFE780C0C7AD
:10EF1000A1679387F70348083ECC230A810026CED9
:10EF200097D0FFFFE780406C45611733FFFF670014
:10EF30006319A2851306710097E0FFFFE780606602
:10EF4000AA84094455D1528597E0FFFFE78060D439
:10EF50000D4459D90546D285268597000000E780E3
:10EF600060EA2A8451B71733FFFFE7020314835581
:10EF700007000346270041112A842E8532C62EC47D
:10EF800097E0FFFFE780E0D001C93246A245228525
:10EF900097000000E78000E741011733FFFF67009B
:10EFA00003131733FFFFE702C30D83C79500411119
:10EFB000AA8A93F7F707A384F5003285AE893284D5
:10EFC00097D0FFFFE780608B93170501C1876357D8
:10EFD000F00AC1452A8A228597C0FFFFE78080702A
:10EFE0002A8D228597D0FFFFE78020892A892285F4
:10EFF00097D0FFFFE7804086930705F893F7F70F58
:10F000001307E007AA8B637BF706228597D0FFFFE3
:10F01000E78080842A8C228597D0FFFFE780C08319
:10F02000AA8C5285032B040097B0FFFFE780408530
:10F0300039E983574400231101008144F11793B744
:10F040001700A300F1000544034711008356210077
:10F05000938784005685DA8822885286CE8597F079
:10F06000FFFFE78020A7A167E90748003EC423020D
:10F07000810026C697D0FFFFE78000574101173374
:10F08000FFFF6700830313061100A28597E0FFFFCF
:10F09000E7802051AA8409E52311010009446DB7D6
:10F0A000930521006A8597F0FFFFE780A0F02A848E
:10F0B00041FD835521009356C90013164901854827
:10F0C0006688E2875E87858A5182268597000000E0
:10F0D000E78060BF2A848DBF1733FFFFE70263FA22
:10F0E00083C7950041112A8B93F7F707A384F50096
:10F0F0003285AE89328497C0FFFFE780007893178E
:10F100000501C1876352F00A2A8A228597C0FFFF52
:10F11000E780A076AA8A228597C0FFFFE780E07586
:10F120002A89228597C0FFFFE7800073930705F8BF
:10F1300093F7F70F1307E0072A8C6377F70622850A
:10F1400097C0FFFFE7804071AA8C228597C0FFFF20
:10F15000E78080702A8D5285832B040097A0FFFFE3
:10F16000E780007239E58357440085440144F11774
:10F1700093B71700A301F100034731009307840000
:10F180005A85DE882688D6865286CE8597F0FFFF80
:10F19000E78040948D4748003EC42302910022C678
:10F1A00097D0FFFFE780404441011733FFFF67001E
:10F1B000C3F0A2851306310097E0FFFFE780603EB1
:10F1C0002A84894455D99356C900131649018548A4
:10F1D0006A88E6876287858A5182D6859700000013
:10F1E000E78060AEAA8449BF1733FFFFE70243EA16
:10F1F0002A8981440144617A916A177BFF1F130BAE
:10F20000EBB897B0FFFFE780006863C7A4002285D2
:10F210001733FFFF670003EB83270900939914005E
:10F22000CE9703D507003307450142074183636446
:10F23000570305C103270B0019C785453E85974035
:10F240000000E78060E9832709000504CE9723903A
:10F25000070085047DB797000000E78060A2832740
:10F2600009000504CE972390070065D5814597F0E6
:10F27000FFFFE780C0BEF1BF1733FFFFE70243E1A6
:10F2800083C7950041112A8A93F7F707A384F500F5
:10F2900032852E89328497C0FFFFE780005E931786
:10F2A0000501C187635AF004AA89832A040097A044
:10F2B000FFFFE780E05C31E583574400854401446B
:10F2C000F11793B71700A301F10003483100D68767
:10F2D00052850147CE862686CA8597D0FFFFE780F4
:10F2E000806AA167F50748003EC42302910022C648
:10F2F00097D0FFFFE780402F41011733FFFF6700E2
:10F3000063DCA2851306310097E0FFFFE7806029E8
:10F310002A8489445DD99777FF1F938727A79C4349
:10F3200081CF044997B0FFFFE780E055AA85268585
:10F3300097400000E78040DA1305040197000000C1
:10F34000E780C0EA228597800000E780003381448F
:10F35000ADBF1733FFFFE702C3D283C7950041114A
:10F36000AA8A93F7F707A384F5003285AE89328421
:10F370002311010097C0FFFFE7802050931705017C
:10F38000C1876354F0062A8AC145228597C0FFFFD2
:10F39000E7804035AA8B5285032B040097A0FFFF1E
:10F3A000E780004E21E98357440085440144F1176A
:10F3B00093B71700A300F100034811000357210081
:10F3C000DA875685D2862686CE8597D0FFFFE780DE
:10F3D000805BA1679387270248003EC42302910007
:10F3E00022C697D0FFFFE780202041011733FFFF9F
:10F3F0006700A3CCA2851306110097E0FFFFE7800A
:10F40000401A2A8489444DD99777FF1F938707981C
:10F4100098433E8901CF044997B0FFFFE780A0469B
:10F42000AA85268597400000E78000CB13050401DC
:10F4300097000000E78080DB97B0FFFFE780A044E3
:10F4400095443DD9930521005E8597F0FFFFE78045
:10F4500060B6AA8435F11C48035721002285239009
:10F46000E70097800000E780402183270900A9D7A3
:10F470000355210097400000E780A0BD35BF17333A
:10F48000FFFFE70203C083C795004111AA8A93F7E3
:10F49000F707A384F5003285AE89328497C0FFFF59
:10F4A000E780A03D93170501C1876351F0062A8AC2
:10F4B000228597C0FFFFE780403C2A895285032BB5
:10F4C000040097A0FFFFE780A03B31E5835744008D
:10F4D00085440144F11793B71700A301F1000348D5
:10F4E0003100DA8756854A87D2862686CE8597D020
:10F4F000FFFFE7804049A167F90748003EC42302A7
:10F50000910022C697D0FFFFE780000E410117331C
:10F51000FFFF670083BAA2851306310097E0FFFF63
:10F52000E78020082A8489445DD99167CA97C20779
:10F530001167C1831307F7EF8544E362F7FA977702
:10F54000FF1F9387A7849843BE8B01CF044997B0D0
:10F55000FFFFE7804033AA85268597400000E780BB
:10F56000A0B71305040197000000E78020C897B0FA
:10F57000FFFFE780403195443DD11C4822858144FE
:10F580002390270197800000E780200F83A70B00BE
:10F59000B9D74A8597400000E780A0AB89B71733F9
:10F5A000FFFFE70283B02A844105B2849700000080
:10F5B000E780C0C311C5228597800000E780E00B7B
:10F5C00081460146A685228597800000E780C04ECF
:10F5D0001C4C89C7DC4799C3228582971733FFFFEC
:10F5E0006700E3AE9767FF1F9387475B9C43014526
:10F5F00099C31385070182809767FF1F9387075A76
:10F60000884382801733FFFFE70223AA9317C600BF
:10F61000DD8DC2054111C1812A8432C697C0FFFF2A
:10F62000E780E0173246228511829375F60F97C066
:10F63000FFFFE780C01441011733FFFF670023A9D4
:10F640001733FFFFE702C3A479713C083ED2B70726
:10F650000C003ED43C083ED683C79500AE842A8970
:10F6600093F7F707A384F500A16593853504481047
:10F6700097A0FFFFE780E02BC165FD150144176AE5
:10F68000FF1F130A2A72930A400EAE892E8B2EC6D4
:10F6900097B0FFFFE78020224205931704014181C4
:10F6A000C183B24563E9A702C167FD176387F5000F
:10F6B000481097C0FFFFE780800E50100147814639
:10F6C000A6854A8597A0FFFFE780004C4561173368
:10F6D000FFFF6700239F3307540383270A0BBA9762
:10F6E00003D6C701630A3601638A350148109700C3
:10F6F0000000E78060F1DA85050451BFB285EDBFF7
:10F700001733FFFFE702E39779717C083EC8B7071C
:10F7100011003ECA7C083ECC83C79500AA89328579
:10F7200093F7F707A384F5002E8997C0FFFFE780C2
:10F73000C01485676378F504A165AA848905080863
:10F7400097A0FFFFE780E01E268597400000E78036
:10F7500060ED133415000A04A285080897C0FFFF66
:10F76000E780E001A685080897C0FFFFE780200337
:10F7700025CC014781461008CA854E8597A0FFFF1A
:10F78000E780804045611733FFFF67000393B307AD
:10F7900054030327CA0ABA9703D70700631C9700CC
:10F7A00003D6270063806505080897000000E780FE
:10F7B000A0E5DE8505042EC697B0FFFFE780A01008
:10F7C0004205931704014181C183B245E3E1A7FCDF
:10F7D000C167FD17E38FF5F8080897C0FFFFE780C2
:10F7E00000FC41BFB285F9B7C165FD150144176A38
:10F7F000FF1F130A2A5B930A80022E8BAE8B65BF14
:10F800001733FFFFE702638A1841834717008346D7
:10F810000700A207D58FD207D1832390F500834735
:10F820002700034717008D45A207D98F9183231026
:10F83000F60097C0FFFFE780A0E91733FFFF6700DE
:10F8400003891733FFFFE702A384C16401441769EA
:10F85000FF1F1309295593098002FD1497B0FFFF7C
:10F86000E78060066347A40001451733FFFF670088
:10F870006385330534038327C90A3E958357050002
:10F88000E38597FE0504D9BF1733FFFFE7024380E6
:10F890002A8AAE89B284B68A97400000E78080D871
:10F8A00019E591473E851733FFFF6700A3812A8939
:10F8B0004E8597C00000E780E08E2A84638E0A049C
:10F8C0008D476DD103570500C547E31D47FD03472D
:10F8D000F9018546AD47E317D7FC8347450081CF43
:10F8E0004146A6855D0597F00000E780C09E8147F0
:10F8F00055D9AD4745BF130965012302E500CA8507
:10F90000268597100000E780606231C1A547E38B30
:10F910000AF82302040079B705C183570500E39272
:10F9200047F94146A685190597F00000E780A09A9F
:10F9300081472DD99947BDB74E8597000000E780D4
:10F9400080F02A84954739DD130955004DBF4146A3
:10F95000A68523104401231134011305190097F0E3
:10F960000000E780A099228597800000E780A0EA48
:10F9700081470DBF1723FFFFE702237379717C00D6
:10F980003ECCB7070A003ECE7C003ED083C7950030
:10F99000B2842E8493F7F707A384F5001306A10021
:10F9A0002A892C00268597000000E780A0E5A16544
:10F9B00028088D0597A0FFFFE780A0F790408355AA
:10F9C000A10003558100854697000000E78000EC08
:10F9D000AA84AA85280897C0FFFFE78040DA03566B
:10F9E000A10083558100280897000000E780C0C16E
:10F9F000300801478146A2854A8597A0FFFFE7802E
:10FA0000A018854748103ED42302910202D697D011
:10FA1000FFFFE78060BD45611723FFFF6700236B91
:10FA20001723FFFFE702636879717C003ECCB707BC
:10FA30000A003ECE7C003ED083C79500B2842E845F
:10FA400093F7F707A384F5001306A1002A892C0079
:10FA5000268597000000E780E0DAA16528088D057B
:10FA600097A0FFFFE780E0EC90408355A10003558D
:10FA70008100814697000000E78040E1AA84AA85C2
:10FA8000280897C0FFFFE78080CF0356A100835569
:10FA90008100280897000000E78000B73008014780
:10FAA0008146A2854A8597A0FFFFE780E00D4810B8
:10FAB0002302910202D402D697D0FFFFE780C0B2A2
:10FAC00045611723FFFF670083601723FFFFE702ED
:10FAD000C35D97000000E78060DB1723FFFF67002E
:10FAE000035F9767FF1F9387A70B884382801723C5
:10FAF000FFFFE702835B835725004111AE842A8410
:10FB00002307B10017F5FFFF130525466C002316E8
:10FB1000F10097A0FFFFE780204991C422859780DC
:10FB20000000E780E0D6FD572310F4001306200202
:10FB30008145130554009720FFFFE780005A4101DB
:10FB40001723FFFF6700A3581723FFFFE702435463
:10FB500079717C003ECCB7070A003ECE7C003ED0D7
:10FB600083C79500AA89AE8493F7F7073285A384EB
:10FB7000F5001306A1002C0097000000E78080C864
:10FB800003558100114497400000E780A0A915C5E6
:10FB90000355A100014497B00000E780A06011CD9B
:10FBA000035705008357810045446318F7008545D6
:10FBB00097000000E780E0F30144216993053900D4
:10FBC000280897A0FFFFE780C0D6A285280897C025
:10FBD000FFFFE780C0BA0356A100835581002808C3
:10FBE00097000000E78040A2300801478146A685C3
:10FBF0004E8597A0FFFFE78020F948104AD42302E2
:10FC0000810202D697D0FFFFE780009E456117234F
:10FC1000FFFF6700234B1723FFFFE7026347976748
:10FC2000FF1F9387A7F72A8488432E8915C503579A
:10FC300045038357C4016311F702232605022318E5
:10FC40000502410597D00000E780209C630609006B
:10FC500097800000E78060DB81449769FF1F9389EC
:10FC60006914130A800297B0FFFFE780C0C563C420
:10FC7000A4049767FF1F938727FB9C4399C70355ED
:10FC8000C40197200000E780C0BD630709002285FA
:10FC900097800000E780C0A01306400E81452285B2
:10FCA0009720FFFFE7806043FD57231EF4001723D2
:10FCB000FFFF670023413385440383A7C90A3E95AC
:10FCC000035705008357C4016317F700CA859700DF
:10FCD0000000E78000E2850479B71723FFFFE70201
:10FCE000233B83C795004111AA8993F7F707A384A3
:10FCF000F5003285AE8497C0FFFFE78000B88567C6
:10FD00006378F5042A8997400000E780A0910144B8
:10FD100001CD83D7040031446388270185459700CE
:10FD20000000E78080EF01444E85A2864A86A685C2
:10FD300097D0FFFFE780A09CA16793871704480036
:10FD40003EC42302810002C697D0FFFFE780C0892E
:10FD500041011723FFFF6700E3361723FFFFE70288
:10FD600023339767FF1F938767E3804329C40145C7
:10FD700097C00000E780002181470148C1641CDC76
:10FD8000232E0403232004041769FF1F130989018C
:10FD900001449309400EFD1497B0FFFFE780A0B126
:10FDA000634FA400814517F5FFFF1305857F97A0DA
:10FDB000FFFFE780601F1723FFFF6700A3303305B5
:10FDC00034038327090B3E958357C501638797004A
:10FDD000854597000000E78040E4050475BF935710
:10FDE000050113D78700A380F50093170501C18390
:10FDF000A1832380E5002381F500A381A5008280F3
:10FE00001723FFFFE702632A2300050083C71500BD
:10FE1000A300F50083C725002301F50083C7350043
:10FE2000A301F50083C745002302F50083C75500F1
:10FE3000A302F50083C7650093059500A3030500A1
:10FE40002303F50023040500328597000000E780B6
:10FE500040F91723FFFF670083271723FFFFE702FF
:10FE600023234111E9540DCD85CD93F9C5FF2E848F
:10FE70002A89AA84338AA900B7EA040063189A027F
:10FE80000D88854411CCB7E704009C5F82972AC691
:10FE900022866C003305390197E00000E7800046B8
:10FEA000268541011723FFFF6700C32183A78A032B
:10FEB0009104829793170501C183A183A38EF4FE59
:10FEC00093570501238FF4FEA183238EA4FEA38FF5
:10FED000F4FE6DB763E6D5021723FFFFE702E31CCC
:10FEE000B28741113686BE8536C697E00000E780AE
:10FEF000E040B246410136851723FFFF6700231D0E
:10FF0000814636858280838705001387F5003D058D
:10FF1000FD8793F77708834607007D158606B58F22
:10FF2000A300F5006307B7007D17834717009D8383
:10FF3000DDB782801723FFFFE7022317B7E704002E
:10FF400083A7070932872A863A85829713351500D9
:10FF50001723FFFF6700A31715C181478DC1172322
:10FF6000FFFFE7028314414697E00000E780003975
:10FF700085473E851723FFFF6700631581473E8550
:10FF800082801DCD1723FFFFE702231241468145E2
:10FF90002A849720FFFFE7804014414681451305DE
:10FFA00004039720FFFFE78040130147C167232226
:10FFB000040438C87CC805451723FFFF67002311D8
:10FFC0000145828081473DCDB5CD1723FFFFE70274
:10FFD000C30DB2842E891306800581452A8497209B
:10FFE000FFFFE780800FCA8524C4268597000000A4
:10FFF000E780C0F64146814522859720FFFFE780D4
:020000040001F9
:10000000C00D3044A285228597000000E780C0F231
:1000100093040401A285268597000000E780E0EEA6
:10002000A6851305040297000000E78000EE2285F4
:1000300097000000E78020F585473E851723FFFFE6
:100040006700E3083E8582801723FFFFE702430431
:100050004111E9540DCD85CD93F9C5FF2E842A8930
:10006000AA84338AA900B7EA0400639844030D8880
:10007000814411CCB7E704009C5F82972AC6228690
:100080006C003305390197E00000E78020272685C2
:1000900041011723FFFF6700E30283A78A0391044E
:1000A000829793170501C183A183A38EF4FE935712
:1000B0000501238FF4FEA183238EA4FEA38FF4FEFB
:1000C0006DB765CD1723FFFFE70283FCB28411E60D
:1000D00005451723FFFF6700E3FE2A842E890145AB
:1000E000EDD93C487848B3E6E700E5D69386F7FFBC
:1000F000B3B7F6007D17032A4404BA9734C87CC806
:1001000063050A06C14913050A03B38949412295CB
:10011000637D3601B2862E86A68597000000E780B3
:10012000A0DB7C40BE9464C065B7CE862E86CE85AB
:1001300097000000E78040DAC114D2944E99232240
:100140000404A2879306040103C7070003C607033C
:100150008507318FA38FE7FEE398F6FE3044A28532
:10016000228597000000E78020DD2699C1493306EB
:10017000994063EC9900A9DCA686A68513050403C3
:1001800097000000E78040D579BF8147B306F400AF
:100190003307F6000347070083C5060085072D8F48
:1001A0002380E600E39437FF3044A2852285970040
:1001B0000000E78060D8C1145DBF014582800DC199
:1001C0001723FFFFE70263EE1306800581459720A2
:1001D000FFFFE78080F005451723FFFF670023EF4F
:1001E00001458280814749C5C1C51723FFFFE7024A
:1001F000C3EBFC4141462E84AA846399C70413864D
:100200000501A2878146C14503C7070003C507034F
:100210008507298F3305D600034505008506298FFC
:10022000A38FE7FEE392B6FE3044A28526859700B1
:100230000000E78060D0228597000000E78060F82A
:1002400085473E851723FFFF670063E81385070393
:100250001D8E814522959720FFFFE78000E87C40B6
:10026000130700F813060402A2972388E70251BF80
:100270003E8582801723FFFFE70223E36D712E8402
:10028000B284AA8590102800368997000000E78084
:10029000A0D309EDD55725A050400C402800970069
:1002A0000000E78040E27DD5FD142104F5F42C0028
:1002B0004A8597000000E78020F3814761DD3E8595
:1002C00051611723FFFF670083E01723FFFFE70259
:1002D000C3DD41112EC432C62C0005469700000034
:1002E000E78080F941011723FFFF670043DE1723F2
:1002F000FFFFE70283DB01112A842EC602C802CA6F
:1003000002CC02CE97E00000E780402BB2462A865E
:10031000A285080897000000E78060FB1375F50FC1
:1003200005611723FFFF670083DA1723FFFFE7024A
:10033000C3D77971B2872A8421462308B1001305F7
:100340001101BE853AC436C697E00000E78000FB85
:10035000B24693059101368597000000E78060A8BA
:100360002285141035460C0897000000E78020F61F
:100370002A84224701E921460C103A8597E00000C3
:10038000E780C0F7228545611723FFFF670023D46C
:100390001723FFFFE70263D17171AE84AA850A8536
:1003A000328497000000E78060BB11C90A86A685E9
:1003B000228597000000E78020B8814711E1C547FA
:1003C0003E854D611723FFFF670063D01723FFFFB2
:1003D000E702A3CA1D712A8AB289BE8435468547C1
:1003E000130511012E8CB68A3A8BC28C468D2308D8
:1003F000F10097E00000E78060F010100C085285D3
:10040000231F010097000000E780C0F82A843DED1B
:10041000A1476313FD089307900591E0E547354632
:10042000E2851305110113990A012308F1001359FC
:10043000090197E00000E78060EC1357890093976B
:100440008A00D98F90080C085285231FF10097006D
:100450000000E78020F42A8415E9A1E49387FA00DC
:1004600091831379F9003EC6631309004149668BF5
:100470008144C14B854DB247639F970C6A868C00BF
:1004800033855C0197E00000E78040E72285256125
:100490001723FFFF670023C293079004C9F0A54705
:1004A000BDBF834701050947C14B2308F1008347BE
:1004B0001105A58FA308F10093872400814463E10F
:1004C000FB04014714083386E6008C08B386E40079
:1004D000BA95DA9683C6060083C505000507AD8E7A
:1004E0002300D600E390E7FE4147639CE7049008B1
:1004F0000C08528597000000E780C0E925D181A053
:10050000B3069B00BA871008B305F60090083E9624
:1005100003C506000346060085078506298E23804D
:10052000C500E39277FF998F90080C085285BE941E
:1005300097000000E78000E68947014749D12A84F7
:10054000B1B790083E96034606001408BE96238075
:10055000C600850759BFB247850463879714814752
:100560001808B306F70098083E973386F90003474A
:100570000700034606008507318F2380E600E391DC
:1005800077FF90080C08528597000000E78080E014
:100590005DF53546E285130511012308B10197E0A9
:1005A0000000E780A0D5139704014183939784004E
:1005B0002183D98F10180C085285231FF100970052
:1005C0000000E78020DD25FD814710183387F90002
:1005D0003E960347070003460600B306FB00850767
:1005E000318F2380E600E39277FF65A81808B306F1
:1005F000F70098083E973386F90003470700034643
:1006000006008507318F2380E600E3E127FFCA87D4
:10061000639E770990080C08528597000000E780D8
:1006200060D711FD81479800B306F70090081810B5
:100630003E973E9603470700034606008507318F25
:100640002380E600E39177FF3546E285130511012B
:100650002308B10197E00000E78040CA1397040126
:100660004183939784002183D98F10180C085285F9
:10067000231FF10097000000E780C0D1E31105ECD3
:10068000814710183387F9003E9603470700034659
:100690000600B306FB008507318F2380E600E3E206
:1006A00027FFC109410BC1BB814785B79408BE969E
:1006B00083C6060018083E972300D700850789BF28
:1006C000638006321723FFFFE702239B59712A84B8
:1006D000BE89B28B85473546130511022E8B468C99
:1006E0004289BA8A368A2300F10297E00000E78047
:1006F000E0C010180C10228523170102970000009B
:10070000E78040C963180512A147631FFC069307E1
:10071000900563930900E5473546DA851305110214
:1007200093140A012300F102C18097E00000E780E2
:10073000E0BC93178A0013D78400D98F90080C105F
:1007400022852317F10297000000E780A0C47DE115
:10075000639209049307FA00BD88918391E0C14434
:10076000C207C183DE8C814A3EC6414DB24763E277
:10077000FA0E6286B3854B01881097E00000E7808F
:1007800080B54DC93D557DA093079004E39609F8C7
:10079000A54759B7834701050947C14C2300F1021A
:1007A00083471105B3C7F900A300F102938729001D
:1007B000814963E1FC04814618103306D7008C0898
:1007C0003387D900B69556970347070083C50500C0
:1007D00085062D8F2300E600E390D7FE4147639006
:1007E000E70690080C10228597000000E78080BA89
:1007F00035D189A0B3863A01BA871010B305F60047
:1008000090083E9603C50600034606008507850648
:10081000298E2380C500E39297FF3387EC40900830
:100820000C102285BA9997000000E780A0B689478E
:10083000014741D165611723FFFF6700C387900817
:100840003E96034606001410BE962380C600850718
:1008500079B7B247850A93990A01939D8A0093D983
:1008600009016391570F85473546DA851305110253
:100870002300F10293D9890097E00000E78000A8E7
:10088000B3ED3D0190000C1022852317B1039700B2
:100890000000E78020B059FD8147A68963EA9706EA
:1008A00026860C084A8597E00000E78020A581474E
:1008B0001810B306F700100898083E973E960347B5
:1008C0000700034606008507318F2380E600E3E139
:1008D00097FE639FA90590080C10228597000000E1
:1008E000E78040AB21F981479810B306F7009008E4
:1008F00018183E973E9603470700034606008507F3
:10090000318F2380E600E391A7FF4109C10CB9BDF7
:1009100018089000B306F7003E963387FC000347A3
:100920000700034606008507318F2380E600B5B730
:1009300098084E97034707001C10CE972380E700C6
:10094000850941BF85473546DA8513051102230025
:10095000F10293D9890097E00000E780209AB3ED77
:100960003D0190000C1022852317B1039700000071
:10097000E78040A2E31005EC814718089000B30619
:10098000F7003E963387FC00034707000346060046
:100990008507318F2380E600E391A7FF41460C08CD
:1009A0004A8597E00000E780609581471810B306FC
:1009B000F700100898083E973E9603470700034645
:1009C00006008507318F2380E600E391A7FF90089A
:1009D0000C10228597000000E780C09B1DD599BDB3
:1009E0007D5582801713FFFFE702236C01112A84D3
:1009F0002E8593055100328902C002C202C402C68C
:100A00009304740097F0FFFFE780A03D1D46A68584
:100A10001305910097E00000E780408E10088A855A
:100A20004A8597000000E780E09619ED93071400CF
:100A3000180883C607000346070085070507B18E1F
:100A4000A38FD7FEE397F4FE05611713FFFF67003E
:100A500003681713FFFFE702A3632E848C41411143
:100A6000AA89838715003289914463D30700A14482
:100A70009757FF1F9387C7699C43A1C7C1CA8D477A
:100A80002310F10083C725004A852301F10083C7A5
:100A90003500A301F10083C745002302F10083C79D
:100AA0005500A302F10083C7650093059100A303DD
:100AB00001002303F1002304010097F0FFFFE7800A
:100AC00040320C404A860A8597F0FFFFE78080336A
:100AD0000328040083564400A6881D088147014767
:100AE000E51642868A854E8597000000E780408E95
:100AF0002A8919E5A685228597B0FFFFE780E0C126
:100B00004A8541011713FFFF6700C35B4A860A85C8
:100B100097F0FFFFE780002F6DB71713FFFFE70285
:100B200023572E848C414111AA898387150032896D
:100B3000914463D30700A1449757FF1F9387475DF4
:100B40009C43A1C7C1C68D472310F10083C7250070
:100B50004A852301F10083C73500A301F10083C753
:100B600045002302F10083C75500A302F10083C7AB
:100B7000650093059100A30301002303F100230402
:100B8000010097F0FFFFE780C0250C404A860A85E8
:100B900097F0FFFFE78000278356440003280400F6
:100BA0008A85858EC2061D08C1822312D400A688BC
:100BB00081470147E51642864E8597000000E78091
:100BC00060B041011713FFFF6700C34F4A860A85D3
:100BD00097F0FFFFE78000234DBF1713FFFFE702E9
:100BE000C34CB335B000011185052A891315F601F0
:100BF000336515012308B1009305110136843AC607
:100C000032C03EC442C297F0FFFFE780801DA2477A
:100C10001248425593D68700230BF10093059101AA
:100C200093578800A30AD100A30BF100230C010104
:100C300097F0FFFFE780E01A3247024603280400DE
:100C4000B337E000835644009207914411C2A14497
:100C50004A85A68842860C0897F0FFFFE780407718
:100C60002A8919E5A685228597B0FFFFE780E0AACB
:100C70004A8505611713FFFF670063451713FFFFE0
:100C8000E702034101113EC68647B335B000850532
:100C9000AA891315F6015D8D2308B1009305110192
:100CA00036843A89B28442C446C297F0FFFFE78097
:100CB000401322489248164593578800A30AF10032
:100CC0009305910193D78800230B0101A30BF10039
:100CD000230C110197F0FFFFE780A010324710406E
:100CE00083564400B337E000920703280900914877
:100CF00091C0A1480C084E8597000000E780809CB9
:100D0000AA8401E9835544004A8597B0FFFFE78034
:100D1000C0A0268505611713FFFF6700A33AAA95B7
:100D20009307F00F171701001307C7986317B50053
:100D300013C5F7FF1375F50F828005058346F5FF90
:100D4000B58FBA9783C70700D5B70357450014413D
:100D50009307F00F171601001306C6953697420742
:100D60004183139506014181631BE500AD8FB29766
:100D700003C50700130515F313351500828085069A
:100D800003C5F6FFA98FB29783C70700D9BF171312
:100D9000FFFFE7028331B28736842E86BA86AA85A2
:100DA0003E85BA8497F0FFFFE7806052634F0500ED
:100DB000228597E00000E78060802A86A686A285CB
:100DC000268597F0FFFFE78080501713FFFF67002D
:100DD00003301713FFFFE702A32B5D712A8BAE8A46
:100DE000171501001305858A2C00B284368ABA894A
:100DF0003E8997F0FFFFE780C04F2A845DE1341001
:100E00004146DA85280097F0FFFFE780404C2A84AE
:100E100049E98547A303F100A6C29307710024089E
:100E2000BEC4A68685470D462C18281002DC02DEBB
:100E3000D6C0BEC697F0FFFFE78000442A8435E1A4
:100E400083477102A6860D4693F7F7072300FA0041
:100E5000C1473EDE2C188947281026DCA303F10089
:100E600097F0FFFFE78040412A8405ED4146A685C3
:100E70004E8597D00000E78060488D47A6860D46D6
:100E80002C182810A303F10097F0FFFFE780C03E65
:100E90002A8401E94146A6854A8597D00000E7806B
:100EA000E045228561611713FFFF6700A321171337
:100EB000FFFFE702831F97F70000938727EF984310
:100EC00083C7470079712A89AE841705010013058D
:100ED000657C0C083AC42306F10097F0FFFFE78019
:100EE00040412A8405ED14104146CA85080897F050
:100EF000FFFFE780C03D2A8415E1140815462C0049
:100F0000081097F0FFFFE780803C2A8401E9214622
:100F10002C08268597D00000E780403E2285456159
:100F20001713FFFF6700A31A1713FFFFE702E3176A
:100F300097F70000938787E79C477971AA842E84EE
:100F400017050100130585750C083EC697F0FFFFD5
:100F5000E780203A0DE914104146A685080897F06D
:100F6000FFFFE780C03605E1140811466C00081049
:100F700097F0FFFFE780A03519E58347F10193F76C
:100F8000F7032300F40045611713FFFF67002314E4
:100F90001713FFFFE70263113688A1488147014715
:100FA000E54697F0FFFFE780A0421713FFFF6700B9
:100FB00003121713FFFFE702430F3688A14881474A
:100FC0000147E54697F0FFFFE780C06F1713FFFF6B
:100FD0006700E30F1713FFFFE702230D01112A84B7
:100FE0002E850C0832C697F0FFFFE780803009EDB0
:100FF0003247970601009386E6681008C1452285AE
:1010000097000000E780E0D805611713FFFF670035
:10101000030C1713FFFFE70243094111C1472EC01C
:1010200032C48A8509463EC23EC697F0FFFFE7807C
:10103000A02441011713FFFF670063091713FFFF87
:10104000E702A3064111AE8613061009AA850A8598
:1010500002C002C202C402C697F0FFFFE780202749
:1010600041011713FFFF670083061713FFFFE70215
:10107000C3033287970601009386C6622E869305C6
:10108000000297000000E780C0D01713FFFF670041
:1010900003041713FFFFE70243017971C1472ACC0C
:1010A0002ED032D42C080D4628003ECE3ED23ED65D
:1010B00002C402C602C802CA97F0FFFFE780C01B45
:1010C00045611713FFFF670083001713FFFFE70257
:1010D000C3FD0111AA842E84170501001305055DC7
:1010E0008A8597F0FFFFE780C02015E51408414688
:1010F000A6850A8597F0FFFFE780601D09ED83470D
:10110000E1010347F101A207D98FCA07C9836177BB
:10111000D98F2310F40005611713FFFF670023FB2D
:1011200015CD1713FFFFE70243F89757FF1F93876B
:10113000A7AB90439755FF1F938545AB1755FF1FEE
:10114000130585A697D00000E78000C51755FF1F3F
:10115000130585A51713FFFF670063F71755FF1FDA
:10116000130585A482808DCD1713FFFFE702E3F3FB
:101170009757FF1F938747A7944301112E840A8630
:101180009755FF1F938585A697D00000E78040C63E
:101190000A850294014505611713FFFF670023F3D9
:1011A0007D5582801713FFFFE70223F097D00000E0
:1011B000E78080D19757FF1F23A8A7A217F5FFFF4D
:1011C0001305E5C997B00000E780C0741713FFFF4F
:1011D0006700E3EF1757FF1F130747A39317150087
:1011E00008433E95FD572310F50082801713FFFF3B
:1011F000E702A3EB2A84084009E51713FFFF670005
:1012000003ED1C4158401CC06313E5005CC08347DC
:10121000550023200500F99BA302F50097A0FFFFCE
:10122000E780207CC9BF1713FFFFE70263E69757EB
:10123000FF1F9387A79F98432A8411CB83473500CC
:1012400093F7070289C703550500894502971305DF
:10125000440197B00000E780403B835504000355EC
:10126000E40097300000E780A00C485819C597A00B
:10127000FFFFE7800077232A040213058403970009
:101280000000E780E0F68144B1499790FFFFE780D6
:10129000C06D63CBA402834734002320040493F77A
:1012A00027FCA301F40000489790FFFFE780E06C63
:1012B00013161500814522859710FFFFE780E0E1B6
:1012C0001713FFFF670003E0B38734030329040308
:1012D00085043E994A8597000000E78060F1230469
:1012E000090065B78347350093F7070299E3014585
:1012F00082808357E500E39CB7FEC167FD17631644
:10130000F60005458280054599A81713FFFFE702FF
:10131000C3D993170601C187B2842A84014963594E
:10132000F002835705009DCB01456367F600034536
:1013300084003E953325A6001375F50F0DA01C48BB
:1013400013171900BA9783D70700E38E97FA050998
:101350009790FFFFE7806062E343A9FE0145171302
:10136000FFFF6700C3D61713FFFFE70263D2AE8902
:10137000AA849790FFFFE78000562A8497D0FFFF4A
:10138000E780A02EAA860147130684019705000076
:10139000938585E41755FF1F130585879790FFFFF9
:1013A000E780801C2A8925C98C441304C500228546
:1013B0009E0593F5050897A0FFFFE780403CCC40D1
:1013C00083877400E18163DD070493E505082285C6
:1013D00097A0FFFFE780A03A0D4693854400228541
:1013E00097A0FFFFE780C03683D50400228597A031
:1013F000FFFFE780E03D83D52400228597A0FFFF13
:10140000E780003D03D6490083A50900228597A007
:10141000FFFFE780E0334A851713FFFF670083CAA9
:1014200093F5F5076DB71713FFFFE70203C8011126
:101430002A84328532C697A0FFFFE780E027978095
:10144000FFFFE7806034835704001757FF1F13071F
:1014500067953246231BF100930700F8A30DF100B6
:101460001C471843231AA1008983858BB307F740D3
:10147000B28548083ECE231C0100230D01009700D1
:101480000000E78080EE05611713FFFF670023C4AB
:101490001713FFFFE702C3BF004101453DC493049A
:1014A000C40026853289AE8997A0FFFFE780C0245B
:1014B00095452A8A2685035B040197A0FFFFE780F4
:1014C0002021268597A0FFFFE780603E8D45AA8AF0
:1014D000268597A0FFFFE780A01F268597A0FFFF26
:1014E000E780E03C5C48420A135A0A01D2975CC488
:1014F00023186401814763983A0146054D813306FC
:1015000025419337160013F5F70F1713FFFF6700F8
:1015100063BB1713FFFFE702C3B689692A8BAE8B43
:10152000328AB68A81440144314CFD199790FFFFFD
:10153000E780A04363CDA4009790FFFFE780E045DC
:10154000018D33B5AA001713FFFF670003B7338976
:10155000840383270B003E9963170A0083478900A1
:1015600085043E94E1B703560A00DE854A8533F6CA
:10157000C90097000000E780E0F16DD10545E1B7B3
:101580001713FFFFE70263B201112A847C000355A1
:10159000E5003ECAB70707003ECC7C003ECE972050
:1015A0000000E78020082A898545480897A0FFFFAA
:1015B000E78020399945480897A0FFFFE780E015AC
:1015C000AA844A8597200000E780A0082380A40011
:1015D0009747FF1F9387077D9C434166130606F0DC
:1015E0009396870113D78701558F93D68700F18E85
:1015F000558FA207B706FF00F58FD98F11462C0033
:10160000138514003EC497D00000E78020CF500817
:10161000A38204008945228597000000E780E0E06E
:1016200019C9AA851305840397A0FFFFE780E0315D
:101630003C4085073CC005611713FFFF670023A9E5
:101640001713FFFFE70263A69790FFFFE780E034E0
:101650002A8405049790FFFFE78020333305A40216
:10166000F14791453305F50297200000E78020BA45
:1016700011E565551713FFFF670063A59747FF1F27
:1016800023AEA7589790FFFFE78020312A840504F6
:101690009790FFFFE780602F3305A4028945060578
:1016A00097200000E780A0B669D59747FF1F23AFBA
:1016B000A7549790FFFFE780402E2A840504979057
:1016C000FFFFE780802C3304A4029747FF1F23917C
:1016D00087549790FFFFE780402C2A849790FFFF64
:1016E000E780A02A930714003385A7029747FF1FBE
:1016F0002391A75297070100938707BF1747FF1F42
:10170000232CF7500145BDB71713FFFFE70243989D
:10171000AA842E8901449749FF1F9389A968130A57
:1017200080069790FFFFE78040266347A4000145AD
:101730001713FFFF670003993305440383A70902CA
:101740004A86A6853E9597000000E780E0B919E13A
:101750000504C1BF0545E9BF1713FFFFE702639208
:10176000AA8A2E8BB28B368C3A8A814401448149F5
:10177000974CFF1F938C0C63130D80069790FFFF0F
:10178000E780A02063C9A40011E085494E851713A6
:10179000FFFF670083923389A40383A70C025E8650
:1017A000D6853E994A8597000000E780E0B31DC1C9
:1017B0009790FFFFE780601E0544636D4501D28668
:1017C0006286DA851305090397000000E780A0D43C
:1017D00011C1854985045DB71713FFFFE702438BED
:1017E000C16441112A8901449749FF1F9389895B8C
:1017F000130A8006FD1436C632C42EC29790FFFF2E
:10180000E780A01892452246B2466348A4000145ED
:1018100041011713FFFF6700E38A3305440383A7E1
:1018200009023E9509C683473500C18B9DC791C605
:101830008347350093F707028DC3630699008357EA
:10184000E500639C27010357050001CB63E7E50032
:1018500083478500BA97E3CDF5FA050469BF1713EE
:10186000FFFFE702E382C1642A8901449749FF1F11
:1018700093894953130A8006FD149790FFFFE78070
:10188000C0106346A4001713FFFF6700A38333054E
:10189000440383A709023E958357E500638A9700B6
:1018A000630499006396270197000000E780E097A2
:1018B0000504E1B71703FFFFE702237C89692A8A41
:1018C000AE8A328BB68B8144174CFF1F130C8C4DA4
:1018D000930C8006314DFD199790FFFFE780E00AD9
:1018E00063C6A4001703FFFF6700E37C33899403FA
:1018F00083270C028355CA015A863E994A85970070
:101900000000E780609E31C1814D15A03384AD0396
:101910008327090303D60B00D68533F6C9003E940E
:10192000228597000000E780E0B609E9850D9790D1
:10193000FFFFE7808003E3CBADFC01A82285970081
:101940000000E780E08A23040400850471B71703D0
:10195000FFFFE70203734169AA8A014A174BFF1F81
:10196000130B4B447D19C14B054C9790FFFFE7804B
:10197000C0016346AA001703FFFF670003749309C1
:101980008006B3073A0383290B02BE9983D7E90087
:10199000638E270163842A01639A570103A4890394
:1019A00001E84E8597000000E780C0BD050A75BFBD
:1019B00083570401639977099304C400268597A08F
:1019C000FFFFE78060D385452A8D2685835C04016F
:1019D00097A0FFFFE780C0CF268597A0FFFFE78095
:1019E000A0E762056185635905048D45268597A0AA
:1019F000FFFFE780E0CD8945268597A0FFFFE780C0
:101A000020CD8945268597A0FFFFE78060CC8545DE
:101A1000268597A0FFFFE780E0CC834705000947B4
:101A200093F7F707639AE7009945268597A0FFFF8C
:101A3000E78040CBA30285014848337D2D01231860
:101A400094016A9548C40040A1BF1703FFFFE70255
:101A5000C36537E404008327041D82979747FF1F5F
:101A600083C747211725FF1F130585A8A300F5008D
:101A70008327441C82978327841C81461306F00F1A
:101A80008145014582971703FFFF670043641747AD
:101A9000FF1F1307270E18439745FF1F83C5851D9A
:101AA0009747FF1F9387871B834687030346970348
:101AB0006397D5009747FF1F238EC71A828083C57F
:101AC00087010347A7036317B6009747FF1F2383C8
:101AD000E71A828003C687016317C7009747FF1F75
:101AE000238AD718828083C687011307500263199F
:101AF000D700930760021747FF1F230DF716828058
:101B000083C68701130660026315D600930770022F
:101B1000DDB783C7870155BF9747FF1F938707141A
:101B2000D44B0947638DE6081703FFFFE702E3572D
:101B30001749FF1F1309C90F3E8483470900918B82
:101B40009DCFB7E4040083A7041D829783A7441C9C
:101B50001745FF1F1305450E829783A7841C8146F6
:101B60001746FF1F0346460F81450145829721C551
:101B700083470900ED9B1747FF1F230BF70A834795
:101B8000040093F7F70F85CB91471747FF1F2321D9
:101B9000F70E97000000E78080EB97000000E780D9
:101BA00040EFB7E70400BC4F414691451745FF1F82
:101BB0000345450B82971703FFFF6700435182805F
:101BC0001703FFFFE702634E8D4741116306F504DB
:101BD000C5476308F50285476310F5029747FF1F65
:101BE000238CA708B7E70400BC4B930500101745EA
:101BF000FF1F03452507829741011703FFFF670079
:101C0000034D85471747FF1F2308F706B7E7040072
:101C1000BC4B93050020E1BF9747FF1F9387070444
:101C2000D44B1147638DE600B7E7040083A7071D77
:101C30008297B7E70400BC4B930500044DBF0549EC
:101C40001747FF1F2326270383C7070032C62E84AA
:101C500093F7F70FD5D3B7E4040083A7041D7D14D1
:101C60001374F40F8297E37689FCB245994703C653
:101C70001500E3F0C7FCFC4409061745FF1F1305D8
:101C8000E5FF8297BC48930500081745FF1F0345F1
:101C900065FD829779BF1703FFFFE70203411747EE
:101CA000FF1F1307A7FB4047184B1C409746FF1F19
:101CB00023ACF6FA6316E4001747FF1F2328F7FA50
:101CC000130584FE9790FFFFE78000AA035564FF89
:101CD0009780FFFFE780807297A0FFFFE78060D0CA
:101CE0001703FFFF6700A33E1703FFFFE702E33B75
:101CF0009747FF1F938787F6D84BDC4789C7970024
:101D00000000E78080F985471747FF1F2322F7F679
:101D10009747FF1F938707E69C43930500021745EB
:101D2000FF1F034525F483C787031747FF1F2303BE
:101D3000F7F4B7E70400BC4B82971703FFFF670077
:101D400003399747FF1F23ADA7F082801703FFFFDA
:101D5000E702033437E404007C4CA1451745FF1F1C
:101D6000034545F082977C48A1451745FF1F034571
:101D700065EF9744FF1F938464EE8297DC4489EB00
:101D800097000000E78080D91703FFFF67008333C7
:101D900003D567FF9780FFFFE7804066AA896DD172
:101DA000D84891476310F7027C4C91451745FF1FB7
:101DB000034545EB82977C4891451745FF1F034536
:101DC00065EA829703A9490103D409018947B7E964
:101DD00004001747FF1F232DF7E883A7091D2104DF
:101DE0004204829783C784011715FF1F13054570AE
:101DF00061191717FF1FA30DF76E83A7491C4180B8
:101E000082979747FF1F238907E683A7C91C81464E
:101E100009469375F40F4A85829711E99747FF1F8A
:101E200083C7C7F589C79710FF1FE78040D9B7E779
:101E30000400BC4F2146A1451745FF1F034585E21D
:101E4000829799B71703FFFFE702232693F7052030
:101E500001112E8481CF97000000E78020E913450F
:101E6000042005611703FFFF6700632693F7051041
:101E7000A9CF9744FF1F938464DEDC4897000000DD
:101E8000E78020C11747FF1F1307C7CE184383C73A
:101E90008401034787036318F700DC4489C7970070
:101EA0000000E78080DF85471747FF1F2322F7DC0C
:101EB000B7E70400BC4B930500021745FF1F03451D
:101EC00065DA82971345041069BF93F70508BDC70B
:101ED0009747FF1F83C797DAE91719469745FF1FF2
:101EE0009385E5D91305D10093F4F70F1749FF1F28
:101EF0000349C9D897C00000E78040409397040188
:101F0000C1831747FF1F1307E7D7231DF100231CC9
:101F1000F1009747FF1F938767D43ACE3ACAD84358
:101F20002306010009CBDC439315890154080D46B3
:101F3000E185680082971345040825B793F72500CB
:101F4000A5C39747FF1F938767D1D84B894763067F
:101F5000F7029747FF1F83C7A7CD13F7270011EF9D
:101F6000918B99CFB7E70400BC4F1306000A89454F
:101F70001745FF1F034505CF829713452400D5B5AC
:101F80009747FF1F938707BF9C4383C78703174764
:101F9000FF1F2301F7CE97000000E78060DBF1BF51
:101FA00093F7050281CB97000000E78060DA1345C4
:101FB000040245BD93F7850081CB97000000E780C0
:101FC000E0D21345840071BD93F7150081CB9700D3
:101FD0000000E780A0B41345140061B593F74500F5
:101FE00081CB97000000E78060B31345440095BDA6
:101FF00093F7050495C39747FF1F83C727C691CB67
:1020000097000000E780A0A491471747FF1F2321F6
:10201000F7C613450404B1B593F705010145E38202
:1020200007E49747FF1F938767C3D84B9147631017
:10203000F7049747FF1F9387A7BF9C4313D7270039
:102040008583D98F858B91E7B7E7040083A7071DA8
:102050008297B7E70400FC4F91451745FF1F0345E2
:1020600065C0829785471747FF1F2323F7C0134595
:102070000401C5BB9747FF1F2382A7D082801703A7
:10208000FFFFE70283029747FF1F23AF07BC974775
:10209000FF1F23AD07BC85471744FF1F130484AD02
:1020A0001747FF1F2326F7BC1C4083C7870317472A
:1020B000FF1F2301F7BC9790FFFFE780409329C5DE
:1020C0009717FF1F23AAA7421C40170500001305FE
:1020D000A5D783C787031747FF1F230DF7B8171727
:1020E000FF1FA307F7409747FF1FA38907B6B7E76E
:1020F000040083A7070882979747FF1F2384A7B68A
:102100001703FFFF6700A3FCB7C7898E938767EDAE
:102110001717FF1F2322F73E45BF1747FF1F03472F
:10212000E7B3795555E79747FF1F938727B303C751
:10213000170005079746FF1FA382E6B203C71700E3
:102140008D463377D7029746FF1FA389E6B083C633
:1021500017001747FF1F1307E7A1184393F6F60F61
:10216000A9EE834787031747FF1F2305F7B085476D
:102170001747FF1F2304F7AE9747FF1F938747AB0F
:102180009C430145998BA9E71703FFFFE702E3F1A1
:1021900037E404007C48C1451745FF1F034585AC63
:1021A00082973C4885451745FF1F0345A5AB82979D
:1021B00001451703FFFF670083F183C717008546BA
:1021C0006395F6008347970379BF8347A70361BFF1
:1021D00082809747FF1F83C767A8A1CF1703FFFF20
:1021E000E702A3EC37E404009747FF1F238807A604
:1021F0007C4885451745FF1F0345C5A682977C4C43
:1022000091451745FF1F0345E5A582977C489145F9
:102210001745FF1F034505A582973C48C145174553
:10222000FF1F034525A4829701451703FFFF6700A1
:1022300003EA795582801703FFFFE70203E72A8448
:10224000035565FF9780FFFFE780401B9747FF1FFF
:102250009387C7A0D847BE841DEF9790FFFFE78004
:1022600080779C48232004009DEB9747FF1F23AFF6
:10227000879E9747FF1F23A9879EB7E70400BC4BA3
:1022800089451745FF1F0345E59D829701451703C3
:10229000FFFF6700C3E3630A8700184375BF80C36D
:1022A0009747FF1F23A4879CC9BF7955CDB7170354
:1022B000FFFFE70283DF9747FF1F938767AC8843E1
:1022C0002326050023240500510597A00000E78080
:1022D000C0331703FFFF670083DF1703FFFFE70229
:1022E000C3DC1744FF1F1304A4A91C40411199CF5C
:1022F0009C472302B5002AC61CC197000000E78056
:1023000040FB1C409C4B99C3324582974101170307
:10231000FFFF6700C3DB1703FFFFE70203D941118B
:10232000444D328532842EC69790FFFFE780C0521D
:102330002AC422859790FFFFE780205403A8440019
:10234000630C0800B245835744001840224683D5E9
:102350004500AA862685029841011703FFFF670002
:1023600003D71703FFFFE70243D4404D1DC808C041
:1023700097050000938565031305440197A00000AD
:10238000E78040169747FF1F9387879F9C4301452F
:1023900089E79747FF1F23A5879E1703FFFF670065
:1023A00003D37D55DDBF1703FFFFE70203D0011103
:1023B00068009305F00F02C602C802CA02CC02CE22
:1023C00097000000E780A0F105611703FFFF670099
:1023D00003D09747FF1F9387A79A9C43D847A167CD
:1023E0009D076319F7021703FFFFE70203CC0111F2
:1023F00032859790FFFFE7802046230AA1008145A0
:10240000680097000000E78080ED05611703FFFF7B
:102410006700E3CB82809747FF1F938767969C43B3
:10242000D847A167938777036319F7021703FFFF64
:10243000E702A3C7011132859790FFFFE780C041F3
:10244000230AA1008145680097000000E78020E989
:1024500005611703FFFF670083C782809747FF1F4F
:10246000938707929C43D84795476316F704170351
:10247000FFFFE70283C30111328532849790FFFF8B
:10248000E780803D230AA10022859790FFFFE78027
:10249000C03E83574400231BA10081453ECC1C4015
:1024A00068003ECE97000000E78060E305611703F7
:1024B000FFFF6700C3C18280930785FF8DC3832719
:1024C000C5FF91CFDC4B81CF1703FFFFE702E3BDD0
:1024D000032585FF82971703FFFF670043BF8280B4
:1024E0001703FFFFE70263BC2A8432859790FFFF42
:1024F000E7808036BD4763EBA70018449377F5006B
:102500000345B70041995D8DA305A7001703FFFFA1
:102510006700E3BB1703FFFFE70223B901117C004B
:102520003ECAB70707003ECC7C003ECE5C4DA9C733
:102530002A8413858700AE8497A00000E780E0FC22
:10254000A1652A899D0548089770FFFFE780603ED6
:102550009305803EB345B902480893F5F50F97906F
:10256000FFFFE780C021014781465008A6852285EC
:102570009770FFFFE780406105611703FFFF670069
:1025800003B51703FFFFE70243B297000000E7809F
:10259000A0F81703FFFF670083B31703FFFFE702ED
:1025A000C3B001117C00AE843ECAA165B707070025
:1025B0002A843ECC48087C00938575033ECE9770F4
:1025C000FFFFE78000371C44480883C5B700BD897A
:1025D0009790FFFFE780A01A500801478146A68523
:1025E00022859770FFFFE780205A05611703FFFFE0
:1025F0006700E3AD1703FFFFE70223AB2A84AE8435
:1026000097000000E78000EEA68522859700000075
:10261000E780E0F81703FFFF670063AB1703FFFFD6
:10262000E702A3A897000000E78060F71703FFFF09
:102630006700E3A91703FFFFE70223A70329C501EA
:102640004111630809022A843285B2849790FFFF02
:10265000E78080202AC626859790FFFFE780E0214B
:10266000832749002A8691C7DC4781C7B245228566
:10267000829741011703FFFF670063A51703FFFF60
:10268000E702A3A2444D91CC2A8432859790FFFFA4
:10269000E780A01EDC40AA8589C79C4799C3228594
:1026A00082971703FFFF670083A21703FFFFE7026C
:1026B000239E032AC5014111630D0A062E89AA84AF
:1026C0009545328532849770FFFFE78080268545E7
:1026D00022859790FFFFE7804004AA89CA8522855A
:1026E0009790FFFFE780A00B83274A008DCBDC4348
:1026F0009DC722859790FFFFE780A00083274A00AF
:10270000104083564400DC437115A307A100B29624
:102710001307F1004E86CA852685829701C523805E
:10272000090001A88345F10022859790FFFFE7800B
:10273000C0FE41011703FFFF6700C3981703FFFFA7
:10274000E702A39665711C083EC2B70780013EC42C
:102750001C0832893EC62A84AE8497000000E780B8
:10276000A0ED4A859790FFFFE78020118357A100D5
:102770008DC3AA855000228597000000E78020F3D2
:10278000014781465000A68522859770FFFFE780AC
:10279000A03F59611703FFFF670063931703FFFF13
:1027A000E702038F65711C088329C5013EC2B70784
:1027B00080013EC41C082A84AE8432893EC697003C
:1027C0000000E780E0EB638A09024A859790FFFFEB
:1027D000E780A00A8357A100AA8585C350002285FF
:1027E00097000000E780A0EC014781465000A685D5
:1027F00022859770FFFFE780203959611703FFFF9B
:102800006700438C1703FFFFE702238A65711C08EA
:102810003EC2B70780013EC42A841C0832853EC6EA
:10282000AE849790FFFFE78040058357A1008DC3DA
:10283000AA855000228597000000E78040E7014705
:1028400081465000A68522859770FFFFE780C03340
:1028500059611703FFFF670083871703FFFFE70234
:10286000C384444D81EC8347450093B71700B307F9
:10287000F0403E851703FFFF670063851845FD574D
:102880006DDB97070000938747032A845CCB97058D
:1028900000009385A5C21385840097A00000E780FF
:1028A00060C480C003474400814761F71737FF1FAA
:1028B000232A974C7DBF17F3FEFFE702637D832930
:1028C000C50141110329850081476387090A032453
:1028D000090191452A8A22859770FFFFE7806005EC
:1028E000854522859790FFFFE78020E38945AA8AE6
:1028F00022859790FFFFE78040E2AA849770FFFF50
:10290000E780400A83A749002A8B8DCB9C439DC753
:1029100022859790FFFFE780C0DE83A74900A306CA
:10292000A1001040835644009C431307D100B29687
:10293000D6851306E1005285829709CD83570B0097
:102940002380F400A183A380F40023800A00A3065F
:10295000010039A88357E10022852380F4008345D4
:10296000D100A183A380F4009790FFFFE780E0DA15
:102970008347D100B337F0000347B9009207014500
:102980003D9BD98FA305F900410117F3FEFF6700B6
:10299000637317F3FEFFE702437141110DED9737A3
:1029A000FF1F9387273E804315C804401309840006
:1029B0009DC95C4099C79C4B89C726852EC68297C6
:1029C000B2459307803EB385F5024A8597A0000083
:1029D000E78060C121A0404DAA8469F8410117F346
:1029E000FEFF6700C36E4A8597A00000E780E0C144
:1029F0005C40EDD7DC4BFDD326858297C5B717F336
:102A0000FEFFE702836A2A8432859790FFFFE78002
:102A1000A0E4AA85228597000000E780C0F717F39D
:102A2000FEFF6700C36A17F3FEFFE70203682A840C
:102A3000AE8497000000E780C0FCA6852285970041
:102A40000000E78060AD17F3FEFF670043680841B0
:102A50003355B5000589828017F3FEFFE702E36472
:102A60001734FF1F130404341C5C011123170100E9
:102A70008D83858BA303F1008327040B23180100AA
:102A80002319010003D7C7013ECA3C002314E1000B
:102A90007D572315E1000357C4023ECC02CE231616
:102AA000E1009770FFFFE78020CE8357E101231EEE
:102AB000A10093F707E093E71710231FF100973762
:102AC000FF1F83C7C73095C305470145638AE700E9
:102AD0008347840393E727001737FF1F2300F7304E
:102AE000056117F3FEFF6700835E814717F700005B
:102AF000130787DB854613067100854548089790C4
:102B00000000E780408F69FD83478403F59B1737FA
:102B1000FF1F2305F72C85471737FF1F2309F72AC7
:102B2000C1B717F3FEFFE7024355973DFF1F938D93
:102B30006D2703A6CD0639712A8981478144930602
:102B400000023357F600058B01C7850493F4F40F98
:102B50008507E398D7FE83A70D0B231701022318DF
:102B6000010203D7C7013EDA3C102314E1027D576E
:102B70002315E10203D7CD023EDC231901022316FF
:102B8000E10202DE9770FFFFE78000C08357E10398
:102B9000231EA102014593F707E093E71710231FB7
:102BA000F1029737FF1F83C78722B9EF9737FF1FBF
:102BB00083C7D7223EC69739FF1F9389A91E0144B8
:102BC000014D9D4A054B954B173CFF1F130CCC2420
:102BD000973CFF1F938CCC2303DAC905630B0A00D3
:102BE000EA8563185903668597000000E78060E670
:102BF0001DC5050DA1478909E310FDFE2DE497379A
